:10000000082003008D7C0200497B02004D7B02002A
:10001000A57C0200A97C0200AD7C0200000000006B
:10002000000000000000000000000000B17C0200A1
:10003000B57C0200000000003D9300005F19020043
:100040000000000000000000B97C0200017B0200FB
:1000500065EA000000000000000000000000000051
:100060000000000000000000957C0200000000007D
:100070000000000000000000B1FC000000000000D3
:10008000B9FD0000FBFD0000A9760200A976020080
:10009000B975020000000000000000000000000030
:1000A000F8B500224FF41261DFF8600B02F0E0F9BE
:1000B000DFF85C4B0022102104F1200002F0D8F997
:1000C000DFF8505B0022182105F10C0002F0D0F996
:1000D0000022082104F1300002F0CAF900220821B0
:1000E00004F1380002F0C4F9002020646064A064C8
:1000F000E0646862A862E862DFF81C6B7063B0635A
:10010000F0632863306470646863A863E863012067
:1001100028640020B064F0644FF0FF306864A86485
:100120000020E864306520657065F06530667066B3
:10013000B066B06202462821304602F099F90020EC
:1001400070600220308100203060DFF8D07A0246F3
:100150000C21384602F08CF9DFF8C40A7860DFF829
:10016000C40A386001203872002028702865688031
:10017000A880E8806065F066A060A065F0626865B0
:10018000A8656066A066E066706730676866286686
:10019000E86501202867E866A8660020E867A86788
:1001A0006867062030860020F067B0672067DFF8B8
:1001B000DC0DE065002020660120A081962068818A
:1001C000062070860C20E0810020B06502464021A8
:1001D00007F10C0002F04CF900220621204602F043
:1001E00047F90022102104F1100002F041F900202B
:1001F000E0616067F1BD10B584B0DFF8204A0C22E1
:10020000214600A802F072F9FFF74AFF0C2200A96C
:10021000204602F06BF91FBD2DE9F0472DED0C8B48
:1002200090B00024254600A821460A460B460EC081
:10023000302102F093F99FEDA98ADFF8D46996ED99
:100240001B0AD6ED140AC6ED1B0ADFF8CC7997ED30
:10025000149A86ED149ADFF8BC8998ED131AB8EE5B
:10026000411ADFED9F1AC1EE819AC7ED149AD8F8B2
:100270004420D8F83490A9EB0200FA30FA21B0FB00
:10028000F1F1FA2303FB110080B2002800F0228470
:100290004C2803DAD8F84010012906D12046F8622C
:1002A0000220A8F8080000F015BCD7F84CA0BAF15D
:1002B000040F24D3F4EE490AF1EE10FA1FD5B4EE80
:1002C000699AF1EE10FA1AD59FED861A20EE811A7E
:1002D000B4EE691AF1EE10FA11D59FED831AF4EE1F
:1002E000419AF1EE10FA0ADB87ED149AC6ED140A72
:1002F00086ED1B0A0320A8F8080000F025BC97ED46
:100300000DAA87ED0EAAD7ED10AAC7ED11AA0146D6
:1003100000EE101AB8EE400AD8ED0B8AC8EE800A3B
:1003200098ED0C1A81EE001A21467963396420E0B9
:10033000521C92B2FA2A00D12246DFF8D03803EBE1
:100340008203D3ED231A71EEE01AD3F8743402EE6F
:10035000103A32EE412AD7ED0D2A41EEA12AC7ED1F
:100360000D2AD7ED101A42EE021AC7ED101A491CD9
:1003700089B28142DCDBD7ED0D0A80EE80BA87EDD1
:100380000DBAD7ED100A80EE80CA87ED10CAD6EDFF
:100390001ABA98ED160AD8ED150A70EEC0CAF5EE35
:1003A00040CAF1EE10FA02DDC6ED1ACA03E030EEE3
:1003B000600A86ED1A0A00F0ADFF012802D120463E
:1003C000F86287E3BAF1000F0BD1B88D052802DB84
:1003D00005462046B885F88D052802DB45192046DC
:1003E000F8851AFA85F0002827D1B6EE00DA3CEE3F
:1003F0002A0A20EE0D0ADFEDA10AB4EE600AF1EE42
:1004000010FA11D43BEE0A0A20EE0D0ADFED9C0A29
:10041000B4EE600AF1EE10FA06D4B3EE040AF4EE7C
:1004200040CAF1EE10FA08D5B88D401CB885C8F85E
:1004300048900620A8F808004CE3B88D002802D0A8
:1004400045192046B8851AFA85F000281BD1B7EE69
:10045000000AF4EE409AF1EE10FA03D50720A8F84E
:10046000080037E39FED870AF4EE409AF1EE10FAA8
:1004700006DBF88D401CF8850820A8F8080029E361
:100480002046F88503E0F88D45192046F885284672
:1004900080B200F0E3FF012808D187ED149AC7ED80
:1004A00010AAC6ED1ABA87ED0DAA13E39FED760ADE
:1004B000F4EE409AF1EE10FA02DBDFF8380C386502
:1004C0002046B885BAF1000F10D1386D786587EDF8
:1004D0000FBAB06E706600F0B5FE40E0000000009C
:1004E00000007A446666E63F01004040B6EE00DA5E
:1004F00000F0A8FE012816D197ED140AF0EE000ACC
:1005000020EE200A87ED140A6BEE0D0AC7ED0D0AE6
:100510002CEE0D1A87ED101AC7ED0E0A87ED111A91
:1005200086ED140A6D1C97ED140AD6ED140A30EE10
:10053000200A20EE0D0A87ED150A97ED0D0AD7ED7A
:100540000E0A30EE200A20EE0D0A87ED0F0A96ED16
:100550001A0A3BEE800A20EE0D0A86ED190A98F879
:100560000100012840F0AB82D8F80C00009000A8F0
:10057000D8F810104160D8F814108160214617E0B7
:1005800000AB03EB820393ED010A50F822C000EEAA
:1005900090CAB4EE600AF1EE10FA05D500EB820CB9
:1005A0008CED000AC3ED010A521C022AE8DB491C4B
:1005B000022901DA2246F8E79DED000AB5EE400A6D
:1005C000F1EE10FA2AD5B5EE400AF1EE10FA01DC90
:1005D000B1EE400AD0ED020A30EE800A80ED020A48
:1005E0009DED000AB5EE400AF1EE10FA01DCB1EE25
:1005F000400AD0ED010A30EE800A80ED010A9DED3F
:10060000000AB5EE400AF1EE10FA01DCB1EE400A44
:10061000DDED000A30EE800A8DED000A90ED010A52
:10062000D0ED020A30EEC01ADDED000A30EE600AAD
:10063000B4EE401AF1EE10FA05D5F0EE410AB0EE34
:10064000401AB0EE600AD6ED0C0AC6ED0D0A31EE86
:10065000400A80EE010A9FED0D1A20EE010A86ED98
:100660000C0AB06BF063F4EE400AF1EE10FA0FD50D
:1006700070EE600AC6ED0E0A0EE000BF00001643E1
:100680000000A042666616400100A0400000C8427B
:1006900070EEC00AC6ED0E0A386F796F081800EBCD
:1006A000D070401002EE100A86ED102AC6ED118AB5
:1006B000D7ED100AC6ED120AD7ED141ADFF8500C68
:1006C000C0EDC41A96ED131A31EE611AD6ED132A55
:1006D00072EEE12A21EE221A00F5447181ED011A31
:1006E000C6ED131AD7ED1B1AC1ED021AD8F818106F
:1006F000039103A9C1ED011AC1ED020AC1ED038AFC
:10070000C1ED041AC1ED058AC1ED061AB8EEC22A80
:1007100081ED072AC1ED081A81ED090AC1ED0A1A17
:1007200081ED0B1ADDED032A9FEDD03A62EE832AAC
:100730009FEDCF3A41EE832A9FEDCE3A20EE833AE9
:10074000DFEDCD3A08EEA33ADFEDCC3A61EEA33A05
:100750009FEDCB4A48EE843A9FEDCA4A21EE844A87
:10076000DFEDC94A02EE244ADFEDC84A61EEA44A31
:100770009FEDC75A40EE054A9FEDC65A21EE855AB5
:10078000DFEDC55A01EE255AF8EE085AF4EE652A57
:10079000F1EE10FA00F19381DFEDC05AB4EE653A44
:1007A000F1EE10FA00F18B81DFEDBD5AF4EE653AFF
:1007B000F1EE10FA00F18381DFEDBA5AB4EE654A2A
:1007C000F1EE10FA00F17B819FEDB76AF4EE464A34
:1007D000F1EE10FA00F173819FEDDE6AB4EE465A35
:1007E000F1EE10FA00F16B81DFEDDB6AF4EE662AC0
:1007F000F1EE10FAC0F26381DFEDD82AB4EE623A6E
:10080000F1EE10FAC0F25B81F4EE653AF1EE10FA07
:10081000C0F25581B4EE464AF1EE10FAC0F24F81B3
:10082000F4EE654AF1EE10FAC0F24981DFEDCC2A10
:10083000B4EE625AF1EE10FAC0F24181DFEDC92A3E
:100840009DED033AB4EE623AF1EE10FA01D5CDED2A
:10085000032ADDED032A9FEDC43AF4EE432AF1EEBC
:1008600010FA02DBDFF8E82B0392DFEDD52AF4EE75
:10087000621AF1EE10FA01D5C1ED012A9FEDD13ACD
:10088000DFEDBA3A91ED014AB4EE634AF1EE10FAA7
:1008900001DB81ED013A9FEDB64AF4EE440AF1EE38
:1008A00010FA01D581ED024AD1ED020A9FEDB14A5D
:1008B000F4EE440AF1EE10FA02DBDFF8982B8A60BE
:1008C000DFEDC10AF4EE608AF1EE10FA01D5C1ED58
:1008D000030A9FEDBE4AD1ED034AF4EE444AF1EE1D
:1008E00010FA02DBDFF8702BCA60F4EE621AF1EE48
:1008F00010FA01D5C1ED042AD1ED044AF4EE634AA1
:10090000F1EE10FA01DB81ED043AF4EE608AF1EECB
:1009100010FA01D5C1ED050AD1ED050AF4EE440A3D
:10092000F1EE10FA02DBDFF8302B4A61F4EE621AC6
:10093000F1EE10FA01D5C1ED062AD1ED060AF4EE6A
:10094000630AF1EE10FA01DB81ED063AF1EE000ADE
:10095000B4EE602AF1EE10FA02D54FF08142CA617E
:10096000D1ED070A9FEDA32AF4EE420AF1EE10FA48
:1009700002DBDFF84C2CCA61F4EE621AF1EE10FAD9
:1009800001D5C1ED082AD1ED080AF4EE630AF1EEB3
:1009900010FA01DB81ED083ADFED970AB4EE600A48
:1009A000F1EE10FA01D5C1ED090A91ED090ADFED6A
:1009B000930AB4EE600AF1EE10FA02DBDFF8442C81
:1009C0004A62F4EE621AF1EE10FA01D5C1ED0A2A7C
:1009D00091ED0A0AB4EE630AF1EE10FA01DB81ED43
:1009E0000A3AB5EE401AF1EE10FA01D52246CA6273
:1009F00091ED0B0ADFED820AB4EE600AF1EE10FA17
:100A000002DBDFF8042CCA62214612E01B1FD3ED83
:100A1000000A92ED031AF4EE410AF1EE10FA01D544
:100A20009FED780AB8EEC00AD2ED020A00EE208AE5
:100A3000491C31293ADA9FED740A0B011A18D2F8D1
:100A400004C0BCF1010F0DF10C0C1B580CEB83031F
:100A5000DCD11B1FD3ED000A92ED031AF4EE410A1C
:100A6000F1EE10FADEDB9FED670ADBE7168733BD98
:100A7000B0568DBD03275BB9E23C9CB9983115BED9
:100A8000BF49D3B97061FDBD55C128BC36CB05BE89
:100A90003D7FDABBDDED0ABEE4BE353E6666A6BF2D
:100AA0003333F3BFCDCC4CBFCDCC8CBFB5EE408A39
:100AB000F1EE10FA03DD0F20A8F808000AE097ED28
:100AC000150A284680B200F0AFF800F055F8044649
:100AD000C8F84890C8F844900020C8F84C00C8F8FE
:100AE0002C00C8F83000C8F840000246102106F17A
:100AF000200001F0BDFC00220C2108F10C0001F0E7
:100B000031FDDFF88804F06500203066F8880028A1
:100B10001AD1F86F00280CD0B86CF968401A398ED9
:100B2000B0EB510F02DB002038810DE0012038814D
:100B30000AE0B88DF98D11FA80F0032802DB01205C
:100B4000388101E002203881204610B0BDEC0C8BCA
:100B5000BDE8F087333333BFCDCC0CC09A9919BFB1
:100B6000CDCC4CBE5017C93FC9AC454216E66840D3
:100B70007D90A341A2F2924438B50025DFF81C4CC9
:100B80000120E06700F01EFD2060E06C218E8842AD
:100B900014D3A06CE060208DA080608DE080A06DFB
:100BA0006061E06DA061206EE061606E2062A06E09
:100BB00060620120A0672846E0670125284632BD13
:100BC000A9F56E3E15E66840BA9F17443564EC44BB
:100BD0001148C16881640021C16441600221018122
:100BE00000218162C1690166416A81660021C16795
:100BF00070470000010058427B4D4F3D47FFC74200
:100C0000BEBA984101000000FFFFFFFF1467030018
:100C1000905B0300905A0300105B030080D2030036
:100C200000002F43000070422DE9F84F2DED048B9A
:100C300082B08346002213461046DFF8604BE56C15
:100C400005F10F0101F00F01EE1D06F007060096F9
:100C5000DFF8506B06EB810787ED030ABBF1000F4D
:100C600018D0074614E0A1F1010CACEB070C0CF115
:100C7000100C4FEAEC0E0CEB1E7E4FEA2E1EBCEB66
:100C80000E1C03D406EB8C0C8CED030A7F1C3FB2C8
:100C90005F45E8DB102D02D2294609B200E00F21A2
:100CA0009FEDBB8ADFEDBA0A9FEDBA1A07461BE03B
:100CB00006EB810CDCED031AF5EE401AF1EE10FAAA
:100CC00010DD38EE218AF4EE610AF1EE10FA01D55A
:100CD000F0EE610AF4EE411AF1EE10FA01D5B0EE31
:100CE000611A7F1C491E09B20029E1D53FB239467D
:100CF00003290BDB78EE600A70EEC10A891E01EE53
:100D0000101AB8EEC11A80EE818A07E0012905DBCE
:100D100000EE907AF8EEE00A88EE208AB5EE408A7E
:100D2000F1EE10FA01D0002F01D1B0EE408A84ED2F
:100D3000168A9FED990AB4EE408AF1EE10FA02D5B8
:100D4000B0EE408A08E09FED950AB4EE408AF1EEDD
:100D500010FA01DBB1EE028AB0EE040AB4EE408A6A
:100D6000F1EE10FA08D494ED1B0AF0EE080AB4EE86
:100D7000600AF1EE10FA02D50321218501E0042179
:100D80002185A76C07F00709DFF8208A09EB080E18
:100D9000218D8EF8B818BBF1000F0BD0A7F1010C14
:100DA0000CF0070CC44407F0070AC2449AF8B8A82C
:100DB0008CF8B8A84FF0080C10E0BAF1040F00D17D
:100DC000401CA9F101090FFA89F9B9F1000F01D509
:100DD00009F10809ACF1010C0FFA8CFCBCF1010F10
:100DE00016DB0FFA89F909EB080A9AF9B8A8BAF1E3
:100DF000030F01D15B1C03E0BAF1040F00D1521CB8
:100E0000BCF1060FDDDBBAF1030FD6D1401ED8E7E7
:100E1000B4F82AC092B29BB29A4207D3934202D24C
:100E2000042060850DE000B2002802D50320608513
:100E300007E0012802DB0420608502E09EF9B80883
:100E40006085B4F82A90B9F1040F01D1104600E092
:100E50001846CC4509D000202081E088002820D108
:100E6000042D1ED3012020811BE012FA83F2012AF7
:100E700015DB052A10DB00EE102AB8EEC00AF6EEEC
:100E8000080A20EE200A00EE900AF8EE600AF4EE5E
:100E9000400AF1EE10FA02D50120208101E0022083
:100EA000208149B2B0EE480A304600F025F9DFED66
:100EB000900AB4EE600AF1EE10FA01D5B0EE600AC5
:100EC00084ED170A584600F1010A00EE90AAF8EEE8
:100ED000E08AD4ED180A48EE800AC4ED180A9FEDA6
:100EE000CE9A20EE080A20EE090A009908EB81014B
:100EF00001F65C0181ED000ABBF1000F1AD04FF042
:100F0000000C15E00099491EA1EB0C0108318A1074
:100F100001EB5272D210B1EBC20105D408EB810192
:100F200001F65C0181ED000A0CF1010C0FFA8CFC5A
:100F30008445E7DB082D02D2284600B203E00720F3
:100F400001E0401E00B20028FBD584ED190A494695
:100F500049B2304600F048F968EE090AB7EE001AC7
:100F6000C1EE200A20EE800AD4ED1A0A48EE800A6B
:100F7000C4ED1A0A0AEB0700A0640AEB0500E0645E
:100F800002B0BDEC048BBDE8F18F000000007A4494
:100F9000000000000000C8426666A63F01009040C5
:100FA00049B2032944D1DFED9D0AB4EE600AF1EEA7
:100FB00010FA01DBB0EE600A9FED991ADFED990A95
:100FC00040EE010A90ED011A9FED970AB4EE401A27
:100FD000F1EE10FA43DADFED951AB4EE611AF1EE94
:100FE00010FA74DBB4EE401AF1EE10FA6FD59FEDF3
:100FF000900A31EE000ADFED8F1A60EE211A9FEDA4
:101000008E0A9FED8E2A01EE002A22EE200A20EEA3
:10101000210A9FEDB72ADFEDB72A41EE022A62EEE0
:10102000A00AB7EE001A31EE611A00EE810A56E00E
:10103000DFED830A60EE200A60EE800A9FEDAE1AB3
:1010400040EE410A9FEDAD0A70EE800A90ED011A64
:101050009FED750AB4EE401AF1EE10FA0ADB90ED3E
:10106000010A9FED751ADFED751A40EE011A21EEA7
:10107000A00A34E0DFED6D1AB4EE611AF1EE10FA59
:1010800025DBB4EE401AF1EE10FA20D59FED680A88
:1010900031EE000ADFED671A60EE211A9FED660A55
:1010A0009FED662A01EE002A22EE200A20EE210A98
:1010B0009FED8F2ADFED8F2A41EE022A62EEA00A11
:1010C000B7EE001A31EE611A00EE810A07E090EDEA
:1010D000010A20EE800ADFED8A0A20EE200A007A5B
:1010E000022803D1DFEDD10A20EE200A704700006C
:1010F000CDCC4C3E0000A04010B52DED028BB0EEE3
:10110000408A0C46DFED7F8A49B2FFF749FF64B29F
:10111000042C31D1DFED7C0AB4EE608AF1EE10FAD6
:1011200016DBB1EE021AB4EE418AF1EE10FA0FD5D9
:10113000DFED760A78EE200AB1EE041A60EE810A3D
:10114000FCEEE00A10EE900AC01D08EE900A3DE0A9
:10115000B4EE608AF1EE10FA03D5072008EE900A8B
:1011600034E0F1EE020AB4EE608AF1EE10FA2DDB03
:10117000122008EE900A29E0F7EE080AB4EE608A21
:10118000F1EE10FA11DBDFEDAA0AB4EE608AF1EE9F
:1011900010FA0AD5FFEE080A78EE200AB1EE041A1A
:1011A00060EE810AFCEEE08A10E0F7EE080AB4EE89
:1011B000608AF1EE10FA09D4DFED9D0AB4EE608A80
:1011C000F1EE10FA02DB062008EE900ADFF8FC0CC4
:1011D00018EE901A00EB8100D0ED000A20EE200AF4
:1011E000BDEC028B10BD0000F0EE0C0A49B20429E0
:1011F00004D19FED901A40EE010A03E09FED8E1A94
:1012000040EE010A9FED8D0A20EE800AD0ED000A23
:1012100020EE200A70470000000070429A991940A1
:101220006ADEF13D8638163F00002A43000016436F
:10123000000016C3CDCC4C3D4260E53A6666263FC1
:101240002575C23E0020DFF8541591ED140AF7EE23
:10125000040AB4EE600AF1EE10FA47DADFF8702CF7
:10126000D288042A42DAD1ED150A9FED751A60EE94
:10127000810AB4EE600AF1EE10FA03D5022A01DB0E
:10128000012012E0DFF84C1C91ED0B0ADFED6D0A36
:10129000B4EE600AF1EE10FA07DBDFED6B0AB4EE94
:1012A000600AF1EE10FA00D5012001281ED1DFF806
:1012B000241C91ED170AD1ED180A70EEC00A9FEDBB
:1012C000631AF4EE410AF1EE10FA07DBF7EE080AB2
:1012D000B4EE600AF1EE10FA00D50020DFEDC50A89
:1012E000B4EE600AF1EE10FA00D50020704700005D
:1012F00052491D3BB81E053F7593E83F2497534064
:10130000C1C0C03B0000000066660640666606C0BD
:10131000A05003000021DFF88424538D032B1FDA33
:1013200092ED140ADFEDA50AB4EE600AF1EE10FAB0
:1013300016DB92ED0D0AF2EE040AB4EE600AF1EE4D
:1013400010FA0DD592ED100ADFEDAB0AB4EE600A8B
:10135000F1EE10FA04D50421DFF8743B1981012164
:1013600092ED100AF6EE000A92ED111A30EE011A13
:1013700021EE201AF3EE0E1AB4EE611AF1EE10FA15
:101380001CD492ED0D1AD2ED0E1A71EE211A61EEF7
:10139000A01AB2EE042AF4EE421AF1EE10FA0DD4BD
:1013A000F3EE041AB4EE610AF1EE10FA06D4B1EECF
:1013B000040AB4EE401AF1EE10FA04D50521DFF864
:1013C000103B1981012192ED140A9FED8C1AB4EEA5
:1013D000410AF1EE10FA27DBDFF8F82A92ED0A0A4B
:1013E00092ED0B1A80EE010A9FED851AB4EE410AC8
:1013F000F1EE10FA18DB00EE100AB8EE400A20EE0B
:10140000200AD2ED080AF4EE400AF1EE10FA0BD5EC
:10141000D2ED090AF4EE400AF1EE10FA04D50E20DE
:10142000DFF8AC1A08810121084670473333733F57
:101430009A993940CDCC4C3ECDCCCC3D0AD7A33B7C
:101440003333333F010020420000C8420100C03F57
:10145000C8AC4542A1F292443464EC4401460020F9
:10146000CE4AD36C13FA81F102291AD392ED140AF1
:10147000DFED8F0AB4EE600AF1EE10FA11DB92EDA7
:10148000110AD2ED100A80EE200ADFED8A0AB4EECE
:10149000600AF1EE10FA04DB0920DFF8343A188113
:1014A000012002291CD39FED840AD2ED110A92ED8E
:1014B000101AC0EE810AF4EE400AF1EE10FA0FDBCA
:1014C000D2ED0E0A92ED0D1AC0EE810AF4EE400A3A
:1014D000F1EE10FA04DB0A20DFF8F439188101205C
:1014E000002913D0DFF8EC1991ED190ADFEDA50AF8
:1014F00020EE200AD1ED1A0AF4EE400AF1EE10FABD
:1015000004D50B20DFF8C8190881012092ED140AD8
:10151000DFED9D0AB4EE600AF1EE10FA08DA92ED02
:10152000150ADFED9A0AB4EE600AF1EE10FA1EDB3E
:1015300092ED100ADFED960AB4EE600AF1EE10FAB1
:101540000DD492ED0D0ADFED930AB4EE600AF1EED0
:1015500010FA04D4DFF87819C988022907DB518D05
:10156000032904DB0C20DFF868190881012092EDC3
:101570000F0ADFED870AB4EE600AF1EE10FA08D424
:1015800092ED1B0AF1EE040AB4EE600AF1EE10FAD5
:1015900012D5116F526F511800EE101ABAEEEF0A01
:1015A000DFED7D0AB4EE600AF1EE10FA04DB0D20E7
:1015B000DFF81C190881012070470000010000407D
:1015C00000005842002075498A6C12F1640F0FD256
:1015D0009FED730AD1ED180AF4EE400AF1EE10FA0D
:1015E00006DAD1ED1A0AF4EE400AF1EE10FA00DB49
:1015F0000120704785EB113F000020420100404070
:101600003433333F46FFC742BDBA984110B4014658
:101610000020DFF8C028654BD3F8144900EE104ACB
:10162000D1ED000AB4EE600AF1EE10FA08D1147898
:10163000641C1470E4B2FE2C04DB3224147001E04C
:101640000446147003F6141393ED010AD1ED010A58
:10165000B4EE600AF1EE10FA08D15478641C5470AC
:10166000E4B2FE2C04DB3224547001E004465470D2
:1016700093ED020AD1ED020AB4EE600AF1EE10FA1F
:1016800008D19178491C9170C9B2FE2904DB32213E
:10169000917001E0014691701178322905DA517894
:1016A000322902DA9178322900DB012010BC704720
:1016B000010060400100A04001007041014600208F
:1016C00091ED000AB5EE400AF1EE10FA01DCB1EE40
:1016D000400ADFF80028DFED340AB4EE600AF1EECC
:1016E00010FA08DBD3785B1CD370DBB2FE2B04DB73
:1016F0003223D37001E00346D37091ED010AB5EEB9
:10170000400AF1EE10FA01DCB1EE400AB4EE600AD4
:10171000F1EE10FA08DB13795B1C1371DBB2FE2BC0
:1017200004DB3223137101E00346137191ED020AC9
:10173000B5EE400AF1EE10FA01DCB1EE400AB4EE6B
:10174000600AF1EE10FA08DB5179491C5171C9B2F7
:10175000FE2904DB3221517101E001465171D1783B
:10176000322905DA1179322902DA5179322900DB7E
:1017700001207047DFF89C0CC0697047DFF8940CBB
:10178000006970479A99993E01009040010080409D
:101790000000C8430000164301008C42105B0300A8
:1017A0008096184B80D2030035336B4114670300D9
:1017B0002DE9F84F2DED068B86B0814688464FF017
:1017C000000A9FEDD88ADFEDD78A9FEDD69ADFED2C
:1017D000D59ADFF8444CE088ADF81000A088ADF849
:1017E00002002089ADF800005046019005464846A9
:1017F000FFF70CFF03904846FFF760FF0290DFF809
:10180000D06628467065B0653081B06EDFF80C7C1C
:10181000D7F8141900EE101AD9ED000A30EEC01AEC
:1018200001EE900AF8EEE11A21EE211AB5EE401A07
:10183000F1EE10FA1BD596ED1D1A70EE411AF5EE79
:10184000401AF1EE10FA01DC71EE401A9FEDB61A63
:10185000F4EE411AF1EE10FA05DB216F491C216705
:10186000F16D491CF16586ED1D0A4042B06607F630
:10187000141090ED010AF16E99ED011A31EE401A43
:1018800001EE901AF8EEE11A21EE211AB5EE401A97
:10189000F1EE10FA1BD596ED1E1A70EE411AF5EE18
:1018A000401AF1EE10FA01DC71EE401A9FED9E1A1B
:1018B000F4EE411AF1EE10FA05DB226F521C22679A
:1018C000326E521C326686ED1E0A4942F16690ED78
:1018D000020A306F99ED021A31EE401A01EE900AB9
:1018E000F8EEE11A21EE211AB5EE401AF1EE10FAE7
:1018F0001BD596ED1F1A70EE411AF5EE401AF1EE67
:1019000010FA01DC71EE401A9FED871AF4EE411ACD
:10191000F1EE10FA05DB216F491C2167716E491C3D
:10192000716686ED1F0A404230673078052805D180
:1019300001203064284630707080B080F06C4044E4
:10194000F064706B716C884201D101203064B06B1F
:1019500000EB400107EB810B0BF6C000C0ED000A65
:10196000D9F804104160D9F8081081604146484612
:1019700000F0B2FA2061DFF85C850398012802D0FC
:101980000298012836D19FED670ADBF8C00800EE07
:10199000900A60EEA00ADBF8C40801EE100A21EEFE
:1019A000011ADBF8C80801EE900A61EEA11A98F856
:1019B0000000322805DA98F80300322801DA30EE08
:1019C000800A98F80100322805DA98F804003228D5
:1019D00001DA30EE010A98F80200322805DA98F8A8
:1019E0000500322801DA30EE210A00F025FDB0EEC4
:1019F00040AA37E00BF50C60D0ED020A90ED011A19
:101A0000DBF8C00800EE100A20EE000A01EE010A21
:101A100000EEA00A00F010FDB0EE40AAD9ED010AD8
:101A200099ED000A20EE000A00EEA00A00F004FD85
:101A3000F0EE408AD9ED020A99ED010A20EE000A83
:101A400000EEA00A00F0F8FCB0EE409AD9ED020AD0
:101A500099ED000A20EE000A00EEA00A00F0ECFC6E
:101A6000F0EE409AF06B002824D128460CE007EBFA
:101A7000800181ED15AA07EB8002C2ED008A81ED9D
:101A8000079AC1ED0E9A401C0728F0DBF068B061A0
:101A90003069F06170693062B1EE0C0A68EE800A5C
:101AA000C6ED030A69EE000AC6ED040A29EE800AB3
:101AB00086ED050AB06B07EB800181ED15AA07E002
:101AC00007EB8A0090ED150A38EE008A0AF1010A48
:101AD000BAF1070FF4DB86ED098A96ED090A706BFF
:101AE00007EB800080ED230AD6ED0B0A70EE800A2A
:101AF000C6ED0B0AF268B2613269F2617269326254
:101B0000B26B07EB8202C2ED008A81ED079AC1ED4C
:101B10000E9A2A46DFED030A9FED021ADFED011A45
:101B200013E000BF00000000CECC4C3E07EB820368
:101B300093ED002A70EE820A93ED072A31EE021A25
:101B400093ED0E2A71EE821A521C072AEEDBC6EDC7
:101B5000030A86ED041AC6ED051AD1ED1C0A70EED3
:101B6000600A00F27442C2ED000A81ED1C0AD6ED53
:101B70000C0AD0F8742401EE102A70EE810AC6ED2A
:101B80000C0AD9ED000AF5EE400AF1EE10FA01DC7C
:101B9000F1EE600A9FEDCB1AF4EE410AF1EE10FA75
:101BA0001BDAD9ED010AF5EE400AF1EE10FA01DC7C
:101BB000F1EE600AF4EE410AF1EE10FA0DDAD9ED19
:101BC000020AF5EE400AF1EE10FA01DCF1EE600ACD
:101BD000F4EE410AF1EE10FA08DB0122C8F81C20ED
:101BE000D8F8102042F00102C8F81020B4EE41AA43
:101BF000F1EE10FA04DAB5EE40AAF1EE10FA08D5CB
:101C00000122C8F81C20D8F8102042F00202C8F8BF
:101C10001020B5EE400AF1EE10FA08D50122C8F8FE
:101C20001C20D8F8102042F00402C8F810209FEDC4
:101C3000A60AD1ED1C0AF4EE400AF1EE10FA08DB18
:101C40000121C8F81C10D8F8101041F00801C8F89C
:101C50001010D0ED230AF4EE400AF1EE10FA08DB82
:101C60000121C8F81C10D8F8101041F01001C8F874
:101C70001010D0F8741400EE101AD8ED050AF4EE26
:101C8000400AF1EE10FA10D1D8F81810491CC8F823
:101C90001810FB290CDB0121C8F81C10D8F8101013
:101CA00041F02001C8F8101002E02946C8F81810C9
:101CB00088ED050AD8F81C10012901D12846FCE05E
:101CC00007F6141199EC030A81EC030AD8F8701096
:101CD000012906D101203064284630707080B08020
:101CE0007CE0316D491C31653278012A01D0032A2C
:101CF00037D102292AD2628D042A27DAE16C002921
:101D00006CD196ED0A0ADFEDD70AB4EE600AF1EE67
:101D100010FA08D5D0F8741401EE101AB4EE601A57
:101D2000F1EE10FA0FDAF9EE0C0AB4EE600AF1EEF9
:101D300010FA53DBD0F8740400EE100AB4EE600A17
:101D4000F1EE10FA4AD50120306447E0272908D384
:101D50007288002A03D011FA82F14B2901D30121A4
:101D60003164D0F8740400EE900A96ED0A0A00F08F
:101D70007BF9D8F87400401CC8F87400FB2805DB18
:101D80000120307030647080B08030653078012878
:101D900024D17088002821D0B18800291ED00322C8
:101DA00011FA80F03D2801DB01203064608D0428A9
:101DB00000DB0222F088824201D2012030642846F2
:101DC00070663066F065FEF727FA0190206F606755
:101DD00028462067B080F080C8F87400706BB16C42
:101DE000401AFA304FF0FA084146B0FBF1F108FB17
:101DF00011007189884201D100F037FA706BB16C23
:101E0000401AFA304146B0FBF1F108FB110064289A
:101E100001D100F06BFAE088BDF81010814204D1C6
:101E2000BDF80210A288914200D00125002812D0EE
:101E3000706BB16C401AFA304146B0FBF1F108FB0F
:101E40001101322902D10120208114E04B2912D145
:101E5000002020810FE0A08800280CD0706BB16CAE
:101E6000401AFA304146B0FBF1F108FB11007D2821
:101E700001D101202081BDF800002189884200D0D5
:101E80000125706B07EB8001D1F87414B162401C1E
:101E90007063FA2801D100207063B06B401CB063FE
:101EA000072801D10020B063F06B401CF06301985B
:101EB0002843401E8041C043C00F06B0BDEC068BD6
:101EC000BDE8F28FC4F51C430C578944D85C03006D
:101ED000905A0300905B030010B4DFF8402590EDAA
:101EE000000AD2F8143900EE903A30EE600A02F699
:101EF0001413D0ED010A93ED011A70EEC10A90EDB2
:101F0000021AD3ED021A31EE611AB5EE400AF1EE73
:101F100010FA02DDF0EE401A01E0F1EE401AF5EEA3
:101F2000400AF1EE10FA02DDB0EE602A01E0B1EEF7
:101F3000602AB5EE401AF1EE10FA02DDF0EE412A09
:101F400001E0F1EE412A71EE821A71EEA21AB5EEAD
:101F5000400AF1EE10FA01DCB1EE400ADFF8B404F9
:101F600090ED082A32EE000A80ED080AF5EE400AEC
:101F7000F1EE10FA01DCF1EE600A90ED090A30EEA4
:101F8000200A80ED090AB5EE401AF1EE10FA01DCE4
:101F9000B1EE411A90ED0A0A30EE010A80ED0A0A0C
:101FA00090ED0B0A30EE210A80ED0B0ADFF8703459
:101FB000DB6B002B12D1002306E002EB840404F655
:101FC0007C04C4ED001A5B1C9BB21C460F2CF4DB96
:101FD000B2EE0E0A21EE800A80ED150A038902EBAB
:101FE0008302D2F87C4800EE104A31EEC00AD0EDF0
:101FF000150A30EE200A80ED150A02F67C02C2EDC9
:10200000001AF2EE0E0A80EE200ADFF80C2482EDB0
:102010001B0AD0ED170AB4EE600AF1EE10FA01D5F2
:1020200080ED170AD0ED180AF4EE400AF1EE10FA2E
:1020300001D580ED180ADFEDAB0AB4EE600AF1EECF
:1020400010FA03D5826D8918816501E00021816550
:10205000591C018189B20F2901D100210181806DB4
:1020600010BC70470100E0409FED9F1ADFF8A80305
:10207000408D042801DBB0EE001ADFF8A403B5EEB2
:10208000400AF1EE10FA07DBF5EE400AF1EE10FA25
:1020900002D5C188491CC1800178002905D00229D8
:1020A00060D02DD3032976D0B0E0F1EE0C1A31EEDA
:1020B000211AB4EE401AF1EE10FA0BDBB4EE601AFE
:1020C000F1EE10FA06D5016D1029C0F08F800021C5
:1020D00001658BE0416BDFF8442302EB8101D1F80D
:1020E000741401EE901ADFF83C1391ED010AF4EE3E
:1020F000401AF1EE10FA40F18980C1ED011A85E035
:10210000416BDFF8182302EB8101D1F8741401EE62
:10211000901ADFF8101391ED002AB4EE612AF1EE67
:1021200010FA01D5C1ED001AF7EE001AB4EE610AFB
:10213000F1EE10FA6ADBB7EE000AF4EE400AF1EEB7
:1021400010FA63D5016D418000210165B9EE0C0ADA
:1021500030EE410AF4EE400AF1EE10FA10D40221FA
:10216000017053E0F9EE0C1A31EEC11AB4EE410AD7
:10217000F1EE10FA4ADBF4EE410AF1EE10FA45D521
:1021800003210170A549426B01EB8201D1F874145F
:10219000A44A51603AE0416BA04A02EB8101D1F8B8
:1021A000741401EE901A9F4991ED012AF4EE421A3F
:1021B000F1EE10FA01D5C1ED011ADFED831AB4EE8C
:1021C000610AF1EE10FA21D5F4EE610AF1EE10FA8F
:1021D0001CDB016D818000210165B1EE0C0A31EE3E
:1021E000000AB4EE600AF1EE10FA0ED5012101707A
:1021F0008C490A6842654A688265884A436B02EBEB
:102200008302D2F874240A6000E0017000787047FD
:1022100000280CD0C168804AD160916490ED070A13
:1022200082ED070A406A506282ED180A9066704794
:10223000002803D07849282200F058B970470028B8
:1022400006D0794942684A6002680A60007A0872DA
:10225000704780B5002801D1002002BD54220146FC
:10226000724800F043F9012002BD10B56A4C608D40
:10227000218D002904D0002802D00020208106E012
:10228000084302D00120208101E0022020810020AB
:10229000E06420626061A0802085E0626065A065E6
:1022A00002464021624800F0E3F8E06F012801D1C6
:1022B000FEF78EFC57484189002909D0628E8A4278
:1022C00001D2218600E02286002141810846A067D4
:1022D000A06F012801D1608E20860020A06710BD6C
:1022E00000000000EC51383E0000000010B54A4CE0
:1022F000608D218D002904D0002802D0002020818B
:1023000006E0084302D00120208101E00220208164
:102310000020206260616085E08002460821454817
:1023200000F0A6F80020E062E06F012801D1FEF77E
:102330004FFCA06F012801D1608E208610BD80B5B2
:10234000012034490867FFF7D1FFFFF78EFFBDE892
:10235000014003E000202F49086770472D48C089DD
:102360002D49098E814200D200E070472A49CA6C8B
:102370000B8E9A4203D20886002088677047254951
:10238000488170472448C16C002904D1818DC08DDB
:1023900010FA81F0704700207047014600200029A4
:1023A00002D0012901D0704702E01B48C06C704781
:1023B0001948018EC26C891A828D891AC08D081A3B
:1023C00000D5002070470000FEFF7FBF38B50446EF
:1023D0001348104D1049012C06D106224A860C22C2
:1023E000EA819622428105E007224A860F22EA818D
:1023F00064224281A889A04209D0088E082803DA05
:10240000488EFFF7B3FF02E0E889FFF7AFFFAC812A
:1024100031BD0000905B0300105B030014670300F4
:10242000905A030020DA030080D20300D85C030036
:102430008CD20300CC6F030081B08DED000A0098B0
:10244000401000F1FE500090DDED000AC0EE200AC1
:102450009DED001A70EE810ACDED000AB5EE001A6E
:10246000DDED001A80EE210A00EE810A01B070470E
:1024700062F30F2262F31F4200B500BF13009646BD
:102480009446103928BFA0E80C50FAD85FEA417C86
:1024900028BF0CC048BF40F8042BC90728BF20F84C
:1024A000022B48BF00F8012B00BD50F8041B61B19E
:1024B00050F8042BD30744BFA9F101039A18002355
:1024C000091F42F8043BFAD1EFE7704762B38B076C
:1024D00008D0521E11F8013B00F8013B00F02480A7
:1024E0008B07F6D1830740F0208000BF103A07D356
:1024F00030B4B1E83810103AA0E83810F9D230BC46
:10250000530724BFB1E80810A0E8081044BF51F8F1
:10251000043B40F8043BD20724BF31F8022B20F8DB
:10252000022B44BF0B7803707047083A07D3B1E819
:102530000810083A40F8043B40F804CBF7D25307A0
:10254000E4E78268521C8260426832B10268531C20
:10255000036011704168491E416070470022FFF717
:102560008BBF000062F30F2262F31F42401810F08D
:10257000030308D0C91A1FD3DB0748BF00F8012D99
:1025800028BF20F8022D130030B414461546103928
:1025900028BF20E93C00FAD8490728BF20E90C00F1
:1025A00048BF40F8042D890028BF20F8022D48BFFD
:1025B00000F8012D30BC7047C91818BF00F8012D74
:1025C000CB0728BF00F8012D7047000010B50FF2AF
:1025D000740001F081FBDFF8844C0020A073208799
:1025E000E06502464021DFF8980DFFF741FF012228
:1025F0003C21AA2001F09EFD00206074E073024699
:1026000004F18001012002F001FB002805D00FF247
:10261000440001F061FB032010BD002204F18C0195
:10262000BC2002F0F3FA002805D00FF2340001F0CC
:1026300053FB032010BDBC2002F0FFFB60650020AF
:1026400010BD000050443A53746172743230303916
:102650003134000050443A45525241434300000097
:1026600050443A45525256480000000010B5DFF879
:10267000EC4B002204F18001012002F023FB002832
:1026800005D00FF22C0001F027FB032010BD002223
:1026900004F18C01BC2002F015FB002805D00FF2DC
:1026A000200001F019FB032010BD002010BD000028
:1026B00050443A4552524143434F464600000000C1
:1026C00050443A45525256484F4646002DE9F84F7D
:1026D0002DED028BA4B003F081F8DFF8C42C0023A9
:1026E00003F0BAF806460F46DFF8704BD4E9100144
:1026F000A6EB00080EA81421FFF730FF0FF27810A8
:1027000090ED008A03F0B4F9451EAD41ED0F0EA91E
:10271000012003F0C6FC207AA84200D02572832055
:1027200002F083FD0546B8F1140000D540420328AD
:1027300015DBA16F491CA167322291FBF2F2322313
:1027400003FB1211002901D00B2808DBCDE900673B
:10275000D4E9102341460FF2241001F0BDFA606F56
:1027600040446067E06E804500DC4046E066206FD4
:10277000404500DA4046206701950EA984B06846BE
:102780001422FFF7B3FE0FBCB0EE480A01F043FB82
:10279000A06D2818A065A06E401CA06641F2717162
:1027A000884259DBD4E91201A6EB000B206D416A87
:1027B000002901D0012500E0002590F828A0606DD7
:1027C000002802D14FF0FF3801E090F9288003F093
:1027D0004FF9814613A84021FFF7C0FE0FF2B40263
:1027E000D2E90001CDE90C010CA803F09FF913A870
:1027F00001F05CFCE16F481CE06716980B9094F9BF
:102800000D000A9094F90C000990A06D089094F9BD
:1028100009000790CDF818800595CDF810A0CDF8E7
:102820000C90CDF808B0BDF9340001909DF932004C
:1028300000909DF931309DF930200FF2600001F0D9
:102840004BFAC4E912670020A066606742F210707C
:10285000E06600202067A06794F9080000F0E0FA25
:10286000002801D000F0D7F8C4E91067002024B098
:10287000BDEC028BBDE8F28F00007A4450443A531D
:10288000544552522825642920256C6C6420256CFF
:102890006C640A00000000000000000050443A2070
:1028A0005B25755D25643A25643A25643A256420E4
:1028B000747325642C6C636425642C7265662874BB
:1028C00025642C6525642C76256429202564202523
:1028D000642C25642C25642C25640A0010B5DFF8CF
:1028E0007C4994F9000000283AD494F90B0094F93B
:1028F0000110814228D1617B0818E07240B23D2866
:1029000001DB3C38E07294F90B100FF2700001F01B
:10291000E3F90020A065DFF8C00C90F90100014642
:1029200011F1010F01D1012010BD94F90120511ABC
:10293000012901DB101A00E0801A40B2012801DBF6
:10294000012010BD002010BDDFF8900C90F901208F
:10295000914203D0D4E90023C0E90023002010BD38
:10296000A06DDFF80C1D884205DB0FF2180001F0A6
:10297000B3F9012010BD002010BD000050443A4EB4
:102980005425640050443A4E6F54696D6500000050
:1029900010B40020DFF8C41802E04B7B9A18CA720A
:1029A00091F90B20002811D44878801A40B20128F0
:1029B000F3DA00280AD0030000D55B4291F90D40FC
:1029C0009C42EDDA101BC8720020E9E73C2A02DBCA
:1029D000A2F13C00C87210BC704780B5DFF87C08DB
:1029E0000021C17301214172002181724FF0FF313A
:1029F00001700F210173142141730021817301873C
:102A0000C1658174016641660A4624211430FFF7CE
:102A10002FFD002002BD30B5A5B00AA85821FFF750
:102A20009DFD00A82821FFF799FD20A81421FFF79C
:102A300095FD0AA800F024FEDFF8384C9DF8290027
:102A400020709DF82900C02806D113A9C88DA4F8CC
:102A50005E00086B206694E0000633D49DF82A00DF
:102A60008DF8800020A89DF82B1041700021817006
:102A70009DF82C10C170BDF833100A0A0271417123
:102A80000DF133018A788271C978C1719DF83710D0
:102A900001729DF8381041729DF82D1081729DF8D9
:102AA0002E10C1729DF82F1001739DF830104173E4
:102AB0000E2220A9601CFFF709FD0F20A4F85E007C
:102AC00024665EE0DDF82A10080C8DF8000000A8EE
:102AD0000A0A42708170DDF82E100A0CC2700A0AD0
:102AE00002714171DDF832100A0C82710A0AC2715A
:102AF0000172DDF836100A0C42720A0A8272C17243
:102B000013990A0C02730A0A4273817313A90A7992
:102B1000C2734A790274CA88130A8DF8113082741C
:102B2000097A8DF81310DDF83A100A0C8DF814208C
:102B30000A0A8DF815208175DDF83E100A0C8DF813
:102B400017200A0A8DF818208DF81910DDF84210A8
:102B50000A0C82760A0A8DF81B208DF81C10DDF80D
:102B600046100A0C8DF81D200A0A82778DF81F1076
:102B7000202200A9601CFFF7A9FC2120A4F85E0018
:102B80002466B4F85E20D01CDFF8D016096D4882A8
:102B9000DFF8E85A0120287068700320A870216EC1
:102BA000E81CFFF793FC2946832003F083F925B046
:102BB00030BD38B5DFF8A4364FF46164C1EB0115C0
:102BC000AD0014FB005414194FF47A756C43DC61AA
:102BD0005B7C009313460A4601460FF20C0001F09D
:102BE0007BF831BD0000000050443A425425643A5D
:102BF00025643A25642C282564290000F8B52DEDBC
:102C0000028B9EB0DFF87867314684B06846402278
:102C1000FFF76CFC0FBC00F0E3FC10EE100A03F0B1
:102C2000B7FA41EC100B9FED7C8BDFF83046256A3C
:102C300053EC102B51EC180B03F0D2FA03F0A2FB6B
:102C400015FA80F020624FF6FF75A84200D3256286
:102C5000314684B068464022FFF748FC0FBC00F0C4
:102C600073FC10EE100A03F093FA41EC100B676A44
:102C700053EC102B51EC180B03F0B2FA03F082FB6B
:102C800017FA80F06062A84200D3656200200D90C0
:102C900002200C90314684B068464022FFF726FCA3
:102CA0000FBC00F0DDFAE18A4018E08280B2FF2814
:102CB00001DBFF20E08200200D9003200C903146C4
:102CC00084B068464022FFF711FC0FBC00F0C8FA40
:102CD000A16A4018A062A84200D3A56200200D900E
:102CE00006200C90314684B068464022FFF7FEFB78
:102CF0000FBC00F0B5FA218B4018208380B2FF286A
:102D000001DBFF20208300200D9007200C9031462E
:102D100084B068464022FFF7E9FB0FBC00F0A0FA40
:102D2000618B4018608380B2FF2801DBFF20608345
:102D300000200D9008200C90314684B06846402257
:102D4000FFF7D4FB0FBC00F08BFAE16A4018E06299
:102D5000A84200D3E56200200D9009200C90314676
:102D600084B068464022FFF7C1FB0FBC00F078FA40
:102D7000216B40182063A84200D325630EA801F000
:102D800095F9276E1C9803F003FA0022DFF85C3DEA
:102D900003F026FA03F0F6FA57FA80F02066616E27
:102DA000491C6166B0FBF1F0207500200D900120F8
:102DB0000C90314684B068464022FFF797FB0FBC69
:102DC00000F04EFA616B40186063A84200D365635F
:102DD000207C00F030FB1EB0BDEC028BF1BDDFF8B3
:102DE0007C04C18A002914D1816A002911D1018B88
:102DF00000290ED1418B00290BD1C16A002908D1CD
:102E0000016B002905D1406B401E8041C043C00FBB
:102E1000704701207047000000000000000059408A
:102E20002DE9F04F9FB0064600250EA801F03EF9AF
:102E3000DFF82844E07B3146884204D0012E79D166
:102E4000284601F043FB28460D9001200C90DFF846
:102E5000301584B068464022FFF748FB0FBC00F0F5
:102E6000FFF907469DED1C0ADFF81405D0ED0E0AA8
:102E700030EE600A10EE100A03F08AF92A46DFF8F5
:102E80006C3C03F0ADF903F07DFA81461FFA89F935
:102E9000DFF8EC044088BDF83A100A1AD2B2099261
:102EA000DFF8DC24D268119B9A4208D1884206D10F
:102EB000DFF8CC04C088BDF83E1088420ED000A8D0
:102EC00029460A460B460EC0119800901C980190A6
:102ED0001D98029000A9A42002F0ECFF002E3FD123
:102EE000002F03D1099850EA090000D001250020E5
:102EF000A0654FF0FF302070D4E90001DFF8DC2638
:102F0000C2E90001DFF8FC2CC2E90001DFF8C826A5
:102F1000C2E90001207BE072E07B002800F0AE8077
:102F20000020E073607C002800F0A8800120A074DD
:102F30000546A3E0002E11D1206D90F82810406ABC
:102F4000002801D0012200E02A46119B0FF2BC208C
:102F500000F0C2FE012001F0B9FA74E7284652E100
:102F60000FF2C022D2E90001CDE9050105A802F067
:102F7000DDFD94F9012094F900104FF47A704FF4BC
:102F800061684FF03C0B11FB08F312FB0B3394F913
:102F900002C043FA8CF3B4F904C000FB03C3BDF9CB
:102FA00018C09DF816A08DF801A09DF901A0CDF8DC
:102FB00020A09DF815A08DF800A09DF900A0CDF8E7
:102FC0001CA09DF914E01EFB08F81AFB0B88DDF825
:102FD00020A0D04400FB08C0F046414509D09DF92F
:102FE0000080424505D094F902809DF901A0D045AA
:102FF00001D1984210D2CDF810C0089803900798DC
:103000000290CDF804E0B4F90400009094F9023085
:103010000FF60C4000F060FE00F0AEF9002819D069
:10302000DDE90501C4E900012846A072D4E90001E8
:10303000DFF8A825C2E900011198009094F9023048
:1030400094F9012094F900100FF6F03000F044FEDE
:10305000FFF79EFCDDE90501C4E90001FFF73EFC36
:1030600000280BD0D4E90001DFF86C25C2E900018B
:10307000607C002801D00120A0740125012E07D119
:10308000E07B3146884203D0002000F041FAE6732D
:10309000012E56D1002F54D0DFF8688B207C617C44
:1030A00008430AD101206074D4E90001C8E9020193
:1030B000A27861782078FFF77CFD94F9010098F9F7
:1030C0000910401A411E222901D2012005E010F109
:1030D000230F01DA012000E0002001282AD1FFF7A8
:1030E0007EFE002826D0207C401C2074C0B215280B
:1030F00009D10FF6643000F0EFFD0120A074142018
:103100002074012516E00020206660660246242116
:1031100004F11400FFF7ACF9607C401C6074A278E5
:1031200061782078FFF745FD0622214608F1080066
:10313000FFF7DCF9FFF762FD40220EA99048FFF788
:10314000D5F9A07B012828D1208F002801D10125A5
:103150001CE0E16D814215D2002F03D1099850EA9D
:10316000090000D00125DFF89C8A98F9020094F943
:10317000022090420AD0481CE065D4E90001C8E969
:10318000000103E00020A0732087E065012E04D138
:10319000607C002801D00120A0742846012801D1BC
:1031A0000021A165216D496A00292BD10021A1656B
:1031B000012826D10FF6AC20D0E90023CDE9042365
:1031C00004A802F0B3FC022000F0A2F9119CDFF881
:1031D000348AD8F81000201A0B2812D31B9802F05A
:1031E000D7FFCDE9020100949DF912309DF911201D
:1031F0009DF910100FF6742000F06EFD1198C8F8BC
:103200001000002528461FB0BDE8F08F50443A6CEE
:1032100063646F6E2063256420652564202825641F
:1032200029000000000000000000000080B5002020
:10323000DFF8B819886500F002F8002002BD00B57B
:1032400091B000A800F032FF402200A9DFF8A009E9
:10325000FFF74CF9012011B000BD0000B058030089
:103260000FB410B590B000249DF98C0001280BD14B
:1032700000F0D2FF1599884202D3441AE4B271E0FB
:103280008038441AE4B26DE000A800F00FFF9DF909
:103290008800401E082865D8DFE800F02905111DC8
:1032A0002935414D590004981699884201D3441A92
:1032B00058E0DFF854291018401A441C52E00598D1
:1032C0001799884201D3441A4CE0DFF83C291018C2
:1032D000401A441C46E006981899884201D3441AC3
:1032E00040E0DFF824291018401A441C3AE0039803
:1032F0001599884201D3441A34E0DFF80C291018DC
:10330000401A441C2EE007981999884201D3441AA8
:1033100028E0DFF8F4281018401A441C22E008982E
:103320001A99884201D3441A1CE0DFF8DC281018EF
:10333000401A441C16E009981B99884201D3441A8C
:1033400010E0DFF8C4281018401A441C0AE00A985C
:103350001C99884201D3441A04E0DFF8AC28101805
:10336000401A441C204610B010BC5DF814FB01202C
:10337000DFF8781888727047DFF87008807A704735
:10338000B0D4030000F09BBEDFF86018792802DBA0
:103390007820088700E008870120887370470000C4
:1033A00040420F0010B5040001D1012402E0072CB7
:1033B00000DB062421460FF6D00000F08DFC641ED1
:1033C000052C2DD8DFE804F0030A11181F26DFF8BA
:1033D0001C08372101733C21417321E0DFF80C0800
:1033E000192101731E2141731AE0DFF800080F2133
:1033F00001731421417313E0DFF8F0070A21017310
:103400000F2141730CE0DFF8E407072101730C2161
:10341000417305E0DFF8D407052101730A214173E8
:10342000DFF8C807017BC172BDE81040FFF7B0BAF2
:10343000DFF8A007704700EB80018800821CDFF8EE
:103440009407DFF8A817CB691B0E92B21354521CD5
:10345000CB691B0C92B21354521CCB691B0A92B25B
:103460001354521CCB6992B21354521C0B6A1B0AA0
:1034700092B21354521C0B6A92B21354521C4B6AF0
:103480001B0A92B21354521C4B6A92B21354521C30
:10349000CB8A92B21354521C8B6A1B0A92B21354F9
:1034A000521C8B6A92B21354521C0B8B92B213545F
:1034B000521C4B8B92B21354521CCB6A1B0A92B211
:1034C0001354521CCB6A92B21354521C0B6B1B0A3E
:1034D00092B21354521C0B6B92B21354521C0B7DBC
:1034E00092B21354521C4B6B1B0A92B21354521CCF
:1034F0004B6B92B21354501C4887704710B5DFF8DD
:10350000EC46618F0FF2887000F0E6FB608F10BD13
:1035100010B5DFF8D846012807DB627C002A04D00A
:1035200001460FF27C7000F0D7FB0022242104F149
:103530001400FEF79DFF002020740120608700200A
:1035400060742066606610BD0FB400B591B000A82D
:1035500000F0ACFD9DED0B0ADDED1D0AB4EE600A36
:10356000F1EE10FA02DB30EE600A05E09FED421A40
:1035700071EE600A30EE800A10EE100A02F008FECA
:10358000DFF85426DFF8543602F028FF02F09AFFE5
:1035900002F0FEFD0022DFF8483602F021FE02F0C4
:1035A000F1FE00EE100AB8EEC00A10EE100A02F0AA
:1035B000EFFDDFF82426DFF82C3602F011FEDFF8ED
:1035C0002826DFF8483602F009FF02F07BFF00EE04
:1035D000100A11B05DF814FB18DA030010DA0300CA
:1035E0000FB400B591B000A800F060FD9DED0D0A8C
:1035F000DDED1F0AB4EE600AF1EE10FA02DB30EEE8
:10360000600A05E09FED1C1A71EE600A30EE800A38
:1036100010EE100A02F0BCFDDFF8BC25DFF8BC3567
:1036200002F0DCFE02F04EFF02F0B2FD0022DFF8F5
:10363000B03502F0D5FD02F0A5FE00EE100AB8EE9E
:10364000C00A10EE100A02F0A3FDDFF88C25DFF8A7
:10365000943502F0C5FDDFF89025DFF8B03502F0B3
:10366000BDFE02F02FFF00EE100A11B05DF814FB52
:1036700040771B009CD003000024744940BD030028
:1036800070B52DED068B9EB004460EA800F00EFD21
:10369000DFF85855A87B012804D1288F002801D1D4
:1036A0000020A873A87C012817D1687C002814D0BA
:1036B000C0216170DFF81C15C0220A70487004F147
:1036C0002406FFF71BFFF085FFF7B2FE30630120F1
:1036D000FFF71EFF0020A874A4E19FEDD48B9FED9F
:1036E000D59BDFF80C5500200D9001200C90294649
:1036F00084B068464022FEF7F9FE0FBCFFF7B0FD2C
:103700000A2880F0BE80002060700D9002200C908E
:10371000294684B068464022FEF7E8FE0FBCFFF75A
:103720009FFD61780843607000200D9003200C908D
:10373000294684B068464022FEF7D8FE0FBCFFF74A
:103740008FFDA07000200D9004200C90294684B0BD
:1037500068464022FEF7CAFE0FBCFFF781FDE0700D
:1037600000200D9005200C90294684B06846402228
:10377000FEF7BCFE0FBCFFF773FD2071294684B035
:1037800068464022FEF7B2FE0FBCFFF729FF10EE9D
:10379000100A02F0FDFC41EC100B53EC102B51EC25
:1037A000190B02F01DFD02F0EDFDA4F80B0004F171
:1037B0000B061C9802F0ECFC53EC182B02F010FDE9
:1037C00002F0E0FDB070BDF83A00F070294684B018
:1037D00068464022FEF78AFE0FBCFFF7B5FE10EEEA
:1037E000100A02F0D5FC41EC1A0B53EC1A2B51ECE9
:1037F000190B02F0F5FC02F0C5FDE0731D9802F014
:10380000C7FC53EC182B02F0EBFC02F0BBFD20745C
:1038100000200D9006200C90294684B06846402276
:10382000FEF764FE0FBCFFF71BFD607100200D90DA
:1038300007200C90294684B068464022FEF756FEC9
:103840000FBCFFF70DFDA07100200D9008200C901B
:10385000294684B068464022FEF748FE0FBCFFF7B9
:10386000FFFCE07100200D9009200C90294684B0E7
:1038700068464022FEF73AFE0FBCFFF7F1FC2072CB
:10388000CEE08020607000200D9002200C90294630
:1038900084B068464022FEF729FE0FBCFFF7E0FC2B
:1038A000C4F8020000200D9003200C90294684B03B
:1038B00068464022FEF71AFE0FBCFFF7D1FCC4F8A1
:1038C000060000200D9004200C90294684B0684624
:1038D0004022FEF70BFE0FBCFFF7C2FCC4F80A0043
:1038E00000200D9005200C90294684B068464022A7
:1038F000FEF7FCFD0FBCFFF7B3FCC4F80E00294631
:1039000084B068464022FEF7F1FD0FBCFFF768FE69
:1039100010EE100A02F03CFC41EC100B53EC102BA3
:1039200051EC190B02F05CFC02F042FD606204F104
:1039300024061C9802F02CFC53EC182B02F050FCCF
:1039400002F020FD3071BDF83A007071294684B054
:1039500068464022FEF7CAFD0FBCFFF7F5FD10EEEA
:10396000100A02F015FC41EC1A0BA24AA24B02F01D
:10397000F1FD06D8A14AA24B02F004FE01D29FED50
:10398000A4AB53EC1A2B51EC180B02F029FC02F0FB
:10399000F9FCF0801D9802F0FBFB53EC182B02F0B1
:1039A0001FFC02F0EFFC307200200D9006200C90FE
:1039B000294684B068464022FEF798FD0FBCFFF709
:1039C0004FFCC4F8120000200D9007200C902946EF
:1039D00084B068464022FEF789FD0FBCFFF740FC2B
:1039E000C4F8160000200D9008200C90294684B0E1
:1039F00068464022FEF77AFD0FBCFFF731FCC4F8A1
:103A00001A0000200D9009200C90294684B06846C9
:103A10004022FEF76BFD0FBCFFF722FCC4F81E002E
:103A2000FFF70DFC1EB0BDEC068B70BD0000000062
:103A300000002440000000000000594010B596B07E
:103A400004460020002C05D10FF26C2000F044F950
:103A5000002048E004F15001497801293CD101A837
:103A60005421FEF77BFD0020ADF8000013E000EECE
:103A7000102AB8EE400ADFED680A20EE200A01A8FD
:103A8000BDF8001000EB810080ED000ABDF80000D9
:103A9000401CADF80000BDF80000142816DABDF88F
:103AA000000054F82020A2F52F70B0F5167FDED963
:103AB000BDF800100FF2102000F00EF901A8BDF8BB
:103AC00000104FF07E5240F82120DFE701201590D2
:103AD00001A800F0FDFC05E0022903D194F8500094
:103AE0000120C046C0B216B010BD00000000244046
:103AF00080B5112802D11078FFF746FC002002BDE6
:103B000010B596B01446102826D0142811D01528C8
:103B100014D0162817D017281AD0292806D03D28E7
:103B200043D1002C41D0FFF781FB3EE0FFF71FFCA3
:103B30003BE021780020FFF725FC36E021780120CA
:103B4000FFF720FC31E021780220FFF71BFC2CE07E
:103B50002078FFF727FC28E000A85421FEF7FEFCA0
:103B6000207814A94870012817D100200FE004EB39
:103B700080014A788B781B0403EB0262CB7802EB5E
:103B800003220979511800AA42F82010401C142879
:103B9000EDDB00A8FFF752FF07E0022805D16078AF
:103BA0008DF8500000A8FFF749FF002016B010BDA7
:103BB0000E4908659831C16183210170142181602B
:103BC00001210173018200214182144941610020D9
:103BD0007047000008BF03007B14AE47E17A743FD2
:103BE00000005940E17A843F2D431CEBB05803009C
:103BF000B0D40300B81E85EB51B89E3F9A999999AD
:103C00009999B93F50D9030080969800E2361A3F3F
:103C10009A9999999999B93F6F12833A40BD0300D7
:103C200050443A2025643A25643A25642E25643EA2
:103C300025643A25643A25642E25640050443A549C
:103C4000696D654E6F7469202564202564202564A4
:103C5000202825642900000050443A425446554C1F
:103C60004C000000000000000000000050443A2515
:103C7000643A25643A25642065783020282564203C
:103C8000252E32662900000050443A555425640020
:103C900050443A4241544C454E4754482025640014
:103CA00050443A436C6561726261746368282564AC
:103CB0002C636E742564290050443A5346205054B6
:103CC0005233206E756C6C0050443A534645525244
:103CD0005B25642C25645D000EB470B5C1B004464C
:103CE00000A84FF48071FEF739FC45AB22464FF433
:103CF000807100A802F05EFC00A802F079FC441C70
:103D0000002000A9611801F8010C274D2878401CFB
:103D10002870802080F3118800BF00BF6878401CA5
:103D20006870224E317808462218F22A0DDA204AAD
:103D30008018002902D00A2100F8011C224600A99F
:103D4000FEF7C4FB3078201830706878401E687029
:103D5000C0B2002802D1002080F3118802F084FD57
:103D600041B070BC5DF810FB10480078002801D00D
:103D7000801C00E00020C0B2704738B50B4C2278A0
:103D8000002A10D000280ED0032101704270084D87
:103D90002946801CFEF79AFB0022F2212846FEF7F6
:103DA00067FB0020207031BD705E03007DDA0300E8
:103DB0007CC903007047000038B5DFF8A80A008806
:103DC0000146102908DA002806D0DFF89C4A04EBE7
:103DD00081004168491C4160DFF88C4A2068401C22
:103DE0002060B0F5617F15DB01250AE004EB85005A
:103DF0004268002A04D029460FF68C20FFF76CFF9A
:103E00006D1C102DF2DB00224021201DFEF730FB3F
:103E10000020206031BD0FB42DE9F0472DED028B5D
:103E200088B0DFF8484AB4F876A004F108050A27FC
:103E3000B5F91E0010FB07F0B5F92010A0EB010842
:103E400004F5BA76304603F097FC94F8740117FB3A
:103E500000F7BFB22A2F18D10FFA88F8B8F1000F77
:103E600013D5B06800280DD10120FEF796FA8046E0
:103E7000FEF765FA0120B060424639460FF614207D
:103E8000FFF72AFF0120706023E0B068012807D106
:103E9000FEF760FA0020B0600FF61020FFF71CFF5D
:103EA0007068282F0DDB002806D1D4F88020394611
:103EB0000FF60420FFF710FF01207060FEF74EFAA6
:103EC00007E0012803D10FF61020FFF705FF0020BF
:103ED0007060129804909DED138A8DED058ADDEDDA
:103EE000148ACDED068ADDF85C8004A890EC030A04
:103EF000404600F08AFCDFF8787995ED030ADDEDA5
:103F0000120AB4EE600AF1EE10FA30D195ED040A0F
:103F1000B4EE480AF1EE10FA29D195ED050AB4EE97
:103F2000680AF1EE10FA22D1F86900F10109C7F828
:103F30001C90B9F1150F02D30020F8611FE0B9F110
:103F4000020F1CD3686902F023F9CDE90201286948
:103F500002F01EF9CDE90001E86802F019F9024605
:103F60000B4649460FF67C10FFF7B6FE07E00498B3
:103F7000E86005982861069868610020F86141466C
:103F800004A8FDF715FC804604F12000FEF750F967
:103F9000A869012814D1F868401CF860FCF72BF9D7
:103FA00004F12000FEF744F9282204F1200104F175
:103FB0004800FEF79BFA0FF64010FFF78DFE18E061
:103FC000FDF7D8FB012812D13869401C3861FDF794
:103FD000D5FB7861FCF70FF904F12000FEF718F922
:103FE0007A6939690FF61810FFF776FE01E000F0E4
:103FF00021F9B869401CB861B0F5617F08DBFB6846
:104000007A6939690FF60810FFF766FE0020B8617B
:10401000FFF7D2FEBAF1000F40D0B4F876000028C6
:104020003CD1287ADFF84C1894ED020ABDEEC00AA4
:1040300010EE102A4FF47A735A4301FB002095EDDD
:10404000010ABDEEC00A10EE101A081841007A6885
:10405000BA603B687B60D4F8800038607869029071
:1040600038690190386800900FF6B800FFF734FE09
:1040700004F18005B068039070680290286A02F02D
:1040800087F8CDE90001A86A02F082F802460B46E3
:10409000D4F880100FF6AC00FFF71EFE404608B0C3
:1040A000BDEC028BBDE8F0075DF814FB002805D0DD
:1040B000DFF8B817096F4022FEF718BA704738B515
:1040C0000C4605000BD1DFF8A40700EE104AB8EE4D
:1040D000400A80ED030A0830FEF7B1F815E0012D23
:1040E0000BD1DFF8880700EE104AB8EE400A80EDE9
:1040F000020A0830FEF7A3F807E0022D05D1DFF829
:104100006C0704740830FEF79AF80D2010FB04F2D7
:1041100029460FF65000FFF7DFFD42F274700446A7
:1041200040F2EF70224601460FF64800BDE83840E5
:10413000FFF7D2BD2DE9F8432DED028B84B0074681
:10414000884691460FF63C00FFF7C6FD42F27470B8
:10415000044640F2EF70224601460FF61800FFF7C2
:10416000BBFDDFF8084700224FF4C0712046FEF780
:104170007FF904F1080504F1B406AE6600EE107A8A
:10418000B8EE408A85ED018A00EE108AB8EE400A4A
:1041900084ED020A85F80890F2EE0A8A48460D215D
:1041A00011FB00F0029020EE280A10EE100A01F038
:1041B000EFFFCDE9000128EE280A10EE100A01F009
:1041C000E7FF02460B460FF2C870FFF785FDFBF7CD
:1041D00067FF2846FEF733F80020606704F174019A
:1041E0000220C88028223046FEF780F90120607145
:1041F00004F5BA7003F0C0FA0020C4F87C01C4F8DA
:10420000780102463C2104F5C07004B0BDEC028B7D
:10421000BDE8F843FEF72CB910B590B0FEF7B2F840
:10422000044600A8FFF742FF0398001910B010BD24
:10423000000000002DE9F041DFF83046251DA86A96
:10424000616D884204D16A8CB4F84E309A4279D0BC
:10425000B0EB010802D5DFF82006804404F15406D3
:1042600095ED100AD6ED060A30EE600AB5EE400A6A
:10427000F1EE10FA03D5DFED940A30EE200AD5ED09
:104280000E0A96ED041A70EEC10AF5EE400AF1EE40
:1042900010FA03D59FED8C1A70EE810A6878012818
:1042A00002D0022827D02DE004F1F40739469FED13
:1042B000CA1A404600F052F8207940442071C0B23A
:1042C00006281FDB04F5807004F174019FEDC21A0B
:1042D000D0ED0A0A90ED080AD4F8000100F03EF88B
:1042E0002079401C2071002240213846FEF7C0F89A
:1042F0000220687006E004F174019FEDB71A404691
:1043000000F02CF8688C002809D10022402104F12B
:10431000F400FEF7ADF8002020710120687028221B
:1043200004F1200104F14800FEF7E0F804F1740004
:10433000F06104F1B407402204F174013846FEF73D
:10434000D5F8F761A88CB4F8BA10884204D004F10B
:104350005406F084A4F8BA00BDE8F081F8B52DED5C
:10436000028BF0EE408AB0EE608AB0EE410A0C4655
:10437000DFF8F854EE8CAF8CA68000F038F894ED9E
:104380000B0A30EE280A84ED0B0A00F075F884ED74
:104390000B0A66802780A86B206394ED0D0A30EE2F
:1043A000080A84ED0D0A00F047F884ED0D0A95ED3A
:1043B000100ADFED8A0A20EE200A84ED0E0ADFEDF6
:1043C000880AB4EE600AF1EE10FA02DBDFF8AC0402
:1043D000A063686BE0636088002801D10020E0637F
:1043E000286BA060288DE080BDEC028BF1BD38B554
:1043F00005460C46E0682818E06000F05CF8E060D4
:104400006088032802D0042807D00DE0206928180E
:10441000206100F050F8206131BD606928186061AA
:1044200000F049F8606131BD20692818206100F072
:1044300042F8206131BD000080B52DED028BB0EE59
:10444000408A9FEDB10AB4EE408AF1EE10FA0DDB1E
:104450009FEDAE0A38EE008A18EE100A01F098FEC1
:1044600002460B460FF23450FFF736FCB0EE480A16
:10447000BDEC028B01BD000080B52DED028BB0EECE
:10448000408A9FEDA10AB4EE408AF1EE10FA0DDBEE
:1044900018EE100A01F07CFE02460B460FF208509F
:1044A000FFF71AFC9FED990A38EE008AB0EE480A31
:1044B000BDEC028B01BDDFF8C013884202D3DFF8E8
:1044C000C01308187047000000247449FDF77EBF30
:1044D000FDF7BFBE2DE9F8432DED048B8AB00446ED
:1044E000B0EE408AF0EE608AB0EE419ADF4D05F5FD
:1044F000C27696ED0B0AF0EE480AB4EE600AF1EED1
:1045000010FA05D1D5F884012018C5F8840102E01D
:104510000020C5F88401F0EE689A96ED0C0AB4EE1E
:10452000690AF1EE10FA03D170682018706001E09A
:1045300000207060B0EE490AD6ED0D0AF4EE400A94
:10454000F1EE10FA03D1B0682018B06001E000204D
:10455000B060D6F80480D5F8849140F6B837B945F4
:1045600004DAB84502DAB068B8422EDB10EE100A61
:1045700001F00EFECDE90801B068069019EE900A30
:1045800001F006FECDE90401CDF80880B0EE480A3E
:1045900010EE100A01F0FCFDCDE900014A4621466B
:1045A0000FF21040FFF798FBD5F88401B84202DB08
:1045B0000020C5F884017068B84201DB00207060FB
:1045C000B068B84201DB0020B0600AB0BDEC048BDB
:1045D000BDE8F18300000000000000008FC2753DBF
:1045E0000100C8412DE9F8432DED048B8AB0044643
:1045F000B0EE408AF0EE608AB0EE419AB5EE400A25
:10460000F1EE10FA01DCB1EE400A984DDFED940AAC
:10461000B4EE600AF1EE10FA05DBD5F8900120182F
:10462000C5F8900102E00020C5F89001F0EE689A0C
:10463000F5EE409AF1EE10FA02DDB0EE690A01E003
:10464000B1EE690A05F5C876B4EE600AF1EE10FA2B
:1046500003DB70682018706001E000207060B0EE2D
:10466000490AB5EE400AF1EE10FA01DCB1EE401A4B
:10467000B4EE601AF1EE10FA03DBB0682018B060F7
:1046800001E00020B060D6F80480D5F8909140F6A3
:10469000B837B94504DAB84502DAB068B8422EDB5B
:1046A00010EE100A01F074FDCDE90801B068069023
:1046B00019EE900A01F06CFDCDE90401CDF80880F7
:1046C000B0EE480A10EE100A01F062FDCDE90001DB
:1046D0004A4621460FF20030FFF7FEFAD5F8900166
:1046E000B84202DB0020C5F890017068B84201DBD7
:1046F00000207060B068B84201DB0020B0600AB0F2
:10470000BDEC048BBDE8F18301247449002474C915
:1047100070B52DED088B8AB00646B0EE408AF0EEFB
:10472000608AB0EE419AF0EE499AB0EE68AA20EEA7
:10473000000A0AEE0A0A09EEA90AFDF77DFE4B4CB3
:10474000D4F89C0104F5CE75002805D10021E9605C
:104750004C49A96000212961D5ED030AF4EE400A15
:10476000F1EE10FA01D585ED030AD5ED020AB4EE9B
:10477000600AF1EE10FA01D585ED020AD5ED040AC2
:1047800070EE80AAC5ED04AA6968491C0BEE101AE8
:1047900085ED01BA3018C4F89C0147F231518842C6
:1047A0002FDB19EE900A01F0F3FCCDE908011AEEB7
:1047B000100A01F0EDFCCDE90601B0EE480A10EE5A
:1047C000100A01F0E5FCCDE90401E86801F0E0FC25
:1047D000CDE90201A86801F0DBFCCDE90001B8EEEB
:1047E000CB0A8AEE800A10EE100A01F0D1FC0246D4
:1047F0000B460FF20820FFF76FFA00206860C4F83C
:104800009C010AB0BDEC088B70BD70B52DED048B1A
:104810000446B0EE408AF0EE608AB0EE419A134D45
:10482000B5F87660FFF756FEB0EE491AF0EE680A6A
:10483000B0EE480A2046FFF7D5FEB0EE491AF0EE7A
:10484000680AB0EE480A2046FFF762FF05F5D87007
:1048500080EC038AA5F88061BDEC048B70BD00007C
:1048600035336B41985A0300ACD30300CCC003002E
:1048700000D8030040420F00819698000000C84114
:10488000806967FF00007A4450443A462564282531
:104890006429000050443A42504F4E205648282583
:1048A00064292053746570282564290050443A42D5
:1048B000504F46460000000050443A537465704320
:1048C0006E7455702056482825642920535445504D
:1048D000282564290000000050443A4558495456A0
:1048E0004800000050443A4E41435B25645D20255A
:1048F000662025662025660050443A4F4652000047
:1049000050443A52432825642C25642900000000B5
:1049100050443A52432825642C2564292C4F4628BC
:104920002564290050443A53532825642C25643EBD
:1049300025643E2564292C52432825642C256429AE
:104940000A00000050443A532825642C252E326674
:104950002C252E3266292C562825642C2564290AFC
:104960000000000050443A50555428256420256426
:104970002900000050443A5052497625642C4D7667
:104980002564000050443A31345345503230000021
:1049900050443A25662025662025640050443A4458
:1049A0006973744F6625660050443A43616C4F4604
:1049B0002566000050443A45532825643A25642C66
:1049C000252E32662F25642C252E32662F25642C49
:1049D000252E32662900000050443A4546282564B9
:1049E0003A25642C252E32662F25642C252E32661E
:1049F0002F25642C252E32662900000050443A4EA3
:104A000043252E32662C252E32662C252E32662F1B
:104A100078252E32662C79252E32662C7A252E3278
:104A2000660A00002DE9F04100242546DFF8807970
:104A30001EE0052000F034FD0020F1690968884778
:104A4000002804D02046441CC0B20228F1DBE4B2A6
:104A5000032C0BDB0020317847F82100307857F821
:104A60002000C8F80400304602F068FF6D1C0024E6
:104A7000252D18DA2C2002F049FF064622462C216B
:104A8000FDF7F6FCDFF82C89304658F835108847DA
:104A9000307847F8206008EBC508307857F82000D8
:104AA000C8F80400C8E72046BDE8F081002200E015
:104AB000521C92B28A4204D2135CFF2BF8D0012020
:104AC00070470020704702B513463721197058709F
:104AD000022200A9981CFDF7F9FC01BD02B51046A1
:104AE00001210170022200A9401CFDF7EFFC01BD6D
:104AF000008A022801DB012070470020704770B552
:104B000088B0064602A80FF614111422FDF7EEFC39
:104B1000DFF89C0850F82600458A281D02F0F6FEB2
:104B20000446224601213046FFF7CDFF211D3046C5
:104B300001F0B7FA281DADF80B002846A0F10801D6
:104B400089B2201DFFF7B2FF00280DD000F0D7FF7B
:104B5000CDE90001082200A928190838FDF7B6FCA4
:104B6000214602A802F0FCFE204602F0E7FE08B053
:104B700070BD10B50C46C17801290ED100216160CD
:104B8000FFF7B6FF002805D0A068002802D001F08A
:104B900007F800E00020A06010BD8068002804D065
:104BA00000F0FEFFA060606010BD606800F0F8FFDC
:104BB0006060A06010BD30B400216FF0004210466C
:104BC00016E0DFF8F04704EBC3035B68002B0ED060
:104BD0001C6A002C0BD0DD78002D08D1E4681B780E
:104BE000052B01D1042C02D0A04200DD2046491C37
:104BF00049B20B46252BE4DB082801D0102800D150
:104C00000420904200D1002030BC70472DE9F041D3
:104C100084B0044615462646DFF8940750F82670FF
:104C200008788DF800004868019088680290002F8D
:104C300001D1032043E000A93846FFF79AFF00A9FD
:104C400007F1200002F0E2FF07F11C0898F80C00C1
:104C500001280BD1204601F057FA07F1100003F0AC
:104C60004FF80020F969496888470DE09DF8000079
:104C7000002809D107F1100003F042F83879012823
:104C800002D12046FFF73BFF2A4600213D20FB6969
:104C90001B699847F878002802D1022003F045F9F3
:104CA000D8F80800002801D0012300E0002398F87C
:104CB0000C2031460FF20C70FFF70EF8002004B004
:104CC000BDE8F081FEB506461446DFF8E40650F86C
:104CD000265008788DF80000486801908868029096
:104CE000002D19D09DF8000000280AD105F11C07FD
:104CF000B868002810D0C0680190B86800690290B8
:104D000003E000A92846FFF734FF00A905F12000C1
:104D100002F09CFF002801D00320FEBDEB6905F1E5
:104D20001C07387B002803D10020D968884704E09D
:104D3000224600213E201B699847022003F0F5F827
:104D4000B868002801D0012300E000233A7B3146F7
:104D50000FF27C60FEF7C0FF0020FEBD2DE9F041A0
:104D600006460C461546DFF8480650F82670002F18
:104D700005D007F11C08D8F80800002801D103204D
:104D80002EE03846FFF7F5FED8F80800C1686268E3
:104D9000914205D10169A268914201D100201FE032
:104DA00000F1080107F1200002F050FF002801D0B7
:104DB000032015E0214607F1200002F027FF2A46D4
:104DC00000213F20FB691B699847022003F0ADF8E2
:104DD00098F80C2031460FF20460FEF77DFF0020AA
:104DE000BDE8F08110B50C4611461A46DFF8C03513
:104DF00053F82030002B01D1012010BD2046DB6983
:104E00001B699847002010BD10B50C4611461A4684
:104E1000DFF89C3553F82030002B01D1012010BD64
:104E2000192C04D1012100F0A7F9002010BD204663
:104E3000DB695B699847002010BD0146CE2901DA85
:104E4000002801D100207047DFF8640550F82100E8
:104E5000704710B582B000218DF80010082804D0EA
:104E600010281CD0202830D013BD00AA01214020DA
:104E7000DFF83C355B68DB695B6998479DF80000AB
:104E8000800703D50021012003F08DF89DF8000074
:104E9000400732D50021022003F085F813BD00AA97
:104EA00001214020DFF808355B68DB695B699847C2
:104EB0009DF80000000703D50021032003F073F8DC
:104EC0000021042003F06FF813BDDFF8E404046A46
:104ED00000F015FEE2699268904700280DD1606AE3
:104EE000002806D00069002803D10021082000F026
:104EF00043F90021084603F056F813BD10B50446E7
:104F0000206AA268002A07D1002810D04269521AEC
:104F1000012A05DB4068F7E74069401A012806DAF4
:104F200000F0EDFDE2699268BDE81040104710BD49
:104F30002DE9F84304460D4604F1100002F058FF35
:104F4000064604F1100002F05AFF07462078372881
:104F500002DA4FF0040801E04FF00308002F43D0BD
:104F600040F2012008EB0601814203DB2046BDE848
:104F7000F243C5E0B5F8031016FA81F2DFF8349475
:104F800008EB020181420DDB0FF25C410FF26C4035
:104F9000FEF7A2FE09F59471284602F0E1FC00201C
:104FA000A5F80300B5F80300484400F59472207892
:104FB000372803DA3946FFF786FD02E03146FFF76E
:104FC0008DFD3A4604F11001B5F8030018FA80F09F
:104FD000484400F5947002F0C3FEB5F8030008EBF6
:104FE00006010818A5F80300BDE8F18338B50446AA
:104FF0001546606A00280FD08069401A01280BDA34
:1050000000F032FD012802D1207B002804D029467F
:105010002046BDE834408BE731BDF0B585B000A82F
:105020000FF20C411422FDF761FA02F074FF0446FE
:105030000025DFF8806328E006EBC5004768002FF5
:1050400014D097F82800002810D0F87800280DD147
:1050500021463846FFF752FF00AA21463846FFF79F
:10506000C5FF214607F1200002F00DFE042D0BD1F3
:10507000BDF80300002807D006F5947100A802F0DF
:105080006FFC0020ADF803006D1C252DD4DBBDF8AE
:105090000300002803D0C84900A802F061FC0020EA
:1050A00005B0F0BD70B5C24951F82050002D26D092
:1050B000C24C2078401C2070802080F3118800BFF3
:1050C00000BF6078401C60702E6A09E006F108019C
:1050D0002846FFF74EFDF06870613069B061766870
:1050E000002EF3D16078401E6070C0B2002802D15B
:1050F000002080F31188BDE8704001F0B5BB70BDA1
:105100002DE9F04385B0044600A80FF2383114228F
:10511000FDF7ECF925784FF4FE70618A90FBF1F60B
:10512000B6B204F1100002F06AFE0746DFF8909272
:1051300019E0B8464A4641462846FFF7C4FC4246B5
:1051400004F1100109F1040002F00AFE608A00FB7C
:1051500008F0001DADF80300494600A802F000FC6D
:10516000A7EB0807BFB2002F03D0B742E1DBB04680
:10517000E0E705B0BDE8F08330B587B004460D46E2
:105180008B4850F82400FFF7BBFF002D13D001A877
:105190000FF2C4211422FDF7A9F900A80FF2CC21C7
:1051A0000A6802608DF802400320ADF8070000A9EC
:1051B00001A802F0D5FB07B030BD30B583B000A820
:1051C0000FF250210CC90CC000240FE0784800A950
:1051D000615C50F82150002D07D02846FFF788FC6D
:1051E000002802D02846FFF78BFF641C052CEDDB5E
:1051F00037BD6F4951F82000002804D0406A0028CC
:1052000001D00120704700207047694951F8200003
:10521000002802D14FF0FF30704790F82810481E48
:105220008041C043C00F40B27047614951F820002F
:10523000002804D0006A002801D0C0687047002010
:1052400070472DE9F0410446012510E0584850F818
:10525000250000280AD0D4E90067012000212A4651
:1052600002F00EFF30433943C4E900016D1C372DB5
:10527000ECDB04F1080681271EE04D4850F82700BA
:10528000002818D0A7F18002501102EB90604FEA7D
:10529000A0185FFA88F806EBC800D0E900450120A5
:1052A0000021A2EB881202F0EBFE2043294306EB1B
:1052B000C802C2E900017F1CCE2FDEDBBDE8F08111
:1052C0002DE9F04186B007460C4600A80FF2A01168
:1052D0001422FDF70BF94FF4FE7002F017FB0500E6
:1052E00019D121E03E462E2010FB06F81FFA88F85F
:1052F00008F10200ADF80300412028706E704246AC
:105300002146A81CFDF7E2F8294600A802F028FB78
:105310004444BF1BFFB2002F03D00C2FE2DB0B264F
:10532000E1E7284602F00AFB06B0BDE8F08138B597
:10533000044601250CE01E4850F82530002B06D00D
:10534000224600214820DB695B6998472E346D1C9A
:10535000372DF0DB31BD70B500240120144A00E088
:10536000401CC0B20146372906DA52F82110002944
:10537000F6D0641CE4B2F3E720462E2111FB00F5C1
:10538000ADB2284602F0C2FA06000FD0002229462C
:10539000FDF7E8F83046FFF7CAFF31462046FFF731
:1053A0008FFF3046BDE8704002F0C8BA70BD000003
:1053B00088AF0300784D0300A04E0300705E030029
:1053C00068B9030023612025642C25642C25640022
:1053D00023722025642C25642C256400236320255A
:1053E000642C256400000000617272616E67655F65
:1053F000646174615F7061636B65740025733A204A
:1054000074785F646174612069732066756C6C28C0
:1054100025642900010E06120800000005000000A6
:10542000000000000000000000000000000000007C
:105430000500000000000000000000000000000067
:105440000000000005000000000000000000000057
:105450000000000000000000050000000000000047
:105460000000000000000000000000000501000036
:105470000500000000000000000000000000000027
:105480000000000010B5DFF8284300220821204664
:10549000FCF7EEFF204610BDDFF814037047000054
:1054A00038B5044602F03AFE4FF47A72624384182B
:1054B00051EBE27500BF00BF00BF00BF00BF02F0AC
:1054C0002DFEA942F6D301D8A042F3D331BD38B5A1
:1054D000044600F014FBB74AC2E90801002C24D0AE
:1054E000B5480078002820D0B44C2078401C2070AB
:1054F000B34D2878401C2870102002F016FD802043
:1055000080F3118800BF00BF2078401E20702878EB
:10551000012804D16868002801D002F06DFF2878C6
:10552000401E2870002080F311881B20BDE8324007
:1055300003F052B838B5044600F0E1FA9D4AC2E9DA
:105540000601002C24D09C480078002820D09B4CD9
:105550002078401C20709A4D2878401C2870082024
:1055600002F0E3FC802080F3118800BF00BF2078A8
:10557000401E20702878012804D16868002801D0D6
:1055800002F03AFF2878401E2870002080F311882E
:105590001C20BDE8324003F01FB838B5044600F0C7
:1055A000AEFA844AC2E90001002C24D18248007876
:1055B000002820D0814C2078401C2070804D287815
:1055C000401C2870202002F0B0FC802080F311885D
:1055D00000BF00BF2078401E20702878012804D129
:1055E0006868002801D002F007FF2878401E287064
:1055F000002080F311882120BDE8324002F0ECBF8A
:1056000080B5002812D0032818D16E4800900023DE
:105610001A4603211C2002F0ABFF6B4800900023C8
:105620001A4603211B2002F0A3FF01BD674800902A
:1056300000231A460221212002F09AFF01BD80B505
:10564000FFF720FF03F036F8BDE80140C8E080B561
:10565000084600F015FA5E4803F0F6F8002805D079
:105660000FF29010BDE80240FEF736BB01BD0023EB
:10567000584A4021564803F047B9FB230FF28412E1
:1056800003F00DB9F8B50C4615461E4605274C48E3
:105690000178491C0170002003F044FA002806D16B
:1056A00033462A462146002003F03FFA074601F020
:1056B000DBF83846C0B2F2BDF8B50C4615461E46BA
:1056C00005273F480178491C0170002003F02AFAA1
:1056D000002806D133462A462146002003F027FA47
:1056E000074601F0C1F83846C0B2F2BD02280ED01C
:1056F00005280CD006280ED008280AD00E2806D07F
:105700001D2806D0222802D0C02802D005E004209F
:1057100070470720704709207047002070472DE927
:10572000F8430C4615461E46052740B2FFF7DEFF3C
:10573000804615F8019B22480178491C01702649D2
:10574000404603F0BEFA002808D10095731EDBB274
:105750004A466108404603F0CAFA074601F084F859
:105760003846C0B2BDE8F2832DE9F04182B00C4664
:1057700015461E46052740B2FFF7B8FF8046104881
:105780000178491C01701449404603F09AFA002838
:1057900007D10096089B2A466108404603F092FA1A
:1057A000074601F061F83846C0B2BDE8F681000056
:1057B00008DA030018D7030080DA030082DA030056
:1057C000705E030035650000CF6400009B6500003B
:1057D00030D403004F660000801A060002F086BC39
:1057E00080B5FFF759FE01210170C17041718171CF
:1057F00001BD00004D534720426F782046756C6C08
:105800000000000073746172745F74785F73747267
:1058100065616D0013F0004C03D55B42524263F1A9
:1058200000039CEA210C00F0178010B5644603D3F6
:105830004942404261F1000100F00EF8640004D3D7
:105840004942404261F10001244203D55B42524289
:1058500063F1000310BD00001B4213D1094236D191
:105860002AB18446B0FBF2F002FB10C2704703F08D
:10587000B5BAFCD30022002370470B0002000021C0
:1058800000207047904271EB030CF6D370B5B1FA6B
:1058900081F4B3FA83F52C1BA340C4F1200532FA3E
:1058A00005F63343A2405FF00046E64002E05B08A5
:1058B0005FEA3202841A71EB030524BF20462946B1
:1058C0007641F4D302000B003000002170BD012AA4
:1058D000CFD970B5140C20D0B1FA81F4B2FA82F5A8
:1058E000C4F120046419B4F12006D6D3B2405FF0AD
:1058F0000044F440002502E052085FEA3303C61A70
:1059000071EB020E24BF3046714664416D41F3D302
:1059100002000B002000290070BD0C46B1FBF2F123
:1059200002FB11452D0445EA1045B5FBF2F402FBDC
:10593000145580B240EA0545B5FBF2F002FB105267
:1059400040EA044070BD000000B585B000A80FF229
:1059500028511422FCF7CAFD00A802F075FF0028A8
:1059600003D00FF2DC40FEF7B7F905B000BD80B5FB
:105970000020DFF8A01448718DF8000000A908206D
:1059800002F011FB0FF2C440FEF7A6F901BD10B5FD
:10599000DFF880444FF47A72DFF87C1404F12400BD
:1059A00003F061FA4FF42F72DFF8781404F1380035
:1059B00003F059FA002010BD7047DFF86C047047FF
:1059C00010B586B0044601A81421FCF7C7FDFFF707
:1059D000F4FF00900D22214601A8FCF777FD04207A
:1059E000ADF8070000A901A801F0BAFF06B010BD8C
:1059F00010B58CB0044606A81421FCF7AFFD00A832
:105A00001821FCF7ABFD0D22214606A8FCF75EFD30
:105A100000A8FFF716FC1820ADF81B0000A906A887
:105A200001F09EFF0CB010BD10B5DFF8E8436070C8
:105A30002078012808D16078082805D1FFF7BDFB40
:105A40000FF2144003F078FA6078042802D10120A4
:105A5000207003E0082801D100202070611C07207D
:105A6000BDE8104002F09FBADFF8A8030078704745
:105A7000DFF8A003C0787047DFF8980340797047DB
:105A800070B504003AD0DFF88C53D5E90401002941
:105A900001D100280ED0D4F80520D4F80930101A0E
:105AA00063EB0101DFF874230123994202D825D367
:105AB000904223D3DFF874633078401C307080202C
:105AC00080F3118800BF00BF7078401C7070FFF732
:105AD00085FED4F80520D4F80930C5E90423C5E9CA
:105AE00006017078401E7070C0B2002802D10020FC
:105AF00080F31188BDE8704000F0B6BE70BD38B5C7
:105B0000FFF76CFEC34AD2E9044520186941D2E987
:105B10000645001BA94134BDBE4902780A7242788D
:105B20004A72807888720020888170470622C049B6
:105B3000FCF7CCBC10B5044602F0EDF9B5490A6A91
:105B4000002A01D0A21A00E00246B2F57A7F00D303
:105B5000024688891018888100B2B0F57A7F05DB8B
:105B6000A0F57A708881887A401C887291F90A00C1
:105B70003C2804DB3C388872487A401C487291F912
:105B800009003C2804DB3C384872087A401C087243
:105B900091F90800182801DB002008720C6210BD82
:105BA00010B5142801DA022400E00A24042801DADE
:105BB000022010BDA12801DBA02010BD90FBF4F055
:105BC00003F0CCF941EC100B03F0E0F951EC100BB1
:105BD00000F0D8FB03F0C2F941EC110B9FED950BDF
:105BE00003F01FFC51EC100B00F0CCFB604310BD28
:105BF00000B587B002A80FF294211422FCF776FCBE
:105C000000A800210A4606C0FFF746FC01788DF87F
:105C1000001000A9C2784A7042798DF8022080797C
:105C2000C87001208DF804000520ADF80B0002A813
:105C300001F096FE07B000BD30B59FB005A8642105
:105C4000FCF78CFC00A80FF258211422FCF74EFC44
:105C50000024FF22642105A8FCF70AFC012517E0B7
:105C60002846C0B2FFF7E9F8002810D02946491E9F
:105C7000012906D9C91E022903D9091F01D01A39E1
:105C800005D105A964B26554408A401C04196D1CF5
:105C9000092DE5DB64B2ADF8034005A900A801F0C9
:105CA0005FFE00201FB030BD38B50446A078014625
:105CB000491F1CD0491E1DD0491E012927D9891E04
:105CC00001292CD9203907D00F390AD0491E4AD0D2
:105CD000491E01292CD94BE0D4F80D00FFF71CFF19
:105CE00046E0B4F80300C0B2FFF79EFE40E04C4827
:105CF00003F0C5F8A078052801D1012000E00020BC
:105D0000444DE870E91C062002F04DF930E0072808
:105D100001D1012000E000203E49087128E03D4DFE
:105D2000092802D10020A87022E00120A8701FE0FD
:105D3000384D3A280ED141A0FDF7CEFF0120687101
:105D400005F1380003F0C6F8D4F80D10082002F071
:105D50002AF90DE00FF21810FDF7BEFF05F138002B
:105D600003F08DF804E0D4F80D10012003F0DCFD01
:105D7000A0781438032801D915380FD18320FFF7F4
:105D80005CF803000AD0D4F80D20B4F80310A07812
:105D9000DB691B6901B0BDE83040184731BD80B5F3
:105DA00081780C2908D018290FD01B2907D02C295D
:105DB0000ED031290FD001BDBDE8024000E6FFF74B
:105DC00017FEBDE80140FFF7C6BABDE801400FE786
:105DD000BDE8014030E70F480078002803D1BDE856
:105DE0000140FDF7E7BF01BD80B500208DF8000040
:105DF000481E042802D201208DF8000005489DF8B5
:105E000000108279914204D0817100A9052002F02E
:105E1000CAF801BD18D303004969000000F2052A41
:105E20003CD303006F690000CC905101705E030009
:105E300020D3030000000000000000404D4F4E0042
:105E4000736B697020524349000000004D4F464675
:105E50002043422100000000232121206170207393
:105E600074617465206368616E6765210A000000D3
:105E70004D4F46460000000004FF310000000000C6
:105E800000000000000000000000000004FF1800F7
:105E90000000000000000000000000000000000002
:105EA00004FF2C00000000000000000000000000C3
:105EB000000000002DE9F04180460C46FEF7BDFFD2
:105EC0000546002702F027F80646B8F1010F1ED05C
:105ED000B8F1040F4BD0B8F1050F78D0B8F1080F26
:105EE00000F08480B8F1250F00F0A980B8F1870F89
:105EF00000F0BE80B8F1A10F00F09480B8F1A40FBB
:105F000000F09680B8F1BB0F00F0AD80B5E003F073
:105F10002EFEDFF85882B4F9000000EE900AF8EE89
:105F2000E00A20EE800A88ED000A03F020FEB4F9B2
:105F3000020000EE900AF8EEE00A20EE800A88EDFA
:105F4000010A03F014FEB4F9040000EE900AF8EE22
:105F5000E00A20EE800A88ED020A2088A8F80C00EA
:105F60006088A8F80E00A088A8F8100085E003F06B
:105F7000B8FEDFF8F881B4F9000000EE900AF8EE00
:105F8000E00A20EE800A88ED050A03F0AAFEB4F9C3
:105F9000020000EE900AF8EEE00A20EE800A88ED9A
:105FA000060A03F09EFEB4F9040000EE900AF8EE33
:105FB000E00A20EE800A88ED070A2088A8F8200071
:105FC0006088A8F82200A088A8F8240055E0DFF82F
:105FD0009C81D8F834002168884200D101271C2216
:105FE000214608F13400FCF771FA46E0DFF87C81C5
:105FF00098F850002178884200D1012701222146DB
:1060000008F15000FCF762FA0222611C08F152000C
:10601000FCF75CFA022204F10B0108F15400FCF7D2
:1060200055FA2AE00C2221465148FCF74FFA24E0A9
:1060300001270C2221464F48FCF748FA1DE0DFF803
:106040002C81D8F858002168884205D1D8F85C0026
:106050006168884200D101270822214608F15800D2
:10606000FCF734FA09E0E078404981F86C0004E07C
:1060700094F903003D4981F86D00002D0FD0002FE9
:106080000DD1686A00280AD04069801B012806DA11
:10609000214605F11000BDE8F04101F035BEBDE834
:1060A000F08102460846012A0ED0042A10D0052AA3
:1060B00012D0082A14D0872A22D0A12A14D0A42AC8
:1060C00016D0BB2A18D0704714222849FCF7FEB915
:1060D00014222949FCF7FAB91C222849FCF7F6B921
:1060E00006222749FCF7F2B90C222149FCF7EEB948
:1060F0000C222049FCF7EAB901222249FCF7E6B953
:1061000001222149FCF7E2B901280CD004280FD064
:10611000052812D008281AD0252813D0872820D087
:10612000BB2819D07047FF2214211048FCF7A0B9F2
:10613000FF2214211048FCF79BB9FF221C210F48B5
:10614000FCF796B9FF2208211048FCF791B9FF220D
:1061500006210B48FCF78CB9FF2201210948FCF706
:1061600087B90420014981F86D007047C0CF030052
:10617000E8CF030020D00300D4CF0300F4CF030006
:1061800010D003002CD003002DD0030018D0030042
:106190005FF0FF0C1CEAD05114BF614506E0C1104E
:1061A000400721F0E04101F16051704779B900F0FA
:1061B000004100020AD0B0FA80FC00FA0CF001F1B4
:1061C0006051A1EB0C5101EBD02140057047410219
:1061D0000CBF40F4E0016FF00001002070470000A8
:1061E000B0B581EA030C0CF0004C40F2FF7515EAE3
:1061F00011541DBF15EA1357AC42AF4239E0E41900
:1062000023EA455343F48013C90241F0004141EAB7
:10621000505EC7021100A7FB020200284FF00000E9
:10622000EEFB01204FF00001E3FB072118BF42F015
:106230000102401800214941E3FB0E01A4F58064EE
:106240000F0302D252004041494154F101046CDD78
:10625000470872F1004250F1000051EB0451A1F5E2
:1062600080115CBF41EA0C01B0BD4CEA0551002031
:10627000B0BD05EA1357AC4214BFAF4241E050EA4B
:10628000410E1CBF52EA430E02E061460020B0BD41
:1062900024423C441BD15FEA070EF6D0090302BF3B
:1062A00001460020AEF1140EB1FA81F7AEEB0704FF
:1062B00001FA07FE0C37C7F1200100FA07F7C840C2
:1062C0004EEA000E23EA455343F48013A2E733F06D
:1062D0000043B3FA83F704BFB2FA82FE77440B3F60
:1062E000E41BB7F1200E2FBF02FA0EF3BB40C7F13B
:1062F000200E22FA0EFE38BF43EA0E03BA40641C99
:1063000082E750EA410E14BF52EA430E6FF00001DB
:106310004FF4001717EB430F8ABF194617EB410FD5
:10632000B5E74CEA05510020B0BDD4F10104B4F149
:1063300020070FDAC4F12007520828BF42F00102FB
:1063400010FA07F501FA07F7E1BF2A43E0403843A6
:10635000E1400FE0352C98DCC7F1200452EA4002FE
:1063600020FA07F218BF42F0010231FA07F0A1400B
:106370000A43002172F1004250F1000051EB0C0180
:10638000B0BD0000F446400D40EAC120490006D2ED
:1063900000F014F8004248BF6FF00040604700F082
:1063A0000DF84FF0004188428CBF084640426047DC
:1063B000400D40EAC120490080F00D8040F00040CF
:1063C000490DA1F58061491C05D4D1F11F0154BFCD
:1063D000C840C01770474FF00000704770B44FF0CE
:1063E000004591EA030C44BF6B4003F0A5BC00BF1D
:1063F000841A71EB030603D2001BB14112197341D9
:106400004FF4001C1CEB410F34BF7CEB430443E012
:106410000C0DA4EB1356352E50DC45EAC323DB0AE2
:1064200045EAC121C912B6F120050DDD63FA05F672
:10643000EB4086EA0305124218BF45F00105C0187B
:1064400051F100010CD213E062FA06F5F24055401A
:10645000F3415A40B340F3405A408018594107D3A2
:1064600049085FEA30005FEA350528BF45F00105BD
:1064700001F58011420875F1004250F1000041EB36
:10648000045170BC4FF4001C1CEB410F38BF704727
:106490000020090D090570471CEB410F10D252EA8C
:1064A00043060BD0BCEB410F05D80C0DAB43661E69
:1064B000342EB5DD02E0AB438018594170BC704703
:1064C00070BC70474FEAF17CBCF1E04C2CBFBCF5CE
:1064D000001F11E05FEA4C0C34BFBCF17F5F2EE07F
:1064E0005FEA9C0C4FEA0C1C4FEA3C0CC10071F1B6
:1064F00000414CEB50707047C90241EA5051C00254
:1065000018BF41F0010141F000414FEA6C50C0F169
:106510000900212810D240EACC7CCCF1200C11FAE1
:106520000CF070F10040CCF1200C21FA0CF00CF0D2
:10653000004C40EB0C0070474FEACC7070474900AC
:1065400011F5001F04D84FEACC10FF30C00570478A
:10655000C81770474FF4001C1CEB410F94BF1CEB95
:10656000430F09E041EA030C50EA4C0C52EA0C0CD0
:1065700003D28B4208BF8242704714BF99429042B7
:10658000704700004FF4001C1CEB410F94BF1CEB44
:10659000430F09E041EA030C50EA4C0C52EA0C0CA0
:1065A00003D2994208BF9042704714BF8B42824287
:1065B0007047000008B584B00023029311B900931E
:1065C000019302E00090481E019004AB00A9074827
:1065D0007844183003F066FC009911B1009A00214C
:1065E0001170002858BF029805B000BD57BFFFFFCB
:1065F00000F10103810704D010F8011B89B1810764
:10660000FAD10268B2F10131914311F0803F04BF29
:1066100050F8042FF6E710F8011B11B110F8011B18
:10662000FBE7C01A7047000030B4802080F3118867
:1066300000BF00BFDFF89413886800220A7182F35C
:10664000118800281CBF0268002A33D043695469AE
:106650009C422FD100E022461468A4B165699D4296
:1066600011D12246146874B165699D420BD122464E
:10667000146844B165699D4205D12246146814B17D
:1066800065699D42E7D0802383F3118800BF00BF76
:1066900003680C69844208BF0B61016A0B601962D0
:1066A00002621168016001B10862106092F829006D
:1066B00082F82800002080F3118830BC704730B584
:1066C000DFF808430020607181B0206AE16900F1C1
:1066D0008040606208001CBF20468847002080F38D
:1066E0001188E56808E0E868616A411A48BF60629D
:1066F000002080F311882D6805B3802080F3118875
:1067000000BF00BF206920B16869216949698842DA
:1067100019D3287C4007EBD5E868216A401A012884
:10672000E1DA284600F0BCF8802080F3118800BF31
:1067300000BF287C0028D6D101B030BD802080F376
:10674000118800BF00BF01B030BD000070B5DFF898
:106750007C420020607001202070E06B68B18020D6
:1067600080F3118800BF00BFE06B8047002080F3FA
:106770001188E063606384F83800A06800281CBFBB
:10678000C16A002904D009680A001CBF4068884714
:1067900094F8310040B1A06894F8301080F82810C7
:1067A000207908B1FFF740FF206948B304E028686A
:1067B0002061002080F31188802080F3118800BFC1
:1067C00000BF25690DB32E7CFEB170070ED5E868B9
:1067D000216A411A012905DA284600F061F8287C6F
:1067E00020B90DE0616A411A48BF606206F0FB0003
:1067F0001028DCD1A86880684068007C0028D6D1C9
:10680000802080F3118800BF00BF607950B92069F3
:1068100000B32069007C0028206909D08068806866
:10682000406805E0FFF74BFF60790028FAD1EEE7FA
:10683000A060A068C16A21B149680A001CBF406815
:106840008847A06890F8280084F8300084F8310068
:10685000204670BD84F8310084F83000A0602070BC
:1068600080F31188204670BD10B5584C2078401E2A
:106870002070C0B298B9606888B1802080F3118818
:1068800000BF00BF606830B101202070204601F0D9
:10689000A0FD00202070607808B980F3118810BD39
:1068A00030B581B08168494C41B1226AC2600A6842
:1068B000496802B151600A6000218160017C11F0D9
:1068C0000301017426D1216991B92061207838B97A
:1068D00001202070204601F07CFD0020207001E0A6
:1068E000012060716078A8B980F3118801B030BDD3
:1068F00042694B699342E8D38142E7D09A4209D179
:1069000003461B68002BEDD05D69AA42EAD18B4299
:10691000F7D1DAE701B030BD30B52C4C227881B028
:106920004169521C227004F10C0200E01A461368FF
:10693000A3B15D69A94211D21A46136873B15D69AA
:10694000A9420BD21A46136843B15D69A94205D228
:106950001A46136813B15D69A942E7D30360026266
:10696000106043B118625A698A420CBF90F829102E
:10697000002180F82810017C51B9802181F3118811
:1069800000BF00BFFFF78CFF607808B980F3118863
:1069900001B0BDE8304067E730B50C4C2578681C85
:1069A000207081B0204601F014FD6078257008B990
:1069B00080F3118801B030BD00B581B004F048F912
:1069C00002480121017001B000BD0000705E0300AB
:1069D0002DE9F043002300E05B1C032B4ADA00247E
:1069E00033E005F1070EAEEB060E4FF007089EFBF5
:1069F000F8F8C8EBC808AEEB080E5FFA8EFE0FF68B
:106A00006468C3EBC30908EBC90808EB8609D9ED34
:106A1000070A07EB000909EB8E0999ED3F1A60EEB2
:106A2000810A08EB860898ED001A0CEB8E0EDEED5D
:106A3000001A41EE610A30EE800A761C072ED0DB88
:106A40000CEB850585ED000A641C032CC4DAC4EB4D
:106A5000C405AF00542515FB030507EB050C0D46D7
:106A6000002A03D100264CF82560EDE79FED440A8B
:106A70000026E3E7BDE8F083D2B218B400230CE0AF
:106A800094ED031A21EE001AF7EE001A71EEC01A07
:106A900001EEA01A84ED001A5B1C032B0ADA51F8F0
:106AA000234000EE904A002A00EB8304E8D1C4EDB5
:106AB000000AF1E70C2201460C3018BCFBF716BDAA
:106AC00038B504460D4600200AE0C0EBC00204EBD6
:106AD000820202EB810155F82020C1F8FC20401C05
:106AE00004F5F27292F902100328EEDB5278C9B273
:106AF0002046FFF76DFF94F8E4219FED220A294616
:106B000004F5A870BDE83840B6E70000F8B50446C3
:106B100094F9E651EDB2002617E0542212FB06422A
:106B200011FB002151F8251000EE901A00EEA00A8A
:106B3000401C1C210328F0DB11FB064000EB8507FD
:106B400004F0A2F887ED5D0A761C032E03DA9FEDB0
:106B50000C0A0020EDE704EB850000F5C87191ED0B
:106B6000070AB5EE400AF1EE10FA06D0D0ED640A3D
:106B700080EE800A81ED0E0AF1BD00208863F1BD30
:106B800000000000A4707D3F10B5044604F5A87015
:106B9000D0ED020A90ED011A94ED540A20EE000A9D
:106BA00001EE010A00EEA00A04F06EF8002002E0F7
:106BB00000228A61401C03280FDA04EB800202F5F0
:106BC000A871B5EE400AF1EE10FAF1D0D2ED540AF8
:106BD000C0EE800AC1ED060AECE710BDD0ED000A58
:106BE00070EE800AC0ED000AD0ED010A40EE000A06
:106BF000C0ED010A89B2531E994215D100EE102A48
:106C0000B8EE400AD0ED000AC0EE800AC0ED000ADE
:106C1000D0ED010A80EE800A80ED010AD0ED000A75
:106C200000EEE00A80ED020A70472DE9F84F0446B5
:106C30000D4694F9E601C0B200902E88322096FBF2
:106C4000F0F0322101FB1067B5F878804FF00009B1
:106C50002AE004EB890A09EB490005EB800B4FF4AD
:106C6000FA7231460BF140009AED5A0AFFF7B6FF6F
:106C700040F2DC5241460BF190009AED5A0AFFF7C0
:106C8000ADFF3222394689B20BF11C00C9EBC903B2
:106C900004EB8303DDF800C003EB8C0393ED3F0AA4
:106CA000FFF79CFF09F10109B9F1030FD1DBBDE842
:106CB000F18F8A1D072392FBF3F3C3EBC303D21AB0
:106CC00050F8222000EE102A00EB8100D0ED000ADF
:106CD00030EEC00AB0EEC00A704730B40A46002158
:106CE000931D072493FBF4F4C4EBC4041B1BDBB219
:106CF000541D072594FBF5F5C5EBC505641BE4B2EF
:106D000050F8233000EE103A50F8222000EE902A7E
:106D1000F4EE400AF1EE10FA0AD500EB840292ED8F
:106D2000001AB4EE401AF1EE10FA01D501210EE07E
:106D3000B4EE600AF1EE10FA09D500EB8400D0ED54
:106D4000000AB4EE600AF1EE10FA00D501210846FF
:106D500030BC70472DE9FE4306460C4696F8E651D6
:106D60002088002800F08A8000273CE0C7EBC7009D
:106D700006EB8009294609F15400FFF79AFF08EB5A
:106D8000870080ED000AD4ED030A30EE800A84ED1E
:106D9000030A09F1A80829464046FFF78AFFD4ED07
:106DA000050A30EE800A84ED050A294609F15400EF
:106DB000FFF793FF00EE100AB8EE400AD4ED040A84
:106DC00030EE200A84ED040A29464046FFF785FF8D
:106DD00000EE100AB8EE400AD4ED060A30EE200AA2
:106DE00084ED060A7F1C0DF10008032FBEDB002096
:106DF0000AE094ED010A08EB8001D1ED000A30EEC3
:106E0000200A84ED010A401C0228F2DB94ED020AFC
:106E1000D8ED020A30EE200A84ED020A294606F572
:106E2000C870FFF746FFD4ED030A30EE800A84ED08
:106E3000030A294606F5D670FFF73BFFD4ED050A95
:106E400030EE800A84ED050A06F5E47629463046E0
:106E5000FFF72FFFD4ED1B0A30EE800A84ED1B0AEA
:106E600029463046FFF739FF00EE100AB8EE400A17
:106E7000D4ED1A0A30EE200A84ED1A0ABDE8F78331
:106E80000A8890F9E631DBB200EB830090ED5D0AF1
:106E90003220034692FBF3F300FB1323002B04D1B3
:106EA00081ED020A81ED030A7047D1ED020AF4EE8A
:106EB000400AF1EE10FA02D581ED020A08E0D1EDA8
:106EC000030AB4EE600AF1EE10FA01D581ED030A6F
:106ED000521C034692FBF3F300FB132000281BD146
:106EE00091ED020AD1ED030A30EE600AD1ED040AF9
:106EF00070EE800AC1ED040A022B0BDBD1ED010A12
:106F000070EE600AF0EEE00A91ED051A71EE200ACB
:106F1000C1ED050A81ED010A088840F2DB5290427A
:106F200009D191ED040AF3EE0E0A80EE200A81EDFC
:106F3000040A012088707047F8B52DED048B84B0E9
:106F40000C460021642749E0C1EBC10200EB82023C
:106F500090F9E63152F8232000EE102A00AA02EB45
:106F6000810282ED000A04EB810202F2B445D5ED04
:106F7000030A70EE800AC5ED030A4FF4C87313FBD1
:106F8000014394F8B06403EB860696ED001A70EEA8
:106F9000C10AC5ED030AD2F8B45400EE905A70EE5F
:106FA000800A02F2B445C5ED000A94F8B0543235B7
:106FB0003E4695FBF6F607FB165503EB850595ED6A
:106FC000001A70EEC10A02F2B442C2ED000A94F84F
:106FD000B02403EB820282ED000A491C0329B3DBD3
:106FE00094F8D804002816D100200EE004EB8001AC
:106FF000D1F8B42400EE102ADFED850A80EE200AD5
:1070000001F2CC4181ED000A401C0328EEDB012097
:1070100084F8D80458E004F5966090ED040ADFED9A
:107020007D0A80EE200A8DED000A90ED050A80EEC3
:10703000200A8DED010A90ED060A80EE200A8DED02
:10704000020A9FED758A9FED740ADFED738A0020B6
:1070500011E004EB8001D1F8CC1400EE901A00A9E5
:1070600051F8201001EE101A00EE818A00EEA00AFD
:1070700041EE018A401C0328EBDB03F005FEB0EE75
:10708000409AB0EE680A03F0FFFD29EE000AB5EE63
:10709000400AF1EE10FA01D088EE008AB0EE480AFC
:1070A00003F000FEDFEDC80A20EE200AF3EE0E0A20
:1070B000B4EE600AF1EE10FA03DB002084F8D80485
:1070C00002E0012084F8D80494F8B004401C84F84D
:1070D000B004C0B2642802D1002084F8B00404B027
:1070E000BDEC048BF1BD000070B52DED048B0646A0
:1070F000301D90ED018A7068FFF74AF841EC190BDA
:1071000018EE100AFFF744F802460B4614461D46D7
:1071100053EC192BDFF8F406DFF8F416FFF760F8EC
:1071200022462B46FFF72EFA1CD253EC192BDFF820
:10713000E406DFF8E416FFF753F802460B46144660
:107140001D469FEDDD0A38EE000A10EE100AFFF72B
:107150001FF822462B46FFF715FA03D2012086F8C6
:10716000740002E0002086F87400BDEC048B70BD52
:1071700070B504460D461646FFF7C8FC2046FFF7DB
:1071800003FD29462046FFF750FD29462046FFF71C
:10719000E1FD05F178012046FFF772FE31462046F9
:1071A000BDE87040C8E6000038B52DED028B90EDCB
:1071B000050A90ED038AFBEE040A9FED841A08EE9F
:1071C000201AB4EE401AF1EE10FA1DD510EE100A96
:1071D000FEF7DEFF02460B4614461D4618EE100A67
:1071E000FEF7D6FFDFF83426DFF83436FEF7F8FF77
:1071F0000022DFF83036FFF7F1F822462B46FFF782
:10720000C1F901D2012000E00020BDEC028B32BDAB
:10721000000048420000C842000000002DE9F04193
:107220002DED028B804600200CE098ED190A01EB51
:10723000410208EB8201D1ED120A30EE200A88EDFE
:10724000190A401CC0B201460329EEDB98ED1A0A68
:10725000D8ED1B0A9FED8F1ADFED8F1A40EE011A51
:10726000F4EE610AF1EE10FA15DB9FED8C1ADFEDFA
:107270008C1A40EE011AF4EE610AF1EE10FA0ADB04
:107280009FED881ADFED881A40EE011AF4EE610ACC
:10729000F1EE10FA4DDA9FED850AF4EE400AF1EEB8
:1072A00010FA46D49FED828BD8F81400FEF770FFD9
:1072B00004460D46D8F80C00FEF76AFF53EC182B75
:1072C000FFF78CF802460B462046294603F01CFDCA
:1072D0000022DFF85435FEF783FFDFF85025DFF892
:1072E0005035FFF77BF802460B4616461F46D8F886
:1072F0001800FEF74DFF04460D46D8F81000FEF7C3
:1073000047FF53EC182BFFF769F802460B4620465F
:10731000294603F0F9FC32463B46FFF733F908D320
:1073200098ED190ADFEDCC0AB4EE600AF1EE10FA1E
:1073300001DB002000E00120BDEC028BBDE8F08104
:107340002DE9F041804698ED1A0ADFEDA10A80EEA2
:10735000200AD8ED1B0A9FED9E1AC0EE810A20EE8E
:10736000200A10EE100AFEF713FF02460B461646DF
:107370001F46D8F80C00FEF70BFF0022DFF8B434EC
:10738000FEF72EFF04460D46D8F81400FEF700FF66
:10739000DFF8A424DFF8A434FFF720F802460B46F8
:1073A0002046294603F0B0FCDFF86824DFF890346B
:1073B000FFF714F832463B46FFF7CCF801D801201E
:1073C00000E00020BDE8F081ED2E65420000FA43A8
:1073D00038B52DED048B05460C4600200CE095EDEC
:1073E0000F0A01EB410205EB8201D1ED080A30EEF4
:1073F000200A85ED0F0A401CC0B201460329EEDBCE
:107400006869FEF7C5FE41EC180B2869FEF7C0FE5F
:1074100041EC190B53EC182BDFF82804DFF8281483
:10742000FEF7DEFE02460B4651EC190BFFF7AAF8F9
:107430002CD253EC182BDFF81404DFF81414FEF7E9
:10744000CFFE53EC192BFFF79DF81FD253EC182BEE
:10745000DFF80004DFF80014FEF7C2FEDFF8CC23EB
:10746000DFF8F833FEF7BAFF53EC192BFFF78AF871
:107470000CD295ED0F0ADFEDC40AB4EE600AF1EE0E
:1074800010FA03D5002C01D1012000E00020BDEC52
:10749000048B32BD00C028C500854F49000048C498
:1074A00000E87D480000C8C200C82F4701806D4534
:1074B0008DEDB5A0F7C6B03E0000CDC338B505468A
:1074C0000C460020A070607095F87A00002806D065
:1074D00095F8741005F17800FFF77AFFA07095F821
:1074E0007400002813D12846FFF75EFE00280CD157
:1074F0002846FFF793FE002807D12846FFF720FF14
:10750000401E8041C043C00F00E0012060706078E1
:10751000002805D1A178481E8041C043C00F00E07B
:107520000120207031BD70B400220378447B241800
:10753000E370437B144610E05B1CDBB20A2593FB2F
:10754000F5F505EB8506A3EB4603DBB21D18ED78D8
:10755000661C16FB052292B2641C0A2CECDB04208C
:1075600008702D2A02DB022048700BE0222A02DB81
:107570000120487006E00F2A02DB0020487001E07D
:107580000020087070BC704710B504469FED9C0A3F
:10759000002008E000EB400104EB8101D1ED090A75
:1075A00000EEA00A401C0328F4DB03F06DFB84ED21
:1075B0001C0ADFED940AB4EE600AF1EE10FA05D56C
:1075C000002211460846BDE81040B3E010BD00009F
:1075D00000401C4670B50C4604F59B65E97BAA7B10
:1075E000121992F8E124891AE973A97B091990ED1F
:1075F0001C0ADFED850AB4EE600AF1EE10FA03DB37
:10760000012081F8E10402E0002081F8E104E87B38
:10761000A97B091991F8E1140818E873904E00222B
:10762000242106F50170FAF723FF96F89A0704283B
:1076300010D196F89B0700280CD0E87B022803DACB
:1076400094F8D804002805D1002204210220BDE8C6
:1076500070406FE070BD0000CDCC4C3E30B591B0B5
:107660007F4C04F5F2718878401C88704A78002AB3
:107670000BD194F8E421002A02D1012284F8E421FC
:1076800040B2072801D101224A7040B2072290FB84
:10769000F2F2C2EBC202801A88708888401C88808F
:1076A000B4F86012491CA4F8601280B2322190FB39
:1076B000F1F1322202FB110131290BD194F8861726
:1076C000491CC9B2052291FBF2F202EB8202891A2F
:1076D00084F88617B0F5FA7F24D104F51875402296
:1076E000294600A8FAF702FF0022B82104F5F47039
:1076F000FAF7BEFEBDF8000040F2DC51884204D02B
:10770000402200A92846FAF7F1FE04F28670C17CF7
:10771000491CC9B20A2291FBF2F202EB8203A1EBEF
:107720004301C17411B030BD002240F29C714C483D
:10773000FAF79EBE2DE9F04106460C461546484F25
:1077400097F8990709300A2190FBF1F101EB8102CA
:10775000A0EB420800220A2107F28F70FAF702FF1D
:107760005FFA88F808EB070080F88F6707F29970D6
:1077700044708570BDE8F081002803D03849B1F825
:107780009A170180704700009A99993EF8B5344CD9
:1077900001462046FFF794F904F5F47504F52876C0
:1077A000324629462046FFF7E3FCB4F8E80140F2F0
:1077B000F31188420DD12846FFF796FC04F28C772E
:1077C00039462846FFF77AFE04F29A713846FFF7E9
:1077D000AAFEB4F8E801322190FBF1F1322202FB5B
:1077E0001100312808D12846FFF7CEFE04F28C7232
:1077F00031462846FFF7EEFEBDE8F1402EE70000D7
:107800000000000052499D390100C04085EB51B88D
:107810001E85F73FD7A3703D0AD71540CDCCCCCC01
:10782000CCCC004000005440000004C09A999999C3
:1078300099991B400000F8BF8DEDB5A0F7C6B03E8A
:107840000AD7E33FE17A14AE47E1BA3FC976BE9F5B
:107850001A2FAD3FEC51B81E85EBA13F9999E93F36
:10786000F089030000000000FDF881C0232FE340F1
:10787000DA1ED9C0F3456E40EDE88DBF0B030F3E15
:107880002D8AE038A267283A8A81D23A5C560C3BAE
:107890008A81D23AA267283A2D8AE0380000000097
:1078A000AD9D27C0EE695740790B1FC088848C3F7F
:1078B00061738ABE9135EC3C61A1F13A0939353CDE
:1078C0004B87E23CDD04173D4B87E23C0939353CF0
:1078D00061A1F13A000000001D1073BE20794C3FF9
:1078E000AE63E7BD2813F53D5676F9BB3631F43A61
:1078F00042CE113D63B55ABE5EB1083FD24136BF9C
:107900005EB1083F63B55ABE42CE113D30B5134D4E
:107910000446287881B020B9281D03F037FB0120E8
:107920002870281D03F04BFB204604F02AFA044679
:10793000281D03F06AFB204601B030BD30B5044677
:10794000064D81B0281D03F03AFB204604F079FB78
:10795000281D01B0BDE8304003F057BB64D90300D7
:107960002DE9F04705460E46B5F80370334C2078F4
:10797000401C2070802080F3118800BF00BF607819
:10798000401C60702878052803D1FCF7EDF980468B
:1079900001E04FF0000808EB070000F10D0A504627
:1079A000FFF7B4FF8146B9F1000F11D151460FF234
:1079B000940001F0C1FA6078401E6070C0B20028E7
:1079C00002D1002080F31188BDE8F047FEF74CBFDC
:1079D000B5F803004044A5F803000D2229464846A7
:1079E000FAF774FD3A46314609F10D00FAF76EFDDB
:1079F000B8F1000F04D007EB09000D30FCF7BDF91A
:107A0000B5F8030000F10D0189B24846FDF735FED7
:107A10006078401E6070C0B2002802D1002080F360
:107A20001188FEF721FFB9F1000F04D04846BDE8E8
:107A3000F047FFF783BFBDE8F0870000705E0300EA
:107A4000FDF715BE747862756666657220697320ED
:107A50006E6F7420616C6C6F63617465642825645B
:107A60002921210A0000000038B50446002500E065
:107A70006468002C0CD0207A0A789042F8D1E06833
:107A80004A689042F4D120698A689042F0D1012579
:107A900029460FF26420FCF71FF9002D00D10024C5
:107AA000204632BD38B504462020FFF72FFF05469B
:107AB00000222021FAF7DCFC0C22214605F1080007
:107AC000FAF714FD60686861A068A8610120287752
:107AD000284632BDF8B500231C4601F10805854A49
:107AE0001678761C1670802686F3118800BF00BFBA
:107AF0005678761C567006686F6801E034467668E2
:107B0000002E04D0D6F80CC06745F7DA0123002B0D
:107B10000AD033680B604E603368002B01D0596087
:107B200000E00160316005E0002C02D061600C6073
:107B300000E001605078401E5070C0B2002802D1B1
:107B4000002080F31188FEF78FFE0020F2BD10B5F3
:107B5000684C2278521C2270802282F3118800BF68
:107B600000BF6278521C62704A680B68002B01D01B
:107B70005A6000E002604868002801D00A6802608C
:107B80000846FFF7DBFE6078401E6070C0B2002838
:107B900002D1002080F31188FEF766FE002010BDA0
:107BA00030B40268002A03D0C168D368994200D07B
:107BB0004268002A28D04F490B785B1C0B70802349
:107BC00083F3118800BF00BF4B785B1C4B70D368F8
:107BD00052699A1AC3689C1A92FBF3F503FB05439A
:107BE000436103699C1A92FBF3F203FB0242826138
:107BF0004878401E4870C0B2002802D1002080F3AF
:107C0000118830BCFEF730BE30BC704770B50446FA
:107C10000D462068FFF728FF06000BD12846FFF726
:107C200041FF064631462046FFF754FF3046FFF736
:107C3000B7FF02E0307F401C3077207A401C207272
:107C4000307A002800D16660002070BD10B504466F
:107C50002068FFF709FF002801D1032010BD017F34
:107C6000491E0177217A491E2172017A002901D12A
:107C700000216160017F002903D101462046FFF702
:107C800066FF002010BD70B51A4A13785B1C137094
:107C9000802383F3118800BF00BF53785B1C5370AF
:107CA000006801E083614068002815D043695C1AD0
:107CB00083695B1A012C05DAC568661994FBF5F433
:107CC00005FB14644461012BECDA04691D1993FB74
:107CD000F4F304FB1353E5E75078401E5070C0B234
:107CE000002802D1002080F31188FEF7BDFD00209E
:107CF00070BD0000705E03002366632025640000F1
:107D0000002141810181704738B50446002926D001
:107D1000002C24D0B4F90800B4F90A2010182288E5
:107D200090FBF2F302FB13036088024665689BB286
:107D300000FB0350FAF7CAFBB4F90A002188884215
:107D400002DA401C608131BD09D12089401C2081AC
:107D500000B2218890FBF1F201FB1200208131BDBD
:107D60002DE9F04104460D461646002D3ED0002C6C
:107D70003CD0B5F9081008462A881346374607EB69
:107D8000000C634509DB698801FB07F26B6801FBA6
:107D900000312046FAF79AFB1CE01B1ABB4201DBBC
:107DA000B04603E0A2EB01081FFA88F8698801FBDE
:107DB00008F26B6801FB00312046FAF787FB688800
:107DC000A6EB080189B200FB01F2696800FB0840DC
:107DD000FAF77CFBB5F908003818298890FBF1F216
:107DE00001FB120028816889801B6881BDE8F08151
:107DF000B0F90A10408811FB00F080B27047B0F96A
:107E00000A0080B27047000080B5FDF7E7FC0090E3
:107E100000A800F083F8042000F087F8444801F03F
:107E20002EF801BD70B5424C2046C068C0460546DC
:107E3000FCF7C1FE0646B54212D031462846FDF792
:107E4000D3FF3146204604F089FB002E204603D0A4
:107E5000BDE8704001F013B8BDE8704001F03AB8D9
:107E600070BD10B582B000200090FDF7A5FD002187
:107E7000022001F059FD23E00098FDF75BFE2D483C
:107E80000178491C0170FDF7C8F8FEF7EDFC00A968
:107E9000294804F071FB0028EED0200702D5082005
:107EA000FCF7D7FFE00602D51020FCF7D2FFA006B2
:107EB00002D52020FCF7CDFFA00701D5FFF7B2FFC8
:107EC0003E2004F077FB04466007E0D4E5E710B5F8
:107ED00084B0174C04F114030822042104F1680053
:107EE00004F08AFB022002904FF40060019004F13C
:107EF00080000090114B50220FF24C0104F134002D
:107F000004F086FB4FF47A720D49204604B0BDE8B8
:107F1000104000F0A8BF0648C068704780B5014611
:107F2000054804F0A7FB40B202BD064904F0C0BBFF
:107F300030790300705E030098790300638E0000BF
:107F4000098E00006479030073656E736F725F744D
:107F500061736B00506002604160086070470A689E
:107F6000F8E748600160704701684068F9E7002061
:107F700007E0364901EBC00241F830201146496064
:107F8000401C0928F5DB704710B402680B4600E07E
:107F90001268824204D09468A342F9D1104600E0EE
:107FA000002010BC70472DE9F04104460D462646DE
:107FB000264F57F8368008E0D8F80820100002D085
:107FC000294620469047D8F8008007EBC600804538
:107FD000F2D10020BDE8F08138B50C46092801DA5D
:107FE000210007D1224601460FF2640000F0A4FFF1
:107FF000032032BD154901EBC00521462846FFF795
:10800000C3FF002806D10C20FFF780FC84602946BE
:10801000FFF7A5FF002032BD70B504460D460B48A2
:1080200000EBC400FFF7B0FF060007D12A46214647
:108030000FF2340000F080FF032070BDFFF794FFC3
:108040003046FFF77BFC002070BD000064D30300C6
:1080500061626E6F726D616C2072656769202825A0
:10806000642025782900000061626E6F726D616C7A
:1080700020756E726567692825642C2578290000B3
:10808000D2B2203A22BF00FA02F1002070475242D9
:10809000D041D2F1200291404140D0409040414037
:1080A00070470000012100F01F029140DFF84C21D1
:1080B000400942F820107047012100F01F02914052
:1080C000DFF83C21400942F82010704780B50FF2DC
:1080D000481000F031FFDFF82C0100210160416100
:1080E0000161BDE8014004F00EBB70477CB504F0AF
:1080F00016FB04460D46444ED6E900239D4208D89F
:1081000001D3944205D2CDE900450FF2C01000F032
:1081100013FFC6E90045204629467CBD80B504F022
:10812000FEFA4FF47A72BDE8084004F05FBCF8B57F
:1081300004460D4616461F4645EA040030430FD15B
:1081400021460FF2CC1000F0F7FE4FF4AD720FF2A3
:10815000E4010FF2D40000F0EFFE0020C046C0465C
:10816000B6F57A7F08D34FF47A70B6FBF0F0451974
:108170004FF47A7101FB1066B5F57A7F08D34FF49E
:108180007A70B5FBF0F004194FF47A7101FB1055C9
:1081900000F025F81B4A069810701C4864216943BA
:1081A00000FB041030180021C2E90201380000D0A1
:1081B000176132462946204604F0DBFABDE8F1405B
:1081C00002E010480078704780B5012004F0DBFB26
:1081D00001200C4988701420BDE8024062E780B598
:1081E000002004F0D0FB074800218170C0780028EF
:1081F00003D11420BDE802405EE701BD00E100E0CC
:1082000080E100E0E0D8030028DA030040420F00DC
:1082100000200146704700005B495D727463496E3F
:1082200069742E2E2E0A00005B455D25732C2025D7
:10823000640A0000443A5C506572666F7263655C64
:1082400053454E534F525F534C4F434154494F4E49
:108250005F494E4E4F565F313731365F38415C4390
:108260004F4E464944454E5449414C5C53656E73EC
:108270006F724875625C4D4153535F50524F4A458F
:1082800043545C50524F445C4135315C545C706CDB
:108290006174666F726D5C6578796E6F73393631B3
:1082A000305C6669726D776172655C6F735C706C6F
:1082B0006174666F726D5C6578796E6F735C7372F2
:1082C000635C7274635C7274632E63005B455D4F24
:1082D0006F7073212C206C6173745F737973746594
:1082E0006D5F74696D655F6E7365632028256C6CC6
:1082F00075292C2073797374656D5F74696D655F82
:108300006E7365632028256C6C75290A00000000D7
:108310005B455D7274635365745469636B54696D36
:10832000652829202D207365632825642920697319
:1083300020696E76616C69640A00000035488168C6
:10834000002904BF08B008E0EFF30982A2F1280277
:10835000036882E8F84F83685A60FEF7F7F981688E
:1083600079B14A6892E8F84F036002F1280282F37B
:10837000098890692849814202D013F47F4F43D085
:108380007047264826490968401A80F308884FF04C
:108390008071C161234981617FF0060E704701BC85
:1083A0002046DFF884E000BDFEE7204800681C4955
:1083B0000968401A203820F0070080F308884FF041
:1083C00000011448417081F3118862B600F018F87A
:1083D000FEE703680CB44FF0000141704FF000015C
:1083E00081F311881249134A0A604FF0800181F32A
:1083F00011880CBC036070470D490E4A0A60704733
:108400000B490C4A0A6070474FF0000181F3118854
:1084100070470000705E0300EE930000E81F030049
:108420009C160200091B0200A99300000010000026
:1084300004ED00E00000001004F00CBB80B5212822
:108440000BDB25220FF2C4110FF2B41000F074FD03
:108450000020BDE8024005F0E3BABDE8044004F0A6
:1084600009BB80B521280CDB2E220FF2A0110FF2E0
:10847000901000F061FD0020C046C0464FF0FF3074
:1084800002BDBDE8024004F013BB80B521280BDB20
:1084900039220FF278110FF2681000F04DFD002024
:1084A000BDE8024005F0BCBABDE8044004F01DBBC5
:1084B00080B521280CDB45220FF250110FF240103D
:1084C00000F03AFD0020C046C0464FF0FF3002BD2C
:1084D000BDE8024004F027BB80B521280BDB512208
:1084E0000FF228110FF2181000F026FD0020BDE851
:1084F000024005F095BABDE8044004F033BB80B5F6
:1085000021280BDB5E220FF204110FF2F40000F0C1
:1085100013FD0020BDE8024005F082BABDE804402A
:1085200004F03EBB80B521280BDB6A220FF2DC0190
:108530000FF2CC0000F000FD0020BDE8024005F085
:108540006FBABDE8044004F049BB80B521280BDBBD
:1085500076220FF2B8010FF2A80000F0EDFC002027
:10856000BDE8024005F05CBABDE8044004F054BB2D
:1085700038B521280BDB85220FF290010FF2800025
:1085800000F0DAFC0020BDE8324005F049BA0529C8
:108590000BDB8A220FF274010FF2640000F0CCFCB6
:1085A0000020BDE8324005F03BBA012A0DD1802BF6
:1085B0000BD38F220FF254010FF2440000F0BCFCE9
:1085C0000020BDE8324005F02BBA049C250002D003
:1085D000009405F039FA31BD80B521280CDB4FF449
:1085E00087720FF228010FF2180000F0A5FC00209E
:1085F000BDE8024005F014BABDE8024004F0BCBB7F
:108600005B455D25732C2025640A0000443A5C50CC
:108610006572666F7263655C53454E534F525F538C
:108620004C4F434154494F4E5F494E4E4F565F3178
:108630003731365F38415C434F4E464944454E54CE
:1086400049414C5C53656E736F724875625C4D4175
:1086500053535F50524F4A4543545C50524F445C11
:108660004135315C545C706C6174666F726D5C6531
:1086700078796E6F73393631305C6669726D776107
:1086800072655C6F735C706C6174666F726D5C6553
:1086900078796E6F735C7372635C6770696F5C6727
:1086A00070696F2E6300000080B505F0BEFA0D49B9
:1086B000086001BD80B500F0E7F80B4806F0ECF962
:1086C000012006F008FAFFF7B7FE06F075FA06F08B
:1086D00087FAFFF7FBFC0FF21400BDE8024000F040
:1086E0002BBC00000C67030000EA32065379737458
:1086F000656D20626F6F7420646F6E65202121218B
:108700000A00000010B588B0044600A81421F9F74B
:1087100025FF05A800210A460B460EC00D22214662
:1087200000A8F9F7D3FE04F10D00CDF80D009DF877
:108730000010062904DB0FF22C10FBF7CDFA58E0ED
:108740009DF80000002801D0022910D1BDF80300D7
:1087500000280CD00422DDF80D1006A8F9F7B6FEAB
:108760000422DDF80D00011D07A8F9F7AFFE9DF802
:10877000000004283DD8DFE800F0030B131B2C0099
:10878000DDF80D2005A99DF80100FCF73FFA30E067
:10879000DDF80D2005A99DF80100FCF793FA28E00B
:1087A000DDF80D2005A99DF80100FCF7D7FA20E0BF
:1087B0009DF80100FF2803D100A8FDF775FA18E025
:1087C000DDF80D30BDF803209DF80210FCF70AFB20
:1087D0000FE09DF80100FF2803D100A8FDF7DFFAA4
:1087E00007E0DDF80D30BDF803209DF80210FCF71E
:1087F0000BFB08B010BD00B591B000A84021F9F7FF
:10880000ADFE00A9144806F0F5F900A8FFF77AFFBD
:10881000F7E710B584B0114C23461022402104F232
:10882000344003F0E9FE022002904FF4966001907C
:1088300004F24C4000900A4B5A220FF2400104F51A
:10884000806003F0E5FE1FBD80B50146024803F0DD
:1088500011FF40B202BD00006874030034700300D1
:10886000F79700005B4552525D206F76657220439A
:108870004D44204D4158202578000000636D645F11
:108880007461736B0000000080B506F0D2FA06F048
:10889000B5FB06F032FCBDE8014006F08FBCF8B530
:1088A00004460D4616461F46002C0DD10FF2F0006F
:1088B00000F042FB36220FF218110FF2081000F000
:1088C0003BFB0020C046C046002D0DD10FF2A0108A
:1088D00000F032FB3B220FF2F8010FF2E80000F04B
:1088E0002BFB0020C046C04606F0BEFC002805D188
:1088F0003A4631460FF2981000F01EFB29462046FA
:10890000BDE8F44006F074BBF8B504460D461646C3
:108910001F46002C0DD10FF2941000F00DFB4922E0
:108920000FF2AC010FF29C0000F006FB0020C046E5
:10893000C046002D0DD10FF2941000F0FDFA4E222A
:108940000FF28C010FF27C0000F0F6FA0020C04616
:10895000C04630000DD10FF2941000F0EDFA532212
:108960000FF26C010FF25C0000F0E6FA0020C04646
:10897000C0463B4632462946204601B0BDE8F0409D
:1089800006F030BB10B5044606F0A4FB012C04D061
:108990002046BDE8104006F082BB10BD000000007C
:1089A0005B455D6D61696C626F78577269746528AB
:1089B00029202D20627566206973204E554C4C0A83
:1089C000000000005B455D25732C2025640A000033
:1089D000443A5C506572666F7263655C53454E53F2
:1089E0004F525F534C4F434154494F4E5F494E4E97
:1089F0004F565F313731365F38415C434F4E464901
:108A000044454E5449414C5C53656E736F724875D2
:108A1000625C4D4153535F50524F4A4543545C5042
:108A2000524F445C4135315C545C706C6174666FCC
:108A3000726D5C6578796E6F73393631305C66695A
:108A4000726D776172655C6F735C706C6174666F78
:108A5000726D5C6578796E6F735C7372635C6D6167
:108A6000696C626F785C6D61696C626F782E63000F
:108A70005B455D6D61696C626F78577269746528DA
:108A800029202D2073697A6520697320300A00003F
:108A90005B495D6D61696C626F7857726974654599
:108AA00076743A202573282564290A005B455D6D9C
:108AB00061696C626F78526561642829202D20629B
:108AC0007566206973204E554C4C0A005B455D6D00
:108AD00061696C626F78526561642829202D20736A
:108AE000697A6520697320300A0000005B455D6D7E
:108AF00061696C626F78526561642829202D20635A
:108B0000616C6C6261636B206973204E554C4C0A3A
:108B10000000000010B5044606F08EFD0120054956
:108B2000605410BD002106F0F6BD06F040BF06F00F
:108B300097BF000030DA03000C2802D36FF4004026
:108B40007047854A42F8201007F00FB92DE9F84F19
:108B500004460C2C80F0898007F07AFA05467F489D
:108B600010F8146000EB440047783046FFF779FCBA
:108B700080463846FFF775FC8146204607F031F9FC
:108B80003846FFF795FC83463046FFF791FC824656
:108B9000524659460FF2C81000F0CEF9BBF1010F52
:108BA00063D0BAF1000F1AD14FF0000B04E00A2095
:108BB00004F024FF0BF10A0BBBF5FA7F08D2304614
:108BC000FFF776FC8246BAF1000FF0D14FF0000BB0
:108BD000BBF1000F03D00FF2A81000F0ADF938463A
:108BE000FFF766FC8346BBF1000F2DD10121304613
:108BF000FFF724FC00213846FFF720FC4FF0000A65
:108C000001E00AF1010ABAF1640F16DA00213046D8
:108C1000FFF73BFC052004F0DDFE01213046FFF7A5
:108C200034FC052004F0D6FE3846FFF741FC01284D
:108C3000E7D10FF26C1000F07FF9BAF1640F03D1A5
:108C40000FF2781000F078F941463046FFF7F6FB56
:108C500049463846FFF7F2FB204606F08DFF2946CD
:108C60002046BDE8F44F07F080B8BDE8F18FF0B5BD
:108C700087B004461D460C2C01D2080602D56FF4BD
:108C800000401CE001910D9E03960C980590049500
:108C9000069201A9204607F087F9070004D0204674
:108CA000FFF754FF38460AE00E98010006D0002175
:108CB000009133462A460F9907F0D2FA002007B0F8
:108CC000F0BD39E71FB5069C002C01D0002B02D166
:108CD0006FF4004009E02270002203920292019397
:108CE000009401232246FFF7C2FF04B010BD2DE916
:108CF000FF4705460E4690469946DDF830A0BAF18A
:108D0000000F02D0B9F1000F02D16FF4004020E053
:108D100009F101073846FEF7F9FD040002D14FF0D2
:108D2000FF3016E04A465146601CF9F7CFFB84F845
:108D30000080002003900290019000903B46224664
:108D400031462846FFF793FF05462046FEF7F6FD1D
:108D5000284604B0BDE8F0875CD603008C650300AC
:108D60005B495D534441206C696E653A25642C2053
:108D700053434C206C696E653A25640A000000007C
:108D80005B455D53434C206C696E652069732073AD
:108D900074696C6C204C4F572121210A000000009F
:108DA0005B495D534441206C696E65206973207294
:108DB00065636F76657265640A0000005B455D530C
:108DC0004441206C696E65206973206E6F74207257
:108DD00065636F76657265640A0000007047000085
:108DE00030B4544982680B6A9A1882600122027476
:108DF0004A692AB9026048610FF23100C8610CE08B
:108E000001F1140384689568651B012D03DB13468B
:108E10001A68002AF7D10260186048694A6A8068B7
:108E2000821A48BF486230BC7047000010B5044643
:108E300010E0A0610168616100210174A069816096
:108E400081F31188A06940688047802080F31188F1
:108E500000BF00BF606928B18168226A8A1A012AAE
:108E6000E7DB616210BD30B4002300241D4638C02A
:108E700018C01438C2608260416030BC704710B5C1
:108E8000802181F3118800BF00BF017C294CC1B152
:108E900004F1140100E011460A6892B182420ED03A
:108EA00011460A686AB1824209D011460A6842B185
:108EB000824204D011460A681AB18242EBD102689C
:108EC0000A60C1688160FFF78BFF607808B980F3A2
:108ED000118810BD802181F3118800BF00BF027C82
:108EE00014490AB30022027482680B6AD21A8260A3
:108EF00001F1140200E01A46136893B183420ED0C8
:108F00001A4613686BB1834209D01A46136843B1FD
:108F1000834204D01A4613681BB18342EBD1006828
:108F20001060486900B9C861487808B980F31188B1
:108F300070470000705E03000EB400B582B003A954
:108F40000091024600AB0121034878440A3000F04A
:108F5000A9FF06BC5DF810FB0BDD0100010040F12C
:108F60000980F446404200F005F851F000416047A6
:108F7000010000BF09D0B0FA80F18840C91CC1F5DA
:108F80008461090501EBD0214005704780B54FF0A1
:108F9000FF3251EC100B07F06BF941EC100B01BDE7
:108FA0002DE9F8452DED088B0FB486B040F2FF7126
:108FB00007989DED080B8DED040BC0F30A50884215
:108FC00008D107980024000305BF06980028022551
:108FD000012512E0012807DA06A807F0F9FA0128AE
:108FE00002DB0024002508E0079A40F2FE3161F31D
:108FF0001E520792441A4FF0FF35002104A807F0D3
:1090000008FB1A9F06460FB10020388036B9DDE90B
:1090100008230020002107F03BFB12D0002D13D5C0
:1090200024B2012C15D1DDE906230020DFF88C13D2
:1090300007F02EFB05D0012E0BD1DF4907F028FBEE
:109040003ED10AB0CD49E8E1022D04D1DDE90601A7
:10905000E2E1012E6FDB022E08BFDDE9080100F01E
:10906000DB81012D2AD107980028099806D4002811
:1090700054BF9FEDD50B9FEDD60BCBE100280ED44E
:1090800056B94FF0FF3104A807F0C3FA002848BFD3
:109090009FEDD10B00F1BE819FEDCB0BBAE156B92C
:1090A0004FF0FF3104A807F0B4FA002848BF9FED45
:1090B000B40B00F1AF819FEDC60BABE1012E11D1D6
:1090C0000998002824B206D4012CACBF9FEDBE0B3A
:1090D0009FEDBF0B9EE1012CACBF9FEDBD0B9FED43
:1090E000BA0B97E10998002810D466B94FF0FF3108
:1090F00004A807F08EFA002842BF079800289FEDC9
:10910000A00B00F187819FEDB20B83E107F0D0FA4D
:109110002221016066B94FF0FF3104A807F079FA07
:10912000002842BF079800289FEDAB0B00F1728129
:109130009FEDA50B6EE10798002848BF002E0CD5C7
:1091400007F0B6FA212101600AB04FF0FF30BDEC04
:10915000088B6FF00041BDE8F485DDE906010022CF
:109160000023FDF7F7F938BF002509D381F000414E
:10917000CDE906014FF0FF3104A807F04AFA054691
:10918000012C13D1DDE906017F4A804BFDF7FAF986
:109190000CD2DDE9062300269FED7D8B00204FF0E9
:1091A0008041FDF71DF8CDE906011CE0DDE906234D
:1091B0009FED798B00207A49FDF712F853EC182BBC
:1091C000FDF70CF9FDF7DEF8A0F120063046FFF7B9
:1091D000C5FE0022734BFDF703F853EC182BFDF787
:1091E000FDF841EC180B0FF2582000EB461ADDE9B0
:1091F000060153EC182B00F095FDDDE9062341EC48
:10920000190B51EC180BFDF7E9F802460B4651EC2F
:10921000190B01F079FD41EC1A0B53EC1A2BFCF7FA
:10922000DFFF41EC1B0B8DED069B07F053F953EC70
:109230001B2BFCF7D5FFDDE9062300F073FD064686
:10924000884600204D4953EC182B00F06BFD00229E
:109250004FF08043FCF7C4FF32464346FDF7BEF8AB
:1092600053EC1A2BFCF7BCFFDDE90623FDF7B6F83B
:1092700041EC180B4C4A4D4B01F046FDCDE9040181
:109280002046FFF76BFE41EC190BDAE9000153ECC5
:10929000192BFDF7A3F8DDE90423FDF79FF8CDE9CD
:1092A0000401DDE90823FCF79BFF0022404BCDE9D8
:1092B0000201FDF767F9C0F0938001223D4BFDF7F5
:1092C00049F940F2918000220023FDF75BF9DDE9C6
:1092D000022339BF0020384900203849FDF77EF8C5
:1092E000FDF750F80446DDE9080153EC182BFCF7B4
:1092F00077FFCDE90201DAE90223DAE904019FED03
:10930000308BFDF76BF8DDE90823FCF769FF53ECC0
:10931000182BFCF765FFDDE90223FDF75FF8CDE9C7
:109320000201DAE9002351EC190BFDF757F8DDE9EA
:109330000823FCF755FF064688462046FFF70EFE39
:1093400002460B463046414600F0ECFC53EC182B2D
:10935000FCF746FFDDE90223FDF740F8CDE9020105
:109360000FB13C80002400940022044B02A807F0B7
:10937000A5F9A8B3012837D042E000BF0000F03FB4
:109380000000000000000080CD3B7F669EA0E63F0D
:10939000000000000000F03F000000000000E03F7F
:1093A000000050400000903FEF39FAFE422EE63FA9
:1093B0000000E0C00000E0400000E0BF0000E03F2F
:1093C000EF39FAFE422EE63F000000000000F07F79
:1093D0000000000000000000000000000000F0FF9E
:1093E0000020CDE9020007E00020014902E000BFB3
:1093F0000000F07FCDE9020107F05AF92221016057
:10940000002D1DBFDDE9020181F0004141EC100B90
:109410009DED020B51EC100B0AB0BDEC088BBDE8C2
:10942000F48580B50020009053EC112B51EC100B0B
:10943000FFF7B6FD41EC100B01BD0000000000007D
:10944000000000000000F0BF0000000000000080ED
:10945000000000000000008000000000000000008C
:10946000000000C05294EEBF00000048204E51BEE4
:10947000000000F86467BCBC0000000000000000B1
:10948000000000208133EDBF00000080B3DB14BE7C
:10949000000000506706A3BC0000000000000000B0
:1094A000000000D0E9DCEBBF00000008C39259BE09
:1094B00000000080B0D3B8BC000000000000000035
:1094C00000000070F98FEABF000000C0A51028BEA0
:1094D000000000E8BFC0B0BC0000000000000000B9
:1094E00000000070284CE9BF00000060134B42BE32
:1094F000000000C03D20B8BC0000000000000000DB
:1095000000000050FA10E8BF000000C05FF62BBE5C
:10951000000000905C71A7BC00000000000000008B
:1095200000000020FCDDE6BF000000C0F8F154BEE2
:1095300000000018E9F6B9BC0000000000000000BF
:10954000000000D0C3B2E5BF00000070E43254BE9A
:1095500000000050DB06B4BC00000000000000006A
:1095600000000010EF8EE4BF00000020F36252BE46
:10957000000000C02A879ABC000000000000000024
:10958000000000B02272E3BF000000F0E8E056BE29
:1095900000000028352DBDBC0000000000000000C8
:1095A000000000000A5CE2BF000000B0FA8E41BE7D
:1095B00000000040AE6FBDBC0000000000000000D5
:1095C00000000000564CE1BF000000F015CD5FBE6A
:1095D00000000000141C90BC00000000000000000F
:1095E00000000040BD42E0BF00000030F93457BE2B
:1095F000000000E06C1E93BC0000000000000000B2
:10960000000000E0F57DDEBF000000B08A535EBEC2
:1096100000000080DA77AABC000000000000000013
:10962000000000C09D81DCBF00000000FFA226BE3C
:109630000000006057E2B0BC000000000000000025
:1096400000000060F98FDABF000000580A8151BEA7
:10965000000000F05F60B8BC0000000000000000E7
:109660000000000098A8D8BF000000607A7F45BEC7
:10967000000000D05433A3BC000000000000000034
:10968000000000600FCBD6BF000000D091CB40BEE1
:10969000000000406D1BA0BC0000000000000000A6
:1096A000000000A0FBF6D4BF00000098C5CE52BE5B
:1096B000000000003A397EBC0000000000000000FD
:1096C000000000E0FE2BD3BF0000004073872BBEDC
:1096D00000000000926879BC00000000000000005B
:1096E00000000040C069D1BF00000058F16353BEC4
:1096F00000000080438D7CBC0000000000000000E2
:1097000000000080D85FCFBF000000181F8354BE48
:10971000000000B03F42A2BC0000000000000000BA
:109720000000008067FCCBBF00000060FAFF53BE62
:1097300000000050E00DB8BC000000000000000078
:109740000000000098A8C8BF000000607A7F35BE06
:10975000000000C0543393BC000000000000000073
:1097600000000000DC63C5BF00000058D6FF54BEF7
:1097700000000000396490BC000000000000000000
:10978000000000C0AD2DC2BF00000080A45915BE6E
:10979000000000E0484BABBC0000000000000000EF
:1097A000000000801A0BBEBF00000050BF3C5ABE34
:1097B000000000A0B364B6BC000000000000000080
:1097C0000000008004D6B7BF00000040BBCF36BE0B
:1097D0000000008076CEA8BC000000000000000061
:1097E0000000008032BBB1BF000000402A0043BE31
:1097F00000000028C60CBDBC0000000000000000F6
:10980000000000009473A7BF000000182B3B59BE56
:10981000000000C0E55DA5BC0000000000000000E5
:1098200000000000EE4397BF000000A0E6C340BE6A
:1098300000000020958DB5BC000000000000000075
:109840000000000000000080000000000000008018
:109850000000000000000080000000000000000088
:1098600010B584B000A80FF2DC011CC91CC0002296
:1098700000A9CD20FBF7CAF9002004B010BD0020DC
:10988000704730B58BB0050001D102204AE00020BE
:10989000029001902C780422691C02A8F8F716FEA9
:1098A0000422691D01A8F8F711FE21460FF2A0005D
:1098B000FFF742FB2046FBF7C0FA00281DD0002529
:1098C000406A00280DD103A829460A460B460EC05F
:1098D000029804900198059003A92046FBF796F999
:1098E0000125FCF7C1F8012803D10820FCF79CF8FA
:1098F0000125002D01D0002014E006A80FF264011C
:109900001422F8F7F3FD00A80FF26C010A68026058
:109910008DF802400320ADF81B0000A906A8FEF751
:109920001FF802200BB030BD002803D0022805D05C
:1099300002D305E00846A2E70846A2E708468FE7FB
:10994000002070470100000014000000000000002B
:1099500023234548206E6F206576656E7428256444
:10996000290A0000050000000000000000000000BF
:1099700000000000000000000A1A000038B50C4684
:10998000082820D1854DE8688DF8000000AA012143
:1099900049206B691B6998472078002813D000EE96
:1099A000100AB8EE400ADFED7C0A80EE200A85ED51
:1099B000040A10EE100AFCF7EBFB02460B460FF20E
:1099C000E810FAF789F9002032BD10B50020734C79
:1099D00000E00120002806D1A06980470028F8D1C6
:1099E00004F1180060616369002B05D10FF2C41007
:1099F000FAF772F9032010BD04F108020021472094
:109A00005B699847002010BD10B5044664490820E2
:109A1000FEF7E2FA2046614949694968BDE810400D
:109A2000084713B586B002A81021F8F797FD00A8E3
:109A300000210A4606C0594C616989688847002898
:109A400001D001206AE0062202A900A8F8F74EFD25
:109A5000FCF712F801284ED1E06801284BD194EDB3
:109A6000040AF7EE000A70EEC00ABDF9000001EE2C
:109A7000100AB8EEC11A21EE001AB4F9000001EE86
:109A8000900AF8EEE11A00EEA11ABDEEC11A11EE2D
:109A9000100AADF8000000A8B0F9021001EE101A8B
:109AA000B8EEC11A21EE001AB4F9021001EE901AB4
:109AB000F8EEE11A00EEA11ABDEEC11A11EE101A6D
:109AC0004180B0F9041001EE101AB8EEC11A21EE6F
:109AD000000AB4F9041001EE101AB8EEC11A00EE33
:109AE000810ABDEEC00A10EE101A8180062200A97C
:109AF00002A8F8F7FBFCBDF80000208000A8418810
:109B000061808088A080082206A90DF10E00F8F778
:109B1000DDFC02A90120FCF7CDF9002008B010BD42
:109B200010B504461E490820FEF776FA20461B4968
:109B30004969C968BDE810400847F8B504460D46B4
:109B40001646164F252C05D13178F9600FF26C00BE
:109B5000FAF7C2F83246294620467B691B6901B0F4
:109B6000BDE8F04018470D4B5B695B6918470B482F
:109B700090ED020A70470B4901F11002C261012207
:109B800002700422427006228270012202820E229A
:109B900042824161002070470000C842C45F030058
:109BA0007DA90000A460030041434F45464620259F
:109BB0002E32660041434320504600004C50462060
:109BC00073746174757320203A20256400000000CE
:109BD0000246012148204F4B5B685B69184770B50E
:109BE00000244C4D00E0641C012C0ADA04EB440014
:109BF00005EBC006B06880470028F4D106F10800E4
:109C000068606B68002B05D10FF21010FAF764F84A
:109C1000032070BD2A46002147205B699847002039
:109C200070BD10B53B4C616849688847002801D079
:109C3000012010BD002204F12001A120FAF7E6FF67
:109C4000002801D0032010BD30A0FAF745F800200D
:109C500010BD83B584B000A81021F8F77FFC00A8E0
:109C60002C49496889688847002801D001200AE00A
:109C7000082204A90DF10600F8F728FC00A9042029
:109C8000FCF718F9002007B000BD10B5214C616841
:109C9000C9688847002801D0012010BD002204F1C6
:109CA0002001A120FBF70EF8002801D0032010BDF1
:109CB00017A0FAF711F8002010BD164B5B685B691E
:109CC0001847144B5B681B69184710B5114C04F119
:109CD0002C020121472063685B69984704F12C003E
:109CE00010BD0C4890ED000A70470B4901F11002BD
:109CF000C261042202704270062282700122028236
:109D00000E224282416100207047000047594F00F7
:109D1000475943005C5F0300F460030047594F203C
:109D20005046000070B44FF0004591EA030F44BF65
:109D30006B40FCF75DBB00BF841A71EB030604D2D5
:109D40006E40001BB141121973414FF4001C1CEB13
:109D5000410F34BF7CEB430684E00C0DA4EB13569B
:109D6000362E7DDC012E43DC45EAC32343EA525301
:109D700012BFD20292025B08240545EAC12141EAE2
:109D80005051D2EBC020994125D407D1B0FA80F6CA
:109D900010FA06F164D00020203608E0B1FA81F60E
:109DA000B140C6F1200220FA02F21143B0404FEA5E
:109DB000F474B4EB465434F001064FEA74040AD844
:109DC000D6F50016760D04F00044F04061FA06F274
:109DD0005040F1404840C00A40EA415021F0004163
:109DE00028BF5FEA500550F1000044EBD12137E075
:109DF00045EAC323DB0A45EAC121C90AB6F12005B9
:109E00000EDD42EA0242120CC5F1200603FA06F604
:109E1000EB4042EA06056D42984161F100010DE018
:109E200062FA06F5F240554063FA06FC82EA0C023B
:109E3000F3405A406D42904161EB030111F4801FE1
:109E400005D1641E620502D06D004041494121F4F4
:109E50008011430875F1004350F1000041EB0451BB
:109E600070BC70471CEB410F15D223F0004352EA3F
:109E700043060BD04FEA4C0CBCEB410F04D80C0D41
:109E8000661E342EB7DDEBE7801A994150EA410691
:109E900008BF0021E4E708BF1CEB430F28BF6FF0A9
:109EA0000001DDE72DE9F04FA1B082460020174602
:109EB0001D4602910B900DF1440B6FF000490AE032
:109EC00017F8011B0298D0470290002800F0A882E2
:109ED0000B98401C0B90387808B90B98A2E2252803
:109EE000EED10020059006900790089009900A9006
:109EF00001E040F0010017F8011F2029F9D02329C3
:109F00000DD02B2904D02D2906D030290AD00CE001
:109F100040F0020080B2EEE740F00400FAE740F0C3
:109F20000800F7E740F01000F4E72A290ED129686D
:109F3000296051F8042B2960002A0D9204D5514262
:109F400040F004000D9180B27F1C11E000210D91C2
:109F500009E00D99494505D001EB810302EB43016E
:109F600030390D917F1C3A78A2F130010A29F0D3E3
:109F700039782E2903D04FF0FF310C911DE017F8EE
:109F8000011F2A2907D1296829607F1C51F8042B59
:109F900029600C9211E000210C9109E00C994945CF
:109FA00005D001EB810302EB430130390C917F1C9A
:109FB0003A78A2F130010A29F0D3ADF838000FF653
:109FC0007440397806F0DEFC08B117F8010B8DF803
:109FD0003A009DF83A00682802BF39786829622063
:109FE00005D06C2804BF38786C2803D171208DF817
:109FF0003A007F1C11A8049017F8014BB4F125001A
:10A000002AD01C3800F0CC80001F022840F2C88003
:10A01000133800F0EE80093800F0C280801E00F096
:10A020004F81401E00F02481401E022840F2B8807B
:10A03000001F00F01D81401F00F08380401E00F0D3
:10A04000D880401E29D0C01E0CD0801E00F0D180C8
:10A05000C01E00F0CE803DE10120059025208DF846
:10A06000440043E12868286050F8044B28600394BA
:10A07000DDF83080B8F1000F04D52046FCF7B8FABF
:10A08000804607E042460021204606F087FC08B1E2
:10A09000A0EB0408CDF8188028E1296829604FF06A
:10A0A0003C0851F8040B29600021CDE9000111A8FA
:10A0B0000390DDE90001049C11B908B90C9AC2B102
:10A0C0000206120FA0EB02123032D2B23A2AA8BF17
:10A0D00027320009A8F1010340EA017009091A5565
:10A0E00008BF0028984604D0039A08EB04039A425C
:10A0F000E6D308EB04000390C8F13C010C980691EC
:10A10000814209DA401A08904FF6EF71BDF8380025
:10A110000840ADF83800E9E0002840F1E7809DF8FC
:10A12000380000F01400102840F0E0800D98059AE7
:10A13000801A089A801A401A0128C0F2D780089025
:10A14000D4E09DF83A0062281AD0682806D06A2820
:10A150000CD06C281CD0712808D019E02868286021
:10A1600050F8041B28600B980880BFE0286828601E
:10A1700050F8042B28600B98C117C2E90001B5E024
:10A180002868286050F8041B28600B980870ADE020
:10A190002868286050F8041B28600B980860A5E028
:10A1A0002868C01D20F007022A60D2E900010832A9
:10A1B0002A60CDE90001002903D5012005902D205A
:10A1C0000CE0BDF83800810703D5012005902B2055
:10A1D00004E0C00704D50120059020208DF844003C
:10A1E000059911A808180390214600A800F0D8F995
:10A1F0007CE09DF83A206C2A0DD0712A18BF6A2A9B
:10A2000009D12868C01D20F007032B60D3E90001A5
:10A2100008332B6005E02968296051F8040B296098
:10A220000021CDE90001682A08BF80B207D0622A68
:10A2300008BFC0B203D0742A18BF7A2A02D1002105
:10A24000CDE900019DF83800000730D5DDE90001B7
:10A25000002908BF00282AD044F02000782826D101
:10A2600030208DF844008BF80140022005901EE05C
:10A270009DF83A00294600F0D8F8CDE90001002900
:10A2800004DA0598411C05912D210EE0BDF8380037
:10A29000810704D50598411C05912B2105E0C007D5
:10A2A00005D50598411C0591202100F80B10059952
:10A2B00011A808180390214600A800F0EDF815E059
:10A2C000012005902868286050F8041B28608DF84C
:10A2D00044100BE0012005902520002C8DF844004F
:10A2E00004D00598411C059100F80B400D98059984
:10A2F000401A0899401A0699401A0999401A079974
:10A30000401A0A99A0EB01089DF8380040070FD4C5
:10A3100020208DF84000002408E0012310AA00A9A5
:10A32000504600F070FC00287AD1641C4445F4DBF0
:10A33000059C11AE0AE016F8011B0298D047029066
:10A3400000286DD00B98401C0B90641E002CF2D19D
:10A3500030208DF840000026089C08E0012310AA58
:10A3600000A9504600F04FFC002859D1761CA642A7
:10A37000F4DB069C039E0AE016F8011B0298D04706
:10A38000029000284CD00B98401C0B90641E002CAF
:10A39000F2D130208DF840000026099C07E001230F
:10A3A00010AA00A9504600F02EFCC8BB761CA6429D
:10A3B000F5DB03980699079C0E1809E016F8011BB7
:10A3C0000298D047029058B30B98401C0B90641E23
:10A3D000002CF3D130208DF8400000260A9C07E0C5
:10A3E000012310AA00A9504600F00DFCC0B9761C4C
:10A3F000A642F5DB9DF8380040077FF56CAD2020C4
:10A400008DF84000002400E0641C4445BFF663ADB5
:10A41000012310AA00A9504600F0F5FB0028F3D054
:10A420004FF0FF3021B0BDE8F08F622826D06828B9
:10A430001DD06A2808D06C2827D0712804D0742831
:10A4400023D07A280CD020E00868C01D20F0070037
:10A450000860D0E9002308300860194610467047AC
:10A460000A680A6052F8040B0A60002170470A6803
:10A470000A6052F8040B0A6000B20BE00A680A6036
:10A4800052F8040B0A6040B204E00A680A6052F80D
:10A49000040B0A60C11770472DE9FA4E05460A46BB
:10A4A0002F696F2A08BF082405D041F020007828C2
:10A4B00014BF0A2410243C26D5E90001642A18BFE1
:10A4C000692A81468A4605D1002903DAD9F10009B3
:10A4D0006AEB4A0ABAF1000F08BFB9F1000F0CD1BC
:10A4E000286B50B9082C36D195F83800000732D5C2
:10A4F00030203B2687F83B002DE0E31748465146C5
:10A500002246FBF7A9F9A4FB0023A9EB0202303293
:10A51000D2B2A6F1010B3A2A5E4603DB9DF8003069
:10A52000513B9A1881465FEA010A0BF8072008BFE1
:10A53000B9F1000F03D0E868F1198842DDD3082C87
:10A5400009D195F83800000705D5F05D302802D014
:10A55000761E3020F055C6F13C00A861F119E96083
:10A56000296B884208DA081A28624FF6EF71288FA3
:10A5700008402887BDE8F38E00290ED595F83810DD
:10A5800001F01401102908D1696B6A69891A2A6AD5
:10A59000891A081A0128A8BF2862BDE8F38E0000B6
:10A5A0002DE9F24F04468EB0D4E90001CDE9020155
:10A5B00004AF9DF8380040F0200BBBF1610F0AD0CA
:10A5C000206B002848BF062004D408BFBBF1670FEA
:10A5D00001D1012020636168C1F30A5040F2FF728B
:10A5E00090421CD1080304BF2068002809D1032031
:10A5F000A0619DF8380061381A2836D30FF24861FF
:10A6000008E00320A0619DF8380061381A2829D39A
:10A610000FF22C61E0680322F7F758FFBEE1012832
:10A6200016DA204605F0D4FF012811DB00250020B2
:10A63000BBF1610F20D1E168302201F8012B4A1CE7
:10A64000E2609DF83820612A0CBF782258220FE082
:10A65000626840F2FE3161F31E52451A62604FF0AB
:10A66000FF30E5E70FF2D451D4E70FF2D851D1E72C
:10A670000A706169891C616110B90026002584E1B6
:10A68000BBF1610F40F09780206B00284CBF212662
:10A69000461CDDE90201D4E900AB00220023FBF7F0
:10A6A00071FF36B23ABF8BF00040CDE902A0CDE990
:10A6B00002AB06F101082D1F8DF810200DF11107D6
:10A6C00000E0C71DB8F1010F33DBDDE90201002214
:10A6D0000023FBF73FFF2CD21C2102A806F08AF9C9
:10A6E000DDE90201FBF74EFEA8F10708B8F1010F02
:10A6F000814609DBFEF732FC02460B46DDE902012A
:10A70000FFF710FBCDE90201F81D072105E009F074
:10A710000F0200F8012D4FEA2919B9F1010F01DBF1
:10A72000491EF4D5491E5CBF002200F8012DF9D561
:10A73000C7E70DF11100391AB142B8BF0E4636B263
:10A7400030000DF111072FD4884206DA04A9411810
:10A7500049780829A8BF0F2100DA002104AA82182D
:10A7600000E0761E12F80139401E8B42F9D00F2905
:10A7700004D104A941184A78521C4A70002802D515
:10A7800004AF761C2D1D36B2701E0DD4C1190A7887
:10A790003032D2B23A2A03DB9DF838303A3B9A186D
:10A7A000401E01F80129F2D5206B002840F1ED8010
:10A7B000701E2063E9E0DDE9020100220023FBF7BF
:10A7C000E1FE3CBF81F00041CDE902012DB247F22C
:10A7D000975068434B49DFF8309190FBF1F52DB26B
:10A7E000C5F1070ABAF1010F90461CDBDDE90267EB
:10A7F0005FEACA7007D542464B4630463946FBF7FA
:10A80000EFFC06460F464FEA6A0A40464946424672
:10A810004B46FBF7E5FCBAF1000F80468946E7D1CD
:10A82000CDE9026724E0CAF1000A0026374F14E0A0
:10A830005FEACA7007D542464B4630463946FBF7B9
:10A84000CFFC06460F464FEA6A0A40464946424652
:10A850004B46FBF7C5FC80468946BAF1000FE7D1AD
:10A86000DDE9020132463B4600F04EFACDE9020135
:10A87000BBF1660F216BDFF898900CBF05F10A0061
:10A8800006204618142EA8BF132630208DF810007D
:10A890000DF11107012E3DDBDDE90201FBF788FD1B
:10A8A00007F1080104220A23B0FBF3F303EB83074B
:10A8B000A0EB4700303001F8010D0A20B3FBF0F0A7
:10A8C00000EB8007A3EB47033033521E01F8013D34
:10A8D000E9D1083E012E01F10807DBDBDDE90201C9
:10A8E000FBF766FDFEF744FB02460B46DDE902017D
:10A8F000FFF718FA00224B46FBF772FCCDE9020184
:10A90000CAE700BFA0860100000024400000F03F1D
:10A9100084D797410DF11100381A0DF1110702E0AB
:10A92000401E6D1E7F1C39783029F9D0BBF1660FAF
:10A9300002D12DB2691C04E0BBF1650F0CBF0121EF
:10A940000021226B8E1836B2B042B8BF064636B22E
:10A9500031001AD4814204DAC85D3528A8BF3920F5
:10A9600000DA3020CA19521E00E0761E12F80139B2
:10A97000491E8342F9D0392802D1C85D401CC85510
:10A98000002902D57F1E761C6D1C2DB29DF8381053
:10A99000009533B23A46204600F003F80FB0BDE808
:10A9A000F08F2DE9F043054685B01E46D5F830807E
:10A9B000012E8946174602DA01260FF2902749F048
:10A9C0002000BDF93040662808BF641C17D06728F6
:10A9D00040F0828014F1040FC0F28480444580F27C
:10A9E000818095F83800641C000702D44645B8BF42
:10A9F000B04624B2B8EB040848BF4FF0000824B2B8
:10AA0000E868A969012C25DA4A1C30230B54B8F1F7
:10AA1000010F03DA95F83810090702D52E211154D9
:10AA2000521C18EB040FB8BFC8F1000424B26142F5
:10AA3000A044B045AA61B8BF4646696236B2EE612D
:10AA40003246AB6939461818F7F740FDA8EB060007
:10AA5000A862C1E00818A64218DA32463946F7F76C
:10AA600035FDA9697118A01BA961B8F1010F6862D1
:10AA700003DA95F83800000705D5EA682E208854D7
:10AA8000E869401CE861C5F82880A5E022463946FF
:10AA9000F7F71CFDA8692018361BB8F1010F03DA7F
:10AAA00095F83810090703D5EA682E218154401C17
:10AAB000A86136B2B045B8BF4646E868AB6936B261
:10AAC0003246E1191818F7F701FDA8693018A86196
:10AAD000A8EB060068627FE0B9F1610F16D14FF074
:10AAE000700918E0464504DA95F83810090758BF90
:10AAF000B046B8F1010848BF4FF00008B9F1670F40
:10AB000014BF4FF045094FF0650904E0B9F1410F5A
:10AB100008BF4FF05009A969E86817F8013B0B54CA
:10AB20004A1CB8F1010F05DA95F83810090758BF2B
:10AB3000AA6117D52E211154531CB8F1010FAB6136
:10AB400010DB761E36B2B045B8BF464636B2324646
:10AB500039461818F7F7BAFCA8693018A861A8EBAD
:10AB600006006862E868A9690F18200007F8019BD1
:10AB700003D42B2007F8010B03E02D2107F8011B5C
:10AB8000644200260DF1080808E00A2200A805F03A
:10AB9000BDFF019808F8010B761C009C21B2012929
:10ABA000F3DA022E06DA49F02000652804BF3020CF
:10ABB00007F8010B4EB9302007F8010B07E0761EAD
:10ABC00002A8305C303007F8010B012EF7DAE86894
:10ABD000A9690818381AE86195F8380000F01400DF
:10ABE00010280DD16869A9690818696A0818E96907
:10ABF0000818A96A0818696B8842BCBF081A28623D
:10AC000005B0BDE8F083F8B504460D4616461F466C
:10AC1000002004E0E86A401CE8627F1E002047B183
:10AC200016F8011BA868A047A8600028F2D14FF0D1
:10AC3000FF30F2BD686A6C747A4C00006E616E0081
:10AC40004E414E00696E6600494E460030000000DD
:10AC500010B5EFF3108072B60A4C216841F47F0101
:10AC6000216080F31088A06E10F4700F04BFA7203D
:10AC700005F054FF4FF00070C4F81C020020C4F827
:10AC8000140210BD20ED00E0B5EEC00AF1EE10FA9E
:10AC900002D4B1EEC00A70476FF0004C00EE10CA4B
:10ACA00005F050BF10EE101A04204FF07E5C01EE4C
:10ACB00090CA49004FEA510100EE101A88BF0820DF
:10ACC000B1F17E5F13D871EEC00ADFF838C031EE03
:10ACD000801A61EE200AF1EEE00A614586BF80F03D
:10ACE000040080EE800A80EE200A05F031BF4900A2
:10ACF00011F1807F9CBF6FF0004100EE101A45F209
:10AD000021877047F404353FF0B540F2FF7581EAC2
:10AD1000030C0CF0004C15EA11541DBF15EA135733
:10AD2000AC42AF42E5E0BC41C1F31301C3F31303EE
:10AD3000801A994143F4801304D2641E40004941B3
:10AD400080185941C90241EA5051B1FBF3F603FBA7
:10AD50001611A2FB0675D7EBC020A94102D2761EC0
:10AD600080185941C90241EA5051B1FBF3FE03FB7F
:10AD70001E11A2FB0E75D7EBC020A94103D2AEF184
:10AD8000010E80185941890241EA9051760546EA40
:10AD90008E2EB1FBF3F603FB1611A2FB0675D7EB63
:10ADA0008020A94102D2761E80185941C90241EA89
:10ADB00050514EEA060EB1FBF3F603FB1611A2FB4F
:10ADC0000675D7EBC020A94102D2761E80185941E2
:10ADD000C90241EA5051B1FBF3F703FB1711A2FB83
:10ADE0000735D3EBC020A94167F100070CBF004233
:10ADF00047F0010766F3D5274FEA1E31B80814F56E
:10AE0000806412DDBD0775F1004250EB0E5051EB2E
:10AE1000045111F5801F5CBF41EA0C01F0BD4CF0FC
:10AE20007F6141F0E0410020F0BDBD076D0840EAC0
:10AE30000E5041F48011D4F10104B4F120060ADA75
:10AE4000C4F120060200E04001FA06F3E140184395
:10AE5000B24015430EE0342C13DCC6F1200445EA61
:10AE600040056D0820FA06F2154321FA06F0A140CC
:10AE70000D43002175F1004250F1000051EB0C012F
:10AE8000F0BD00205FEA0C01F0BDCFB992185B4124
:10AE9000B3FA83F704BFB2FA82F6BF190B3FB7F1DA
:10AEA00020062FBF02FA06F3BB40C7F1200622FAA4
:10AEB00006F638BF3343BA401CB1E419641E33E7C9
:10AEC0007F4231F00041B1FA81F404BFB0FA80F65C
:10AED000A4190B3CB4F120062FBF00FA06F1A140E3
:10AEE000C4F1200620FA06F638BF3143A0403C1BCF
:10AEF0001AE7AC421ABF05EA1357AF4212E050EA14
:10AF000041061CBF52EA4306BFE750EA41073046FC
:10AF100061461CBF41EA0551F0BD52EA430C08BF2F
:10AF2000C143F0BD00204FF4001616EB410F98BF4F
:10AF300016EB430F08BF16EB410F24BFC14305E0DA
:10AF400016EB430F0CBF61464CEA0551F0BD000003
:10AF500070B504463748384E0568B5B1287A88B1CF
:10AF60006868A0420ED1012028723078401C3070F1
:10AF7000287A401E2872C0B210B9284605F03AFE61
:10AF8000FBF772FCED68002DE8D170BD2B492C4A0F
:10AF90000A60002100220B468C46A0E80E101038F3
:10AFA000802181F3118800BF00BF22490A68C26076
:10AFB00008602148407808B980F31188704730B59F
:10AFC0001D4D04462878401C287081B0A868217A5D
:10AFD00039B9606001252572FBF746FC284601B0AF
:10AFE00030BD6168814208D01021204605F018FE6E
:10AFF000207A0028F8D1A8686060207A451C257264
:10B00000FBF732FC284601B030BD0B490A78521CD0
:10B010000A70017A491E0172C9B2002918BFFBF7F4
:10B0200023BC00B581B005F0E5FD01B05DF804EB8F
:10B03000FBF71ABC68DA0300705E030040DA030015
:10B0400051BF000000F5E0700268914203D34368ED
:10B050009A18914202D380680028F5D17047DFF832
:10B060006007016891B94FF4803181604FF48051DD
:10B0700041604FF0FF31C16001610421DFF84427D6
:10B080004161C2F8BC11DFF8401701600120704730
:10B0900001F1080313F0070305D001F10803C3F120
:10B0A000080303F007035918D21A8161C26042F005
:10B0B00001034B60511828234B60DFF8041709691E
:10B0C000C16170472DE9F04F064601F1080010F00C
:10B0D000070083B008BF884607D001F10800C0F11F
:10B0E000080000F0070000EB010802F1080010F072
:10B0F000070006D002F10800C0F1080000F00700C8
:10B1000082181546A5EB0800A0EB030943F00300E5
:10B1100003EB080BC8F80400AB4528BF05F09EFD03
:10B120002879C00758BF05F099FDB9F1100F38BF55
:10B1300005F094FDB069854209D1F0684844F0609B
:10B14000C6F818B040F00100CBF804006DE170695A
:10B1500085420BD1B0684844B060C6F814B040F0E6
:10B160000101CBF8041040F80B005EE1686800F0C4
:10B170000301012940F0AD80C008C0000190C00863
:10B1800020283AD2D5F808A0EF680090BD4208BF49
:10B1900005F064FD554508BF05F060FD686800993D
:10B1A000C008C000B0EBC10F18BF05F057FD0098F4
:10B1B00006EBC00000F128018A4507D031698A45B5
:10B1C000C0F08280DAF80C10A9427DD1574506D133
:10B1D000009A3068012191408843306076E0283041
:10B1E000874205D0306987426ED3B868A8426BD1D8
:10B1F000CAF80C70C7F808A068E0EF68D5F818A086
:10B20000AF420CD0A8683169884223D3C168A942F3
:10B2100004BFB968A9421DD1C760B8601CE005F140
:10B220001400076837B905F110000768A7B101E0FD
:10B230000846076807F114010A68002A02BF07F1EF
:10B2400010010A68002AF3D13169884202D3002133
:10B25000016001E005F002FDBAF1000F36D0E869A7
:10B2600006EB800000F5987001688D4208D10760F8
:10B27000A7B9EA697068012191408843706025E0B0
:10B280003069824508D3DAF81000A84214BFCAF822
:10B290001470CAF8107001E005F0E0FCB7B1306935
:10B2A000874211D3C7F818A0296929B1814226BF66
:10B2B00039618F6105F0D2FC686938B13169884223
:10B2C00002D37861876101E005F0C8FC0198451957
:10B2D000814468684008400068604FEAD90549F039
:10B2E0000100CBF8040049F80B90202D23D206EB87
:10B2F000C50000F12807B9F1100F38BF05F0AEFC0A
:10B30000306820FA05F1C907BA4604D40121A940E2
:10B310000843306006E0B868316988422CBF824635
:10B3200005F09CFCC7F808B0CAF80CB0CBF808A030
:10B33000CBF80C7079E05FEA192108BF002023D018
:10B34000B1F5803F28BF1F201ED2A1F58070000CF0
:10B3500000F008008140A1F58052120C02F00402B6
:10B360009140A1F580431B0CC0F10E0003F00203D5
:10B37000801AC01A994000EBD130C11D29FA01F2A0
:10B3800002F0010101EB4000CBF81C000022CBF8D9
:10B390001420CBF8102006EB8001726822FA00F32B
:10B3A000DB0701F5987107D4012303FA00F010437D
:10B3B0007060C1F800B01DE01F2809680EBF0020B2
:10B3C0004008C0F1190009FA00F000E011464A688F
:10B3D000D208D2004A4514D0C20F01EB820202F11A
:10B3E000100340001A68002AF0D1306983421AD352
:10B3F000C3F800B0CBF81810CBF80CB0CBF808B0FD
:10B4000013E032698868914228BF90420BD3C0F89C
:10B410000CB0C1F808B0CBF80800CBF80C10002035
:10B42000CBF8180001E005F019FC08F1080000F065
:10B4300005BE2DE9FA4D0546DFF88403006884B0A7
:10B4400008B9FFF70CFEDFF878030499806841180B
:10B450002F31401E21EA00000499814280F0AB8127
:10B4600005F5D876B16841B1D5F8B021801882428F
:10B4700080F0A1818142C0F09E8105F0F3FB00289D
:10B480001EBF0446D0F8008014F1010F00F0938134
:10B49000D5F8B0014044C5F8B0017168814238BFA9
:10B4A00001467160A86980BB286908B1844200D256
:10B4B0002C613461C6F814800020F06105F1280188
:10B4C000BF48006868624FF0FF3028620020C96002
:10B4D000896001F10802801C1031D260202892603E
:10B4E000F5D3B848854203D1A8F12802214629E0C6
:10B4F00055F8040CC00805EBC000A0F1080108EBEA
:10B500000400401AA0F128021CE005F5E07108468D
:10B5100000E08068D0B1026843689A189442F8D17C
:10B52000027B120712D4AA6903689A420ED34768B5
:10B530003B449A420AD208EB07014160E868A969D6
:10B5400008EB00022846FFF7A3FD1EE128698442AC
:10B55000084638BF2C6108EB040100E0806880B128
:10B5600002688A42FAD1017B09070AD40460416863
:10B57000414441602146049B284606B0BDE8F04D99
:10B58000A0E5AF6939462846FFF75CFD01684068D1
:10B59000401802902F3800F1080111F0070105D082
:10B5A00000F10801C1F1080101F00701081807F1D5
:10B5B0001001884234BF0097009000980830019035
:10B5C00004F10801009800F1180A11F007014FF08A
:10B5D000000BA8F1280005D004F10801C1F1080111
:10B5E00001F007010A19401AAA61E86040F0010160
:10B5F000516080182821416071480069E861019814
:10B6000010F0070018BF05F029FB00991B204860C7
:10B6100005F5E071B1E80C500198A0E80C503461D8
:10B62000C6F81480C6F81CB00198B061029800E01A
:10B630008A460722CAF804200AF104010A1D824240
:10B640000BF1010BF4D3BBF1020FB8BF05F006FB01
:10B650000098B84200F09980C01BC119C4084A681C
:10B66000520852004A6040F001017960C051202C1C
:10B6700020D205EBC40101F12806102838BF05F0DF
:10B68000EDFA286820FA04F1C907B04604D4012174
:10B69000A1400843286006E0B068296988422CBFB1
:10B6A000804605F0DBFAB760C8F80C70C7F8088070
:10B6B000FE606AE0010A08BF002223D0B1F5803F96
:10B6C00028BF1F221ED2A1F58072120C02F00802C0
:10B6D0009140A1F580531B0C03F004039940A1F5A0
:10B6E0008044240CC2F10E0204F00204D21A121B90
:10B6F000A14002EBD131CA1D20FA02F303F001028E
:10B7000002EB4102FA6100237B613B6105EB8201A0
:10B710006B6823FA02F4E40701F5987105D401205F
:10B720009040184368600F601CE01F2A09680EBF34
:10B7300000225208C2F1190200FA02F200E0194692
:10B740004B68DB08DB00834210D0D30F01EB83038F
:10B7500003F1100452002368002BF0D128698442C1
:10B7600011D32760B961FF60BF600EE02A69886865
:10B77000914228BF904206D3C7608F60B860F960DD
:10B780000020B86101E005F069FAE8680499814297
:10B7900011D2401AE860A969049A5218AA6140F0CF
:10B7A00001005060049840F00300486006B001F1C9
:10B7B0000800BDE8F08D002006B0BDE8F08D000067
:10B7C00010D9030068BB03006859883C2DE9F04D8F
:10B7D0000446884600265FEA1820C8F1000B08BF1F
:10B7E000002123D0B0F5803F28BF1F211ED2A0F535
:10B7F0008071090C01F008018840A0F58052120CFC
:10B8000002F004029040A0F580431B0CC1F10E0130
:10B8100003F00203891AC91A984001EBD030C11D08
:10B8200028FA01F202F0010101EB400104EB810072
:10B83000D0F8300128B31F290EBF00224A08C2F1F8
:10B84000190208FA02F2002300E052004768FF08DC
:10B85000FF00A7EB08075F4503D25FEA070B064628
:10B860000BD04769D50F00EB8500002F00691CBF86
:10B8700087423B460028E8D1184600283CD1002EDC
:10B880003CD10120884040004142084361680840A3
:10B8900000F0678141420840411E080B00F0100093
:10B8A00021FA00F2510901F0080122FA01F39A0885
:10B8B00002F00407FB405A0802F00205081823FAB8
:10B8C00005F23844C2F340032818181822FA03F18D
:10B8D000081804EB8000D0F830010DE008464168FC
:10B8E000C908C900A1EB080159453CBF8B46064673
:10B8F00001690029F2D140690028F0D1002E00F042
:10B900003081A068A0EB0800834580F02A8120697F
:10B910008642C0F024817068C008C00008EB0B01AB
:10B92000884208EB060518BF05F098F9AE4280F092
:10B930001681F768D6F818A0B7420CD0B068216914
:10B94000884223D3C168B14204BFB968B1421DD156
:10B95000C760B8601CE006F11400076837B906F14B
:10B9600010000768A7B101E00846076807F1140155
:10B970000A68002A02BF07F110010A68002AF3D101
:10B980002169884202D30021016001E005F066F9D7
:10B99000BAF1000F38D0F06904EB800000F5987020
:10B9A00001688E4209D10760380014D1F2696068DD
:10B9B000012191408843606026E02069824508D3D8
:10B9C000DAF81000B04214BFCAF81470CAF8107048
:10B9D00001E005F043F9BFB12069874212D3C7F8EF
:10B9E00018A0306930B12169884226BF386187616B
:10B9F00005F034F9706938B12169884202D3786161
:10BA0000876101E005F02AF9BBF1100F0CD208EBB9
:10BA10000B0040F00300706008EB0B0080194168D8
:10BA200041F00101416096E048F0030070604BF086
:10BA3000010068604FEADB004BF805B020281DD2FA
:10BA400004EBC00101F12807216821FA00F2D207B6
:10BA5000BB4605D4012202FA00F00843206006E04C
:10BA6000B868216988422CBF834605F0F7F8BD60AD
:10BA7000CBF80C50C5F808B0EF606CE05FEA1B2112
:10BA800008BF002023D0B1F5803F28BF1F201ED261
:10BA9000A1F58070000C00F008008140A1F58052F3
:10BAA000120C02F004029140A1F580431B0CC0F17E
:10BAB0000E0003F00203801AC01A994000EBD13047
:10BAC000C11D2BFA01F202F0010101EB4000E86117
:10BAD00000226A612A6104EB8001626822FA00F3A5
:10BAE000DB0701F5987106D4012303FA00F0104337
:10BAF00060600D601CE01F2809680EBF0020400830
:10BB0000C0F119000BFA00F000E011464A68D208B3
:10BB1000D2005A4510D0C20F01EB820202F110038D
:10BB200040001A68002AF0D12069834211D31D60B9
:10BB3000A961ED60AD600EE022698868914228BF7E
:10BB4000904206D3C5608D60A860E9600020A861BE
:10BB500001E005F083F806F10800BDE8F08D05F07E
:10BB60007DF80020BDE8F08D2DE9F84F04468846A9
:10BB7000606841420840411E080B00F0100021FAA5
:10BB800000F2510901F0080122FA01F39A0802F0CB
:10BB9000040223FA02F56B0803F00203081825FAE1
:10BBA00003F61018C6F340051818284426FA05F1C4
:10BBB000081804EB8000D0F830014168C908C900BA
:10BBC0000646A1EB080A09E008464168C908C90011
:10BBD000A1EB080151453CBF8A4606460169002990
:10BBE000F2D140690028F0D120698642C0F0C480BB
:10BBF0007068C00808EB0A09C000484508EB060B4E
:10BC000018BF05F02BF85E4580F0B680F768B5697F
:10BC1000B7420CD0B0682169884223D3C168B142D1
:10BC200004BFB968B1421DD1C760B8601CE006F11D
:10BC30001400076837B906F110000768A7B101E0E2
:10BC40000846076807F114010A68002A02BF07F1D5
:10BC500010010A68002AF3D12169884202D3002129
:10BC6000016001E004F0FAFF002D34D0F06904EB2C
:10BC7000800000F5987001688E4209D10760380095
:10BC800011D1F2696068012191408843606022E02F
:10BC90002069854205D32869B04214BF6F612F61C6
:10BCA00001E004F0DBFFB7B12069874211D3BD6129
:10BCB000306930B12169884226BF3861876104F05C
:10BCC000CDFF706938B12169884202D378618761FC
:10BCD00001E004F0C3FFBAF1100F09D249F00300EC
:10BCE000706009EB0600416841F0010141603FE0EE
:10BCF00048F0030070604AF00100CBF804004AF8F5
:10BD00000BA0D4F808804FEAD805202D28BF04F0F6
:10BD1000A5FFB8F1000F27D0D4F81490009504EBDC
:10BD2000C50000F12805B8F1100F38BF04F096FFE8
:10BD30002068009920FA01F2D1072F4605D4009A15
:10BD4000012191400843206006E0A86821698842EB
:10BD50002CBF074604F082FFC5F80890C7F80C9086
:10BD6000C9F80870C9F80C50C4F808A0C4F814B099
:10BD700006F10800BDE8F28F04F070FF0020BDE876
:10BD8000F28F2DE9F04F83B00546C046C046F52D31
:10BD9000DFF8C04780F007810B2D31BF102705F178
:10BDA0000B00C008C7002168FE0821FA06F010F059
:10BDB000030F42D0C04300F00100861904EBC60017
:10BDC00000F12808F700D8F808506868C008C000DB
:10BDD000B84218BF04F042FFD5F80890454508BFA7
:10BDE00004F03CFF4D4508BF04F038FF6868C00808
:10BDF000C000B84218BF04F031FFC84505D1206823
:10BE00000121B140884320600DE02069814508D3BD
:10BE1000D9F80C00A84204D1C8F80890C9F80C80E1
:10BE200001E004F01BFF47F0030068607819083553
:10BE3000416841F001014160FDE0A168B94280F034
:10BE4000C480002800F0A680012505FA06F149000B
:10BE50004A42B0401143084041420840411E080B8D
:10BE600000F0100021FA00F2510901F0080322FA53
:10BE700003F18A0802F0040221FA02F6710801F0C7
:10BE80000208181826FA08F11018C1F340064044B9
:10BE9000301821FA06F202EB000804EBC80000F1AA
:10BEA00028094FEAC80AD9F808607068C008C000BD
:10BEB000504518BF04F0D2FED6F808B04E4508BF72
:10BEC00004F0CCFE5E4508BF04F0C8FE7068C008F0
:10BED000C000504518BF04F0C1FED94505D1206807
:10BEE00005FA08F1884320600DE02069834508D3F6
:10BEF000DBF80C00B04204D1C9F808B0CBF80C90C4
:10BF000001E004F0ABFE47F003007060AAEB070805
:10BF1000B819019048F0010001994860019848F86B
:10BF20000080A7684FEAD70ABAF1200F28BF04F0B3
:10BF300095FE47B3CDF800A004EBCA00D4F81490E6
:10BF400000F1280A102F38BF04F088FE20680099FD
:10BF500020FA01F2D107D34605D4009905FA01F180
:10BF60000843206007E0DAF80800216988422CBF06
:10BF7000834604F073FECAF80890CBF80C90C9F819
:10BF800008B0C9F80CA0C4F8088006F108050198AB
:10BF9000606150E06068C0B339462046FFF7E4FDB9
:10BFA000050012D047E015F1400F28BF4FF0FF37D2
:10BFB0000BD205F10B00C008C700606828B13946F4
:10BFC0002046FFF703FC050035D1A068B8421CD31A
:10BFD000C11B626910290AD3B8186061A16041F0E1
:10BFE00001034360095047F0030050600AE000215C
:10BFF000A160616140F0030151608018416841F027
:10C000000101416002F1080515E0E06887420DD2A8
:10C01000C01BA169E0607A18A26140F00100506085
:10C0200001F1080547F00300486004E03946204666
:10C03000FFF7FFF90546C046C046284603B0BDE8F5
:10C04000F08F00B970472DE9F047A0F10804C04611
:10C05000C046DFF8005528698442C0F074826168E8
:10C0600001F00302012A00F06E82CA084FEAC208FA
:10C07000CA0708EB040936D4226811F0030F00F058
:10C080006482A41A84429044C0F05D8269698C4243
:10C0900000F0D880D608202E70D2D4F80CA0A76863
:10C0A000544508BF04F0DAFDBC4208BF04F0D6FDD9
:10C0B0006068C008C000B0EBC60F18BF04F0CEFD2A
:10C0C00005EBC60000F128018F4205D029698F4297
:10C0D00051D3F968A1424ED1BA453DD1286801211A
:10C0E000B140884328604C4580F02D82D9F8040087
:10C0F000C10740F12882810700F17A81A969894549
:10C1000040F0B580E868AC614044E86040F001016F
:10C11000616069698C4202D100216961A960E969A5
:10C12000814280F01282DFF83004006808B9FEF71F
:10C1300096FFA969002900F00882E868292824BF31
:10C140002846FEF77FFFE869E968884280F0FD81B4
:10C150004FF0FF30E861F8E12830824506D02869C9
:10C16000824508D3DAF80800A04204D1C7F80CA031
:10C17000CAF80870B7E704F071FDB4E7E768A6698C
:10C18000A7420BD0A168814222D3C868A04204BF55
:10C19000B868A0421CD1CF60B9601BE004F1140163
:10C1A0000F6837B904F110010F689FB101E0114623
:10C1B0000F6807F114021368002B02BF07F1100289
:10C1C0001368002BF3D1814202D30020086001E004
:10C1D00004F044FD002E86D0E06905EB800000F5F8
:10C1E000987001688C4209D10760380011D1E2696A
:10C1F0006868012191408843686074E72869864235
:10C2000005D33069A04214BF7761376101E004F0C3
:10C2100025FD002F3FF467AF28698742ABD3BE618D
:10C22000216929B1814226BF39618F6104F016FD71
:10C23000606900283FF457AF296988429BD3786131
:10C24000876150E799F8040000F0030003287FF4A9
:10C250004AAFC5F80880D9F8040040084000C9F882
:10C26000040048F00100606048F804806DE16969ED
:10C27000894508D1A8686C614044A86040F001017C
:10C280006160005161E1C008C0004FEAD00ABAF114
:10C29000200F804436D2D9F80C70D9F80860B9451F
:10C2A00008BF04F0DBFCB14508BF04F0D7FCD9F8A7
:10C2B0000400C008C000B0EBCA0F18BF04F0CEFCE9
:10C2C00005EBCA0000F128018E4206D029698E4292
:10C2D000C0F08180F16849457DD1B74206D1286818
:10C2E000012101FA0AF18843286076E0283087426C
:10C2F00005D0286987426ED3B86848456BD1F7608E
:10C30000BE606AE0D9F80C70D9F818604F450DD0BE
:10C31000D9F808002969884223D3C168494504BF78
:10C32000B96849451DD1C760B8601CE009F1140027
:10C33000076837B909F110000768A7B101E008469E
:10C34000076807F114010A68002A02BF07F110010B
:10C350000A68002AF3D12969884202D300210160CA
:10C3600001E004F07BFC002E37D0D9F81C0005EB6F
:10C37000800000F59870016889450AD1076038008F
:10C3800012D1D9F81C206868012191408843686067
:10C3900023E02869864205D33069484514BF776198
:10C3A000376101E004F05AFCBFB12869874212D31B
:10C3B000BE61D9F8101029B1814226BF39618F6161
:10C3C00004F04CFCD9F8140038B12969884202D332
:10C3D0007861876101E004F041FC48F00100606091
:10C3E00048F80480686984420BD1C5F80880ACE045
:10C3F00040084000C9F8040048F00100606048F8B7
:10C4000004804FEAD807202F22D205EBC70000F1A5
:10C410002809B8F1100F38BF04F020FC286820FA72
:10C4200007F1C9074E4604D40121B94008432860EA
:10C4300007E0D9F80800296988422CBF064604F0B5
:10C440000DFCC9F80840F460A660C4F80C907CE0CC
:10C450005FEA182008BF002123D0B0F5803F28BF35
:10C460001F211ED2A0F58071090C01F0080188403F
:10C47000A0F58052120C02F004029040A0F5804317
:10C480001B0CC1F10E0103F00203891AC91A98406E
:10C4900001EBD030C11D28FA01F202F0010101EBDD
:10C4A0004001E16100226261226105EB81006A685E
:10C4B00022FA01F3DB0700F5987006D4012303FA92
:10C4C00001F11143696004601CE01F2900680EBF80
:10C4D00000214908C1F1190108FA01F100E01046F4
:10C4E0004268D208D200424510D0CA0F00EB820247
:10C4F00002F1100349001A68002AF0D129698B4221
:10C5000011D31C60A061E460A4600EE02A69816818
:10C51000904228BF914206D3CC608460A160E06065
:10C520000020A06101E004F099FB286A401E286207
:10C530000BD1D5F8C80100E080680028FCD14FF08D
:10C54000FF30286201E004F089FBC046C046BDE828
:10C55000F087000068BB030010D90300802282F33B
:10C56000118800BF00BFC1600248407808B980F35D
:10C5700011887047705E030000B581B0802282F39D
:10C58000118800BF00BF8368094A33B9507808B9E1
:10C5900080F31188012001B000BD13785B1C13707B
:10C5A00004F099FBFAF760F9002001B000BD00BF6C
:10C5B000705E030010B50F4C2178491C217080215A
:10C5C00081F3118800BF00BFA1688A69024205D1CA
:10C5D000C861082008742046FBF7FBFEA168886943
:10C5E00000228A612178491E2170617809B981F39E
:10C5F000118810BD705E030070B40024002526462B
:10C6000070C070C018384360C260818270BC7047CF
:10C610002DE9F0470E46089F099DDDF82890044655
:10C62000924698463421F5F799FF1049C4F814A0B2
:10C63000207C09780843207484F8299006B166624A
:10C64000E819C008C000002140F8501D4FF080716B
:10C65000416407490164C0F84C806FF002014162F7
:10C6600060602046BDE8F047FAF756B981DA03006A
:10C670009F93000030B50D4D2A78521C2A7081B06E
:10C680000124802282F3118800BF00BF8268C36842
:10C690009A4202D204F0FCFA0024687808B980F3C8
:10C6A0001188FAF7E1F8204601B030BD705E030052
:10C6B00000B581B0802282F3118800BF00BF8A6973
:10C6C000104388610A7C02F0F802082A05D1CA6981
:10C6D00002421CBF0846FAF7E3F80348407808B95D
:10C6E00080F3118801B000BD705E0300DFF8D01246
:10C6F0000A68002803D042F0010008607047500823
:10C70000400008607047DFF8B8024FF0FF31416029
:10C71000092101604FF4807101600020E6E7F0B468
:10C72000DFF8A4120A6E086810F00103DFF8940223
:10C730000CD00A6ED0E902454FF0144647F2357727
:10C74000A4197D41C0E9024501230B60DFF87C128A
:10C75000A1FB0223D20B42EA4342D0E9024512195F
:10C7600055EBD333D0E90045101943EB0501F0BC7C
:10C770007047F8B505460E461746DFF84442206874
:10C78000400403D50FF24820FCF7D6FB6FF00040C1
:10C79000854201D30F20EEE0B5F1804F0CD30E207F
:10C7A00079004FF47A72B1FBF2F101EB4601B1FB73
:10C7B000F2F101EB4505DEE0B5F1005F0CD30D2091
:10C7C000B9004FF47A72B1FBF2F101EB8601B1FBD3
:10C7D000F2F101EB8505CEE0B5F1805F0CD30C20C2
:10C7E000F9004FF47A72B1FBF2F101EBC601B1FB33
:10C7F000F2F101EBC505BEE0B5F1006F0CD30B20E3
:10C8000039014FF47A72B1FBF2F101EB0611B1FB81
:10C81000F2F101EB0515AEE0B5F1806F0CD30A2003
:10C8200079014FF47A72B1FBF2F101EB4611B1FBE1
:10C83000F2F101EB45159EE0B5F1007F0CD3092024
:10C84000B9014FF47A72B1FBF2F101EB8611B1FB41
:10C85000F2F101EB85158EE0B5F1807F0CD3082055
:10C86000F9014FF47A72B1FBF2F101EBC611B1FBA1
:10C87000F2F101EBC5157EE0B5F5000F0CD30720F2
:10C8800039024FF47A72B1FBF2F101EB0621B1FBF0
:10C89000F2F101EB05256EE0B5F5800F0CD3062013
:10C8A00079024FF47A72B1FBF2F101EB4621B1FB50
:10C8B000F2F101EB45255EE0B5F5001F0CD3052034
:10C8C000B9024FF47A72B1FBF2F101EB8621B1FBB0
:10C8D000F2F101EB85254EE0B5F5801F0CD3042065
:10C8E000F9024FF47A72B1FBF2F101EBC621B1FB10
:10C8F000F2F101EBC5253EE0B5F5002F0FD3032083
:10C9000040F6FE7101FB07F24FF47A73B2FBF3F2CB
:10C9100001FB0622B2FBF3F201FB05252BE0B5F586
:10C92000802F0CD3022079034FF47A72B1FBF2F11D
:10C9300001EB4631B1FBF2F101EB45351BE0B5F5FA
:10C94000003F0CD30120B9034FF47A72B1FBF2F12E
:10C9500001EB8631B1FBF2F101EB85350BE00020F4
:10C96000F9034FF47A72B1FBF2F101EBC631B1FB7E
:10C97000F2F101EBC535A560216821F4705141EA5F
:10C9800080202060F1BD0E490A68002803D042F4DF
:10C9900080400860704722F48040086070470A4970
:10C9A0000A6802F00402104308607047002006493C
:10C9B0000A6812F004020A6000D0012070470000EB
:10C9C00040004240B8D903003000424000CA9A3BC0
:10C9D0005B495D525443205469636B206973207234
:10C9E000756E6E696E67200A00000000F0B492B2A6
:10C9F00013460246B1FBF3F403FB1410110C01EBD8
:10CA00000041B1FBF3F0254600240646274647EADD
:10CA1000164714EB06447D4103FB1010000410FA86
:10CA200082F0B0FBF3F0002120186941F0BC7047A0
:10CA3000012100F01F029140874A400942F820106E
:10CA40007047012100F01F029140844A400942F8DA
:10CA50002010704710B5002403E0204600F065F96F
:10CA6000641C072CF9DB0420FFF7EBFF0420BDE872
:10CA70001040DDE718B4342212FB00F00FF2FC3254
:10CA800083185C68002C11D0805C00F00F00DA691C
:10CA90000092009A12686043714B53F8243083402F
:10CAA0009A4301FA00F010430099086011BC7047E6
:10CAB00081B0342111FB00F00FF2C03142185368ED
:10CAC000002B02D14FF0FF300DE0D2690092009AA6
:10CAD0001268405C00F00F0058431146C1406048A6
:10CAE00050F82300084001B0704718B4342212FBFC
:10CAF00000F00FF2883283189C68002C11D0805C03
:10CB000000F00F001A6A0092009A12686043544BBA
:10CB100053F8243083409A4301FA00F010430099FF
:10CB2000086011BC704781B0342111FB00F00FF296
:10CB30004C3142189368002B02D14FF0FF300FE0C8
:10CB4000405C00F00F00116A00910099096803FB36
:10CB500000F2434850F82300904001400846D0407E
:10CB600001B0704718B4342212FB00F00FF20C32FF
:10CB70008318DC68002C11D0805C00F00F005A6A2A
:10CB80000092009A12686043354B53F8243083407A
:10CB90009A4301FA00F010430099086011BC7047F5
:10CBA00018B4342212FB00F00FF2D02283181C6953
:10CBB000002C11D0805C00F00F009A6A0092009A5D
:10CBC00012686043264B53F8243083409A4301FA9D
:10CBD00000F010430099086011BC704718B434226B
:10CBE00012FB00F00FF2942283185C69002C11D024
:10CBF000805C00F00F00DA6A0092009A12686043CD
:10CC0000174B53F8243083409A4301FA00F0104345
:10CC10000099086011BC704718B4342212FB00F070
:10CC20000FF2582283189C69002C11D0805C00F010
:10CC30000F001A6B0092009A12686043084B53F879
:10CC4000243083409A4301FA00F0104300990860B1
:10CC500011BC70470000000000E100E080E200E04D
:10CC6000BC6503002DE9F8430F4615461E4600EB50
:10CC7000C0014FEA81080FF6B80908EB09040F213B
:10CC8000207CFFF7F7FE58F80900616900910099D0
:10CC9000096807228240914307FA00F0084300998F
:10CCA00008606768A069009000980068FF21B9409B
:10CCB00020EA0108012D0CD1802E0AD34FF4B07266
:10CCC0000FF218110FF20810FCF736F90020C046D9
:10CCD000C046002D12D0012D05D146F08000B8408D
:10CCE00040EA08080AE040F26B120FF2F0010FF27E
:10CCF000E000FCF721F90020C046C0460098C0F8CB
:10CD00000080206A00900120E16800FA01F1009A99
:10CD10001160E169009100990968A268904021EAD8
:10CD2000000000990860BDE8F18310B582B00FF6ED
:10CD3000000100EBC00201EB82040021207CFFF720
:10CD400099FEE0690090009800680121A26801FA4C
:10CD500002F21043009A1060206A0090E06801FA25
:10CD600000F00099086013BD0FF2C47100EBC0021F
:10CD700001EB8200007CD6E681B00FF2B47100EBCB
:10CD8000C00201EB8200C168006A00900098006850
:10CD90000246CA40D00703D50120884000990860A8
:10CDA00001B0704781B00FF2887100EBC00201EB57
:10CDB0008200016A009100990968C0680A46C24071
:10CDC000D00701D5012000E0002001B0704700002D
:10CDD0005B455D25732C2025640A0000443A5C50B5
:10CDE0006572666F7263655C53454E534F525F5375
:10CDF0004C4F434154494F4E5F494E4E4F565F3161
:10CE00003731365F38415C434F4E464944454E54B6
:10CE100049414C5C53656E736F724875625C4D415D
:10CE200053535F50524F4A4543545C50524F445CF9
:10CE30004135315C545C706C6174666F726D5C6519
:10CE400078796E6F73393631305C6669726D7761EF
:10CE500072655C6F735C706C6174666F726D5C653B
:10CE600078796E6F735C7372635C6770696F5C670F
:10CE700070696F4472762E630000000000000000AD
:10CE80000400000001000000040000000400000095
:10CE900002000000040000000000184004001840D8
:10CEA000080018400C0018401000184014001840EA
:10CEB0000100000004000000010000000400000068
:10CEC0000400000002000000040000000000184000
:10CED00004001840080018400C00184010001840CA
:10CEE00014001840020000000400000001000000CF
:10CEF0000400000004000000020000000400000024
:10CF00000000184004001840080018400C001840A9
:10CF10001000184014001840030000000400000036
:10CF200001000000040000000400000002000000F6
:10CF300004000000000018400400184008001840D9
:10CF40000C001840100018401400184000000000A9
:10CF500004000000010000000400000004000000C4
:10CF600002000000040000002000184024001840C7
:10CF7000280018402C001840300018403400184099
:10CF80000100000004000000010000000400000097
:10CF9000040000000200000004000000200018400F
:10CFA00024001840280018402C0018403000184079
:10CFB00034001840020000000400000001000000DE
:10CFC0000400000004000000020000000400000053
:10CFD0002000184024001840280018402C00184059
:10CFE0003000184034001840000000000400000029
:10CFF0000100000004000000040000000000000028
:10D00000000000000000624004006240080062402E
:10D010000C0062401C0062401C00624000000000E6
:10D0200004000000010000000400000004000000F3
:10D030000000000000000000200062402400624068
:10D04000280062402C0062403C0062403C0062408C
:10D0500000000000040000000100000004000000C7
:10D0600004000000000000000000000040006240DA
:10D0700044006240480062404C0062405C006240F4
:10D080005C0062400000000004000000010000009D
:10D090000400000004000000000000000000000088
:10D0A0006000624064006240680062406C00624060
:10D0B0007C0062407C006240000000000400000030
:10D0C0000100000004000000040000000000000057
:10D0D00000000000800062408400624088006240DE
:10D0E0008C0062409C0062409C0062400000000096
:10D0F0000400000001000000040000000400000023
:10D100000000000000000000A0006240A400624097
:10D11000A8006240AC006240BC006240BC006240BB
:10D1200000000000040000000100000004000000F6
:10D13000040000000000000000000000C000624089
:10D14000C4006240C8006240CC006240DC00624023
:10D15000DC0062400000000004000000010000004C
:10D1600004000000040000000000000000000000B7
:10D17000E0006240E4006240E8006240EC0062408F
:10D18000FC006240FC00624000000000040000005F
:10D190000100000004000000040000000000000086
:10D1A000000000000001624004016240080162408A
:10D1B0000C0162401C0162401C0162400000000042
:10D1C0000400000001000000040000000400000052
:10D1D00000000000000000002001624024016240C5
:10D1E000280162402C0162403C0162403C016240E7
:10D1F0000000000004000000010000000400000026
:10D200000400000000000000000000004001624037
:10D2100044016240480162404C0162405C0162404E
:10D220005C016240000000000400000001000000FA
:10D2300004000000040000000000000000000000E6
:10D240006001624064016240680162406C016240BA
:10D250007C0162407C01624000000000040000008C
:10D2600001000000040000000400000000000000B5
:10D270000000000080016240840162408801624039
:10D280008C0162409C0162409C01624000000000F1
:10D290000400000001000000040000000400000081
:10D2A0000000000000000000A0016240A4016240F4
:10D2B000A8016240AC016240BC016240BC01624016
:10D2C0000000000004000000010000000400000055
:10D2D000040000000000000000000000C0016240E7
:10D2E000C4016240C8016240CC016240DC0162407E
:10D2F000DC016240000000000400000001000000AA
:10D300000400000004000000000000000000000015
:10D31000E0016240E4016240E8016240EC016240E9
:10D32000FC016240FC0162400000000004000000BB
:10D3300001000000040000000400000000000000E4
:10D3400000000000000262400402624008026240E5
:10D350000C0262401C0262401C026240000000009D
:10D3600004000000010000000400000004000000B0
:10D370000000000000000000200262402402624021
:10D38000280262402C0262403C0262403C02624041
:10D390000000000004000000010000000400000084
:10D3A0000400000000000000000000004002624095
:10D3B00044026240480262404C0262405C026240A9
:10D3C0005C02624000000000040000000100000058
:10D3D0000400000004000000000000000000000045
:10D3E0006002624064026240680262406C02624015
:10D3F0007C0262407C0262400000000004000000E9
:10D400000100000004000000040000000000000013
:10D410000000000080026240840262408802624094
:10D420008C0262409C0262409C026240000000004C
:10D4300004000000010000000400000004000000DF
:10D440000000000000000000A0026240A402624050
:10D45000A8026240AC026240BC026240BC02624070
:10D4600000000000040000000100000004000000B3
:10D47000040000000000000000000000C002624044
:10D48000C4026240C8026240CC026240DC026240D8
:10D49000DC02624000000000040000000100000007
:10D4A0000400000004000000000000000000000074
:10D4B000E0026240E4026240E8026240EC02624044
:10D4C000FC026240FC026240000000000400000018
:10D4D0000100000004000000040000000000000043
:10D4E0000000000000036240040362400803624041
:10D4F0000C0362401C0362401C03624000000000F9
:10D50000040000000100000004000000040000000E
:10D51000000000000000000020036240240362407D
:10D52000280362402C0362403C0362403C0362409B
:10D5300000000000000000000000000000000000EB
:10D5400000000000000718400008184000091840BB
:10D55000000A18400400000008000000010000005C
:10D5600001000000010000000007184000081840FA
:10D5700000091840000A18400800000010000000D0
:10D580000200000002000000020000000007184036
:10D590000008184000091840000A18400C0000005C
:10D5A000180000000300000003000000030000005A
:10D5B000000718400008184000091840000A1840E9
:10D5C000000000000000000000000000000000005B
:10D5D000040000000407184004081840040918401B
:10D5E000040A1840040000000800000001000000C8
:10D5F000010000000500000004071840040818405E
:10D6000004091840040A1840080000001000000037
:10D61000020000000200000006000000040718409D
:10D620000408184004091840040A184000000000CB
:10D6300000000000000000000000000007000000E3
:10D64000000762400008624000096240000A624030
:10D6500000000000000000000000000000000000CA
:10D6600008000000040762400408624004096240A8
:10D67000040A6240000000000000000000000000FA
:10D68000000000000900000008076240080862402E
:10D6900008096240080A6240000000000000000023
:10D6A00000000000000000000A0000000C076240BB
:10D6B0000C0862400C0962400C0A62400000000045
:10D6C0000000000000000000000000000B0000004F
:10D6D000100762401008624010096240100A624060
:10D6E000000000000000000000000000000000003A
:10D6F0000C000000140762401408624014096240E4
:10D70000140A624000000000000000000000000059
:10D71000000000000D000000180762401808624079
:10D7200018096240180A6240000000000000000072
:10D7300000000000000000000E0000001C07624016
:10D740001C0862401C0962401C0A62400000000084
:10D750000000000000000000000000000F000000BA
:10D76000200762402008624020096240200A62408F
:10D7700000000000000000000000000000000000A9
:10D78000100000002407624024086240240962401F
:10D79000240A6240000000000000000000000000B9
:10D7A00000000000110000002807624028086240C5
:10D7B00028096240280A62400000000000000000C2
:10D7C0000000000000000000120000002C07624072
:10D7D0002C0862402C0962402C0A624000000000C4
:10D7E0000000000000000000000000001300000026
:10D7F000300762403008624030096240300A6240BF
:10D800000000000000000000000000000000000018
:10D81000140000003407624034086240340962405A
:10D82000340A624000000000000000000000000018
:10D830000000000015000000380762403808624010
:10D8400038096240380A6240000000000000000011
:10D850000000000000000000160000003C076240CD
:10D860003C0862403C0962403C0A62400000000003
:10D870000000000000000000000000001700000091
:10D88000400762404008624040096240400A6240EE
:10D890000000000000000000000000000000000088
:10D8A0001800000044076240440862404409624096
:10D8B000440A624000000000000000000000000078
:10D8C000000000001900000048076240480862405C
:10D8D00048096240480A6240000000000000000061
:10D8E00000000000000000001A0000004C07624029
:10D8F0004C0862404C0962404C0A62400000000043
:10D900000000000000000000000000001B000000FC
:10D91000500762405008624050096240500A62401D
:10D9200000000000000000000000000000000000F7
:10D930001C000000540762405408624054096240D1
:10D94000540A6240000000000000000000000000D7
:10D95000000000001D0000005807624058086240A7
:10D9600058096240580A62400000000000000000B0
:10D9700000000000000000001E0000005C07624084
:10D980005C0862405C0962405C0A62400000000082
:10D990000000000000000000000000001F00000068
:10D9A000600762406008624060096240600A62404D
:10D9B0000000000000000000000000000000000067
:10D9C000200000006407624064086240640962400D
:10D9D000640A624010B582B00446032001F05EF88C
:10D9E0000549B0FBF1F0604300900098411E0091A2
:10D9F0000028FAD113BD0000404B4C0010B582B096
:10DA00000446032001F04AF841F28831B0FBF1F0FE
:10DA1000604300900098411E00910028FAD113BD88
:10DA200070470000012100F01F0291404E4A40095A
:10DA300042F820107047012100F01F0291404B4A2C
:10DA4000400942F820107047F8B500EB4004A500EB
:10DA5000474E069CAF197C600127AF510094FFF739
:10DA600001F9F1BDF8B500260420FFF7E4FF3446C4
:10DA70000AE02A460FF2FC010FF22010FBF75CFAD5
:10DA80002046FFF779F9641CE4B22546072D21DA18
:10DA90002046FFF787F90028F5D0012605EB450061
:10DAA000800033494258002AE3D04718786800289C
:10DAB00005D02046FFF758F979688847E3E72A46FA
:10DAC0000FF2B0010FF2BC00FBF736FA2046FFF769
:10DAD00053F9D8E7002E05D10FF298010FF2E000BC
:10DAE000FBF72AFA0420BDE8F2409BE770B5044634
:10DAF0001320FFF7A0FF25462046FFF753F9002823
:10DB000026D005EB4500800019494258002A14D060
:10DB100046187068002805D02046FFF725F971687F
:10DB200088471CE02A460FF2B0010FF25800FBF7BD
:10DB300003FA2046FFF720F911E02A460FF2980178
:10DB40000FF25800FBF7F8F92046FFF715F906E049
:10DB50002A460FF284010FF29400FBF7EDF913202F
:10DB6000BDE870405EE7000000E100E080E100E019
:10DB700018C403006770696F5F49525148616E6451
:10DB80006C6572005B455D25732C206362206E75A9
:10DB90006C6C20282564290A000000005B455D2587
:10DBA000732C20696E74207365656D7320737570B6
:10DBB0007572696F757320282564290A00000000BA
:10DBC0005B455D25732C206E6F2070656E64696EF9
:10DBD0006720696E740A00006770696F436D677033
:10DBE00049525148616E646C657200005B455D2569
:10DBF000732C20696E74206973206E6F74207065B9
:10DC00006E64696E6720282564290A00DFF84019D0
:10DC100008607047DFF8381951F830007047DFF8B6
:10DC2000301901EBC0004068704780B50120FFF754
:10DC3000F1FF406C02BD10B504460120FFF7EAFF7A
:10DC4000A0F84A4010BD2DE9F04F93B00020FFF737
:10DC5000E1FF074607F580760FF674140FF63415CA
:10DC60000B223146284603F063F800280BD00196BA
:10DC7000009533460FF6081221460FF62410FBF7E5
:10DC80005BF90020F7E03069DFF8C838984209D026
:10DC900000900FF6EC0221460FF64010FBF74CF90E
:10DCA0000020E8E0DFF8A858AE60F069C0192861EC
:10DCB000706BC0192865706AC019A861F16AC9192A
:10DCC000A965F16BC9192967B1697269891A696017
:10DCD000316AF269891A6961B16B726B891A696577
:10DCE000B16A726A8A1AEA61316BF36AC91AE96524
:10DCF000316CF36BC91A6967A86746F22C41DFF8EB
:10DD000058389A180A50A86F00F5C4429C322A620B
:10DD10004FF4BE726A6200F5C8431B1DAB6200235C
:10DD2000EB6200F5C24320332B636A6300F5C44203
:10DD30008832AA630022EA63A86443F290021318AF
:10DD40002B64EA646A6400F5C84238322A660858CF
:10DD500068668318AB666020E866A869E9690818F8
:10DD600003F1600188420AD2B06A019060200090FD
:10DD70000FF60C0221460FF69C00FBF7DDF8686FEA
:10DD80000A90286F0990686D0890286D0790E86DDB
:10DD90000690A86D0590E8690490A86903906869E9
:10DDA000029028690190686800902B6832692146CA
:10DDB0000FF69800FBF7C0F80D20FFF730FF129028
:10DDC0000D20FFF727FF11900C20FFF728FF109080
:10DDD0000C20FFF71FFF0F900420FFF720FF0E908D
:10DDE0000420FFF717FF0D900620FFF718FF0C9097
:10DDF0000620FFF70FFF06460820FFF710FF074633
:10DE00000820FFF707FF80460920FFF708FF81463B
:10DE10000920FFF7FFFE82460320FFF700FF83463D
:10DE20000320FFF7F7FE12990B9111990A911099AF
:10DE300009910F9908910E9907910D9906910C99E6
:10DE4000059104960397CDF80880CDF80490CDF89D
:10DE500000A05B46024621460FF66400FBF76CF813
:10DE60001E200090102340F2013221460FF6DC0004
:10DE7000FBF762F8A86F13B0BDE8F08FFFF7BEBDE7
:10DE800001684068814201D101207047002070473D
:10DE900001684068491C01F00F01814201D1012055
:10DEA0007047002070472DE9F04182B004460E46CD
:10DEB00017460025002C01D1092000E00820FFF7BB
:10DEC000A9FE804640F20230874226DA72B640460A
:10DED000FFF7DEFF002814D1D8F800004FF442719C
:10DEE00001FB0080103007603A463146001DF4F710
:10DEF000EDFAD8F80000401C00F00F00C8F8000050
:10DF000009E00FF684020FF2C8610FF68C00FBF7F0
:10DF100013F86FF0150562B60AE03B460FF668028B
:10DF20000FF2AC610FF68400FBF706F86FF01505F1
:10DF3000002D12D12046401E8041C043C00F002159
:10DF400000F007F9050017D00FF63C020FF28061D0
:10DF50000FF67400FAF7F0FF0EE0D8F80030D8F8AA
:10DF6000040000900FF620020FF264610FF67400B7
:10DF7000FAF7E2FF00F00FFA2846BDE8F68170B527
:10DF80000C46002801D1092000E00820FFF742FEDE
:10DF90000546002672B6FFF773FF00280DD16868AA
:10DFA0004FF4427101FB0050103001682160696834
:10DFB000491C01F00F016960061D62B6304670BD54
:10DFC0001CB50820FFF726FE026843688168C06818
:10DFD0000FF2FC540190009121460FF62800FAF749
:10DFE000ABFF0920FFF716FE026843688168C0682E
:10DFF0000190009121460FF63800FAF79DFF13BDFE
:10E0000000B583B0DFF84805806F00F5C8402430C4
:10E0100081680191416800910368C2680FF2B051B4
:10E020000FF63800FAF788FF07BDF8B5DFF820458E
:10E03000A06F002805D10FF64C010FF65400FAF737
:10E040007BFF002010E043F2900141430022A36FC8
:10E05000CA50A36FCB185A60A36FCB189A600122E5
:10E06000A36FC918CA60401C0228ECDB002000F036
:10E070002FFA002146F2201711E000EB4003A66FB3
:10E08000961916EB8306BD51A66F961916EB8303FE
:10E0900046F22416F550401C1E28EEDB491C0229CE
:10E0A00021DA4FF4BE7000FB01F20020A36FD318F9
:10E0B00046F28C25E850A36FD31846F28825E85025
:10E0C000A36FD31846F29025E8500120A36FD31810
:10E0D00046F29425E8500020A36FD31846F2982505
:10E0E000E850FF25D8E7F1BD10B4DFF86414896F5C
:10E0F0004FF4BE7212FB001000F5C2422032002025
:10E1000072B602F5B4714B68D2F86841A3420CD0E4
:10E1100003EB430002EB8000002282604A68521C3D
:10E120001E2A00D100224A6010E08C68002C0DD01D
:10E1300003EB430002EB8000002282604A68521C1D
:10E140001E2A00D100224A6000228A6062B610BCFA
:10E1500070472DE9FE4F0E46DFF8F413896F4FF438
:10E16000BE7212FB001101F5C2472037022802DA05
:10E170004FF0000801E04FF004084FF00009002FB5
:10E1800006D0B8F1000F0FF248440FF2207515D0F9
:10E1900043460FF218720FF238410FF21C70FAF773
:10E1A000CBFE4FF0FF309DE009EB89000090334635
:10E1B0002A4621460FF2D470FAF7BEFE72B607F572
:10E1C000B47ADAF80800002840F08E80D7F86801A9
:10E1D00000EB400117EB810B08D129460FF20070CC
:10E1E000FAF7AAFE62B64FF0FF307BE0DAF81010C3
:10E1F000002000F028F90290002844D0002000F010
:10E200004AF9019002980090DAF810302A46214627
:10E210000FF2E460FAF790FE0520FFF72FFEDAF820
:10E220001010002000F00FF9002804D0484600F13B
:10E2300001090528F0DBDAF81010002000F003F9DE
:10E240000346CDF80490DAF8100000902A462146E3
:10E250000FF2CC60FAF770FEDAF81010002000F030
:10E26000F2F800280FD0DAF81010002000F0EBF8D8
:10E2700003462A4621460FF2E860FAF75DFE62B6D1
:10E280004FF0FF302EE0CBF800600120CBF8080003
:10E29000DAF81000CBF80400D7F86801401C1E28FB
:10E2A00000D10020C7F86801DAF81000401C0F28E0
:10E2B00000D10320CAF81000D7F86801DAF804107A
:10E2C000884202D10120CAF8080062B6B8F1040FF2
:10E2D00007D0BBF1000F24D0DBF80410404600F05B
:10E2E0000CF90020BDE8FE8F62B60520FFF7C6FDE1
:10E2F000DAF80800002804D0484600F10109052892
:10E30000F3DBDAF8080000283FF44EAF2A46214636
:10E310000FF2A060FAF710FE00F03DF84FF0FF306A
:10E32000E0E74FF0FF30DDE77FB58949896F4FF4B3
:10E33000BE7212FB001101F5C2442034012801D144
:10E3400081A300E081A304F5B4700FF28425016974
:10E3500003918168029140680190D4F868010090AF
:10E36000224629460FF27060FAF7E6FD00260FE01C
:10E3700006EB4600800001198A6801924968009105
:10E380000359324629460FF28060FAF7D5FD761C14
:10E390001E2EEDDB7FBD38B50FF234240FF28C65F5
:10E3A0002A4621460FF29060FAF7C6FD0120FFF7DA
:10E3B000BBFF2A4621460FF29860FAF7BDFD002008
:10E3C000FFF7B2FF2A4621460FF29C60FAF7B4FD30
:10E3D000FFF7F6FD2A4621460FF2A460FAF7ACFDDE
:10E3E000BDE831400CE630B4594B9C6F002C16D080
:10E3F00046F224410A59521C0C19E5686D1CE5606F
:10E400009C6F0D592C1946F238452855986F0B18FA
:10E410009B689A4202D100220A5000E00A5030BCA8
:10E42000704710B44D4B03EBC004616003F830201B
:10E4300010BC7047494911F83000002801D0102065
:10E4400070470020704710B4444A02EBC003012417
:10E4500012F830000028586804D0806A04FA01F1EC
:10E46000084004E04069103104FA01F1084010BC92
:10E4700070473A4B03EBC000406800EB8200C0F8E5
:10E4800080107047354A02EBC000406800EB810005
:10E49000D0F880007047314901EBC00211F830001C
:10E4A0000028506801D040697047806A704710B4F6
:10E4B0002A4A02EBC003012404FA01F112F83000E9
:10E4C0000028586801D0C16000E0016210BC7047AC
:10E4D00038B504464FF6FF750020FFF7ABFF05FA8D
:10E4E00000F01E4901EBC40211F8341000295168F4
:10E4F00001D0C86031BD086231BD38B504460D4653
:10E50000002C01D100F0A6FE144800EBC40101224A
:10E5100010F83400002804D002FA05F04968C861F8
:10E5200031BD05F1100002FA00F04968886031BD84
:10E530000A4A02EBC0004068016070470448806FDF
:10E5400046F21841085870474132430043324100B7
:10E5500044CF030020C30200689BFFFF40D70300A5
:10E5600038B505460121FFF78DFF044602212846F4
:10E57000FFF788FF224601460020104334BD00000B
:10E580006970635F6765745F636875625F6D617012
:10E59000000000004E616E6F687562204F530000EE
:10E5A0005B455D25733A2025733A2025702068610C
:10E5B000732077726F6E67206D61676963206B658A
:10E5C000793A202573202D3E2025730A0000000093
:10E5D0006E616E6F6875622D697063005B455D25C5
:10E5E000733A2025733A206970635F7665727369A8
:10E5F0006F6E20646F65736E2774206D617463683D
:10E600003A2041502025642C20436875623A202529
:10E61000640A00005B495D25733A2025733A207730
:10E62000726F6E67207065727369737462756620AD
:10E63000616464723A25702C2025642C2069706313
:10E640005F656E643A307825780A00005B495D2585
:10E65000733A20636F6E74657874687562206D61BB
:10E660007020696E666F726D6174696F6E287625B1
:10E6700075290A20626C282570202564290A206FDC
:10E6800073282570202564290A2069706328257065
:10E69000202564290A2072616D28257020256429AF
:10E6A0000A20736861726564282570202564290A30
:10E6B0002064756D70282570202564290A000000EB
:10E6C0005B495D25733A206970635F6D61702069F5
:10E6D0006E666F726D6174696F6E0A20697063286F
:10E6E0002570202564290A20646174615F633261AA
:10E6F000282570202564290A20646174615F6132D5
:10E7000063282570202564290A206576745F6332AA
:10E7100061282570202564290A206576745F61329E
:10E7200063282570202564290A206C6F67282570CE
:10E73000202564290A207065727369737462756696
:10E74000282570202564290A000000005B495D250A
:10E75000733A206970635F6D617020646174615FFA
:10E7600063683A73697A653A2564206F6E20256480
:10E77000206368616E6E656C2E206576745F6368D9
:10E780003A25640A000000006970635F777269745B
:10E79000655F6461746100005B495D25733A202503
:10E7A000733A2069732066756C6C0A005B495D25BD
:10E7B000733A2025733A20696E76616C6964207320
:10E7C000697A653A25640A005B495D25733A20251C
:10E7D000733A206661696C206279206164645F65C8
:10E7E00076740A005B495D25733A2025733A2065EB
:10E7F00072726F723A2065713A25642C2064713A06
:10E8000025640A005B495D25733A206132633A2032
:10E8100065713A25642064713A25642066756C6CD4
:10E820003A256420656D7074793A25640A00000009
:10E830005B495D25733A206332613A2065713A2560
:10E84000642064713A25642066756C6C3A256420F6
:10E85000656D7074793A25640A0000005B495D2596
:10E86000733A20746F6B656E3A25642C2065713A9B
:10E8700025642C2064713A25642C2073697A653AEA
:10E8800025640A006970635F696E697400000000A6
:10E890005B455D25733A206970635F6D6170206927
:10E8A00073204E554C4C2E0A000000006970635FC7
:10E8B0006164645F657674005B455D25733A20256D
:10E8C000733A20696E76616C6964206970635F6574
:10E8D00076742C206F776E65723A25640A0000000A
:10E8E0005B455D25733A20696E76616C69642063CF
:10E8F00075725F6576740A005B455D25733A202565
:10E90000733A206972713A25642070656E64696E8D
:10E91000673A307825782D3E307825780A00000057
:10E920005B495D25733A2025733A2070656E6469F2
:10E930006E672069727120776169743A2070656E24
:10E94000643A2564206972712025642064757269B7
:10E950006E672025642074696D65730A00000000ED
:10E960005B455D25733A2025733A206661696C200A
:10E97000746F20616464206576742062792070650C
:10E980006E64696E673A307825780A005B495D25C8
:10E99000733A2025733A20657674202564206475C7
:10E9A00072696E67202564206D7320697320667517
:10E9B0006C6C0A005B455D25733A2025733A20662E
:10E9C00061696C20746F20616464206576742062D4
:10E9D000792066756C6C0A005B495D25733A206589
:10E9E0007674282570292D25733A2065713A25649F
:10E9F0002064713A25642066756C6C3A2564206940
:10EA000072713A25640A00005B495D25733A2065FE
:10EA100076742564286576743A25642C6972713A97
:10EA200025642C663A2564290A0000006970635F3A
:10EA300064756D70000000005B495D25733A202508
:10EA4000733A20613278206576656E740A000000A2
:10EA50005B495D25733A2025733A20633261206556
:10EA600076656E740A0000005B495D25733A2025C7
:10EA7000733A2064617461206275666665720A008B
:10EA80005B495D25733A2025733A206C6F672062DD
:10EA900075666665720A000002F060B980B50F28DD
:10EAA0000BDB23220FF240010FF23000FAF744FA99
:10EAB0000020C046C046002002BDBDE8024002F072
:10EAC0008DBA0F2801DB00207047102901D30020E8
:10EAD000704702F0C9BA02F004BB00005B455D2537
:10EAE000732C2025640A0000443A5C506572666FFE
:10EAF0007263655C53454E534F525F534C4F4341D5
:10EB000054494F4E5F494E4E4F565F313731365F55
:10EB100038415C434F4E464944454E5449414C5C54
:10EB200053656E736F724875625C4D4153535F500D
:10EB3000524F4A4543545C50524F445C4135315C1E
:10EB4000545C706C6174666F726D5C6578796E6F21
:10EB500073393631305C6669726D776172655C6FEE
:10EB6000735C706C6174666F726D5C6578796E6FE2
:10EB7000735C7372635C636D755C636D752E6300AB
:10EB8000102810D8DFE800F0090B090B090B090B5E
:10EB90000F0F0F0F0F0F0F0F0D00002070470120F8
:10EBA00070470220704703207047024951F8200047
:10EBB00070470000C056030002F04ABB02F055BB8C
:10EBC00002F060BB10B5044602F071FB20702078A3
:10EBD000FFF7D6FF60702078FFF7E7FF606010BD99
:10EBE00080B502F093FB02F0D1FBBDE8014002F0DA
:10EBF000EFBB000030B5044610480D460178491CB3
:10EC0000017081B0802080F3118800BF00BFA06830
:10EC100058B94021204602F003F8802080F3118883
:10EC200000BF00BFA0680028F3D02946204602F0AC
:10EC300052F801B0BDE83040F7F716BE705E030031
:10EC4000012100F01F0291408A4A400942F8201039
:10EC50007047012100F01F029140874A400942F8A5
:10EC60002010704780B50020FFF768FC0FF21021DC
:10EC70000FF21820BDE80440FAF75EB980B50246ED
:10EC8000D21E052A0BD8DFE802F0030C0C030A079A
:10EC90000020FFF70CFC04E0FFF7E4FF01E000F0C8
:10ECA00051F90020FFF75CFCBDE80440F9F71DBAFC
:10ECB000F0B585B00020FFF7EEFB04460020FFF71B
:10ECC000B9FB054605F10F062046F040C00747D5C1
:10ECD00003210020FFF7D6FBC7B2022F0AD103227F
:10ECE00000210846FFF7C5FB0020FEF7A4FF00F057
:10ECF000B6FA0BE0012F09D100F0ACFA0322002193
:10ED00000846FFF7B6FB0120FEF795FF082F01D15B
:10ED100000F0A0FA0120B040844331460020FFF704
:10ED2000C6FB022F03D00F210020FFF7E6FB012FC7
:10ED300005D0022F03D0042F01D0082F10D100A836
:10ED40000FF2EC111422F3F7D1FBADF8037000A819
:10ED5000F9F77AFD002803D00FF26410FAF7ECF807
:10ED6000002C27D00AE0076829460020FFF79FFB08
:10ED700029463846C0B2FFF781FF6D1CB54219DA4B
:10ED80002046E840C007F8D50120FFF7ADF900287C
:10ED9000E9D100F033F90020FFF77DFB0090234616
:10EDA0002A460FF204110FF22810FAF7C5F80020D6
:10EDB000FFF78EFB05B0F0BD70B50120FFF76BFBD0
:10EDC00004460120FFF736FB054621460FF23410BA
:10EDD000FAF7B2F82E460BE02046F040C00706D501
:10EDE000304600F047F931460120FFF760FB761C02
:10EDF00005F110008642EFD370BD70B50FF2101010
:10EE0000FAF79AF80320FFF746FB04460320FFF7C2
:10EE100011FB05462E4607E02046F040C00702D50C
:10EE2000701B00F0A6F9761C05F10F008642F3D3A3
:10EE300070BD80B50020FEF7E9FEFEF704FF002854
:10EE400017D00C20FEF7E6FE0C4908600E20FFF7F5
:10EE500000FF0E20FFF7F4FE1020FFF7FAFE10204F
:10EE6000FFF7EEFE1120FFF7F4FE1120BDE802408F
:10EE7000E6E601BD00E100E080E200E05CDA0300CC
:10EE800068616E646C654465627567005B495D2509
:10EE9000733A20646F65736E277420737570706F9A
:10EEA000727465642E0A00006D61696C626F78414E
:10EEB000505F49525148616E646C657200000000F9
:10EEC0004D534720426F782046756C6C0A00000055
:10EED0005B455D2573282564293A206576656E7447
:10EEE0007120697320656D7074792C20737461745E
:10EEF00075733A307825782853523A307825782936
:10EF00000A0000005B495D6841504D3A25780A00CF
:10EF10005B495D4D61696C626F78476E7373324314
:10EF20006875625F49525148616E646C65720A008F
:10EF300003FF380000000000000000000000000097
:10EF40000000000010B5ADF5427D334C207800285C
:10EF500021D0002240F2013101A8F3F789FA00A97B
:10EF60000120FFF70CF8010003D0009A01A8F3F785
:10EF7000ADFA009840F20231884204D2014601A85D
:10EF800000F036F82BE002460FF294010FF2AC00CD
:10EF9000F9F7D2FF23E0A068002820D000A90120C3
:10EFA000FEF7EDFF002807D0009A0146A068F3F7AE
:10EFB0008DFA0020009002E04FF0FF300090A16831
:10EFC0006368180003D0009AE068984707E00023C0
:10EFD0000A460FF24C010FF28000F9F7ADFF0DF574
:10EFE000427D10BD0C494A60CB60886000207047AC
:10EFF0000A4692B201460020FEF755BF80B5FFF7E2
:10F0000014F8002205491046FFF70BFA01210020F1
:10F01000BDE80440FFF78CBAA8D9030000003840CF
:10F020006D61696C626F7844727648616E646C657C
:10F0300052784D6573736167650000005B455D251F
:10F04000733A20696E76616C69642073697A653AF7
:10F050002025640A000000005B455D25733A206EA0
:10F060006F2063616C6C6261636B3A2025782C20A1
:10F0700025780A0010B5044621460FF2A400F9F7DE
:10F080005BFF002C0AD102210120FFF7FBF90146AA
:10F090000FF2A000BDE81040F9F74EBF10BD38B523
:10F0A0001C4C4FF4803504E00FF29C00F9F744FF4C
:10F0B00025600120FFF7EFF90028FAD00021012098
:10F0C000FFF7F5F902210120FFF7DCF90100EBD58C
:10F0D000256031BD80B510490A68521C53015B0997
:10F0E0000B60002240EA03110120FFF7C2F9002162
:10F0F0000120BDE80440FFF700BA80B500220749AF
:10F100000120FFF78EF901210846BDE80440FFF712
:10F110000FBA000080E200E058DA03000000374038
:10F120005B495D206841504D3A6972713D25640A22
:10F13000000000005B495D206841504D3A73723217
:10F140003D253038580A00005B495D453A30782546
:10F150003038580A00000000234A42F82010704757
:10F1600001460320FFF7C9B900F110010320FFF7A2
:10F170009EB910B50446FFF7F7FF1B4850F824105E
:10F180000A0008D122460FF274010FF28800BDE890
:10F190001040F9F7D1BE002C01D0012C01D18847D5
:10F1A00003E0022C01D180688047002C01D0012CA3
:10F1B00003D12046BDE81040D2E710BD80B5012242
:10F1C0000A490320FFF72DF902F0DAFA0849002076
:10F1D000FFF7C2FF07490120FFF7BEFF06490220E3
:10F1E000BDE80440B8E7000070D4030000003940D7
:10F1F000410201004B020100512501006D61696C63
:10F20000626F78476E737344727668616E646C6582
:10F21000497271005B455D25733A2057726F6E67C6
:10F2200020696E74657272757074206861707065A3
:10F230006E6564286576656E743A20256429000041
:10F2400041F210003C494860704740F201103A49D1
:10F250004860704741F2100037490860704740F23B
:10F26000011035490860704740F2011032494A6880
:10F27000824204D10968814201D1002070470120F7
:10F28000704700002DE9F0412C4E346800254FF006
:10F29000FF302B49086072B62846F9F773FB02F07D
:10F2A000B5FB0746274802F0ADFB274A1068C002AD
:10F2B00003D54FF480102549086010682946204086
:10F2C000294001D100280CD06FF0604002F09CFB77
:10F2D000384602F097FB34600220F9F753FB62B620
:10F2E00028E0DFF8688010686040C8F8000018481F
:10F2F00001600068C00303D54FF000701549086035
:10F300000120F9F73FFB4FF48030306030BF00BF81
:10F31000F8F765FF29460120FFF7C9F84FF4881078
:10F32000C8F800006FF0604002F06EFB384602F053
:10F3300069FB3460BDE8F081FC66030000E100E099
:10F3400080E100E0FFFFFE1F00E200E080E200E05D
:10F3500010E000E004ED00E0103003689343002962
:10F3600000D013430360704701680A68437B002B99
:10F3700002D122F0100201E042F01002837B002B48
:10F3800002D122F0080201E042F00802C37B002B08
:10F3900002D122F0040201E042F004020A6002F00D
:10F3A00001030168096801F001019942F9D1704730
:10F3B00003689B089B00002901D043F00203002A48
:10F3C00001D043F001030360704710B582B00446DA
:10F3D00000221146FFF7ECFF002020622046016862
:10F3E0000091009941F0200100910099016004F121
:10F3F00014010A680092009A12F4FC3FF9D10A68DD
:10F400000092009A12F4FC6FF9D101680091009902
:10F4100021F020010091009901600168009100999C
:10F420008906FAD413BD2030036823F480330360C7
:10F4300062F30F03002901D043F480330360704767
:10F4400010B4016808310A6890F83030012B02D1FD
:10F4500042F0040201E022F0040290F83130012B66
:10F4600002D142F0020201E022F0020290F84430A0
:10F47000012B02D142F0010201E052085200036A5E
:10F48000DFF86046002B02D0224042EAC34424F455
:10F49000C02290F8243042EA434222F4FC62C36A5C
:10F4A00042EA431222F4FC32836A42EAC32290F811
:10F4B0006500002802D042F0080001E022F00800B8
:10F4C000086010BC704708300268002902D042F082
:10F4D000080101E022F008010160704701680C3169
:10F4E0000A6890F84C30002B02D042F0040201E090
:10F4F00022F0040222F47C72806C42EA0010086060
:10F50000704790F85C1090F85D2042EA01110068A5
:10F510008162704790F85E100068C16270471030D9
:10F52000016841F00301016070471F21416270478B
:10F530000C300268002902D05108490001E042F075
:10F54000010101600020704770B504460FF2AC5510
:10F550000FF2A0562368002231462846F9F7ECFC4A
:10F56000A368082231462846F9F7E6FCE3680C2236
:10F5700031462846F9F7E0FC236910223146284637
:10F58000F9F7DAFC6369142231462846F9F7D4FC0E
:10F59000A369182231462846F9F7CEFCE3691C22FC
:10F5A00031462846F9F7C8FC236A2022314628460E
:10F5B000F9F7C2FC636A242231462846F9F7BCFCFD
:10F5C000A36A282231462846F9F7B6FCE36A2C22C2
:10F5D00031462846BDE87040F9F7AEBCF0B583B0BF
:10F5E00006460027F8F714FE04460D4670698001B0
:10F5F00021D43846471C42F211718842F6DB0020C4
:10F600000146001BA941DFF8E02400239942EDD315
:10F6100001D89042EAD300200146CDE900012246FC
:10F620002B460FF2F4410FF20850F9F785FC3046F3
:10F63000BDE8FE4088E7F7BD10B4DFF8B024E4234E
:10F6400003FB00204A68426091F84C2080F84C206F
:10F65000021D0B1D5C6954615C7A54729C7A947231
:10F66000DC7AD4721C6914611B7E137691F8242015
:10F6700080F8242000F1240201F124031C7B147380
:10F680005B7B537391F85E1080F85E1010BC70477E
:10F6900010B5DFF85814E42202FB00140120E062E8
:10F6A0002046FFF761FE2046FFF7CAFE2046FFF71F
:10F6B00015FF2046FFF725FF2046FFF72BFF94F8A4
:10F6C0003100042803D094F83000042802D12068C7
:10F6D000FFF725FF2068FFF728FF94F83100042882
:10F6E00003D094F83000042810D10020C4F8900012
:10F6F000C4F8A000C4F89800C4F8A800C4F8B0008A
:10F70000C4F8B800C4F8C800C4F8C0002068FFF707
:10F710005CFE002010BD80B5E4214143DFF8CC231E
:10F720000FF23C4353F820308B5089184860FFF7A4
:10F73000AFFF002802D04FF0FF3002BD002002BD15
:10F74000F8B50F461D46DFF8A413E42303FB0016AB
:10F7500096F82400002841D196F84C000028144661
:10F7600014D0294603E017F8012B0276491E3068B1
:10F770000029F8D101221146FFF71AFE002D25D0ED
:10F780003068007F04F8010B6D1EF7E70022114678
:10F790003068FFF748FE012211463068FFF708FE87
:10F7A00001213068FFF7C4FE0AE017F8011B01765B
:10F7B0003068FFF713FF3068007F04F8010B6D1EFF
:10F7C0003068002DF1D10021FFF7B2FE3068FFF75D
:10F7D00005FF3068FFF7F9FD0020F2BD012843D195
:10F7E00096F84C000028144614D0294603E037F858
:10F7F000022B0283491E30680029F8D101221146EC
:10F80000FFF7D6FD002DE1D03068808B24F8020B85
:10F810006D1EF7E7002211463068FFF704FE012253
:10F8200011463068FFF7C4FD002D0EE0401EFDD1EB
:10F8300000213068FFF77CFE3068808B24F8020BD3
:10F840003068808B24F8020B6D1EBFD00121306818
:10F85000FFF76EFE37F8020B3168088337F8020BAA
:10F86000316808839620E2E70228AFD196F84C0071
:10F870000028144614D0294603E057F8042B82616F
:10F88000491E30680029F8D101221146FFF790FD8A
:10F89000002D9BD03068C06944F8040B6D1EF7E75B
:10F8A000002211463068FFF7BEFD01221146306884
:10F8B000FFF77EFD002D0EE0401EFDD100213068D7
:10F8C000FFF736FE3068C06944F8040B3068C06941
:10F8D00044F8040B6D1E3FF479AF01213068FFF747
:10F8E00027FE57F8040B3168886157F8040B31681C
:10F8F00088619620E1E738B57C4CE42505FB00449F
:10F90000C4F8CC10C4F8D0300020C4F8D400C4F837
:10F91000D820C4F8DC30C4F8E000022201212068BD
:10F92000FFF71AFD012211462068FFF715FD0020A0
:10F9300032BD2DE9F84304460D4616461F464FF0EA
:10F9400000086A48E42101FB040999F864000028D2
:10F9500003D0D9F80000FFF738FD99F865000028BA
:10F9600004D00121D9F80000FFF7ADFD99F831006E
:10F97000002807D13B46324629462046FFF7E0FEE5
:10F98000804608E0042806D13B46324629462046F8
:10F99000FFF7B1FF804699F86500002804D00021E8
:10F9A000D9F80000FFF78FFD4046BDE8F2832DE94E
:10F9B000F84F04468A4615461E464C48E42101FB92
:10F9C00004074FF00009FF2E02D94FF0FF080FE0A7
:10F9D000B0460DE00BF1040105EB8900F2F776FD6E
:10F9E00008EB0900864201D2A6EB0908C144CA44CB
:10F9F000B14532D2DFF8F8B0584697F82410002904
:10FA000003D14AF08001017008E0012903D14AF4D2
:10FA10000041018002E04AF00041016008F1010369
:10FA20005A4659462046FFF784FF002816D197F81A
:10FA30002400002807D142460BF1010109EB050023
:10FA4000F2F744FDCCE701284246C3D10BF1020195
:10FA500005EB4900F2F73AFDC2E70020BDE8F28F5E
:10FA60002DE9F84F04468A4615461E461F48E421F4
:10FA700001FB04074FF00009FF2E02D94FF0FF08E9
:10FA800009E0B04607E008EB0900864201D2A6EB88
:10FA90000908C144CA44B14520D2DFF854B05846E1
:10FAA000014697F82420002A07D181F800A03246A9
:10FAB0002946401CF2F70AFD06E0C1F800A0B2009A
:10FAC0002946001DF2F702FD08F101030022594604
:10FAD0002046FFF72EFF0028D5D000E00020BDE82B
:10FAE000F28F00000000F81F819698008C910300AF
:10FAF00090A4030064756D70537069005B4C4F47B0
:10FB00005F494E464F5D25733A202B25643A2030DD
:10FB10007825780A000000005F5F776169745F757F
:10FB20006E74696C5F74785F646F6E6500000000CE
:10FB30005B4C4F475F4552524F525D25733A206FE1
:10FB400075742120696E54696D653A256C6C752C4D
:10FB5000206F757454696D653A256C6C750A0000E8
:10FB600000001C4000007040000070400000724027
:10FB7000000074400000764000EB40010801DFF80F
:10FB8000E8144258136843F000431360405801687A
:10FB9000490049080160704770B4022802D2DFF8BA
:10FBA000CC4401E0DFF8C84400EB40021001DFF86C
:10FBB000B82483185B6886581B01B4FBF3F3DDB2ED
:10FBC0004FF0FF3301292DD106F15C010E6826F4B8
:10FBD0007F0646EA05460E60691CC4EBC404DFF8E4
:10FBE0009454B4FBF5F4642515FB01F1B4FBF1F179
:10FBF0008458583425682D0A1E46CE408E40F6B2F1
:10FC000056EA05252560491E80585430026822F4C2
:10FC10007F021C46CC4004FA01F1C9B242EA01411C
:10FC200001602CE006F168010E6826F47F0646EAC2
:10FC300005460E60691C04EBC404DFF83854B4FBBD
:10FC4000F5F401EB81056900B4FBF1F184586434EB
:10FC500025682D0A1E46CE408E40F6B256EA05258E
:10FC60002560491E80586030026822F47F021C46DD
:10FC7000CC4004FA01F1C9B242EA0141016000201E
:10FC800070BC704710B504460021FFF785FF0028BF
:10FC900010D1DFF8D40304EB440100EB01104068FD
:10FCA000DFF8D413884208D301212046FFF774FF00
:10FCB000002802D0DFF8C40310BD002010BD38B505
:10FCC00000EB40010C01DFF8A053605901680FF20E
:10FCD000C030F9F731F9605941680FF2C830F9F7CF
:10FCE0002BF9605981680FF2D430F9F725F9605982
:10FCF000016A0FF2E430F9F71FF96059416A0FF217
:10FD0000EC30F9F719F96059016B0FF2F830F9F797
:10FD100013F96059016C0FF20440F9F70DF96059BD
:10FD2000416C0FF20C40F9F707F96059016D0FF2C1
:10FD30001440F9F701F96059416D0FF22440F9F7C9
:10FD4000FBF86059816D0FF23040F9F7F5F8605912
:10FD5000C16D0FF23C40F9F7EFF86059016F0FF2F7
:10FD60004840BDE83440F9F7E7B82DE9F8430746C5
:10FD7000884607EB47000401BB4D6619307BC0077E
:10FD800001D500202BE00FF2A84050F82700605169
:10FD9000C6F804800020B060F06030613846FFF79C
:10FDA000EBFE6059016841F00809C0F80090384640
:10FDB000FFF768FF0F2061598860AF48804506D380
:10FDC00060594030016841F00059C0F8009049F096
:10FDD00000406159086401203061F0600020BDE8F6
:10FDE000F283A14900EB400201EB02100021C16047
:10FDF00001610846704780B59B4900EB4002100145
:10FE00004058016D01F00F00012805D00FF2AC3011
:10FE1000F9F792F8002002BD012002BD2DE9F84F4C
:10FE200004460D46002604EB44000701DFF8388243
:10FE300057F808301968586C4833D3F800C04FEAB7
:10FE40004C0C4FEA5C0CC3F800C08D4B57F808C04F
:10FE5000CCF804302B79DB0704D541F0400140F4A5
:10FE6000803003E021F0400120F48030012A02D1EB
:10FE700040F4003001E020F4003057F808207032E0
:10FE8000136803F4700395F800C00CF07F0C43EA8C
:10FE90008C23136057F808201160000C2979C907DA
:10FEA00003D5A96851EA004002E0E96851EA004040
:10FEB00057F80810486457F808004430016841F0CA
:10FEC00000410160DFF8BC91CA4607EB080BDBF884
:10FED00008002979C9072BD5002862D101F096FDC9
:10FEE00040F0210001F08EFD802057F808100862D4
:10FEF000654908460246501E002A4BD057F8082094
:10FF0000136BDB0104D4926B28693254761C0846CB
:10FF1000AA689642EED308460146481E002939D009
:10FF200057F8081024310A680A60110630D4F3E744
:10FF300000281DD101F06AFD40F0210001F062FDB2
:10FF4000802057F8081008624F480AE057F8081058
:10FF50000A6B02F07F02102A03D26A69B25C761C37
:10FF60004A630146481E002902D0E9688E42EDD35B
:10FF7000DBF80800002814D143480146481E002938
:10FF800008D057F8081024310A680A601106F4D521
:10FF90004FF0000ACA4504D12046FFF790FE4846BC
:10FFA00000E05046BDE8F28F2DE9F04104460D46D1
:10FFB00001260027002D02D16FF4004046E02A48B8
:10FFC00004EB440100EB011898F80C00C00701D4C1
:10FFD0002E483BE02046FFF70EFF002807D12046C1
:10FFE000FFF7FFFED8F804102046FFF7BEFE3846A4
:10FFF0006860A868002800D03E46E868002824D041
:020000021000EC
:100000004FF480406860324629462046FFF706FFDD
:10001000070006D039460FF2D010F8F78DFF3846AA
:1000200014E0002E11D1686840F0010068600122E0
:1000300029462046FFF7F2FE070006D039460FF2A8
:10004000CC10F8F779FF384600E03846BDE8F0817B
:100050000C2801D300207047034900EB400201EB5C
:10006000021040687047000024B5030000EA320621
:100070000080BB0040420F00811A0600FE7FFFFF98
:1000800083000800FD7FFFFFA0860100FC7FFFFFCB
:100090005B495D4932432043544C203A2025780A7D
:1000A000000000005B495D493243204649464F5FEE
:1000B00043544C203A2025580A0000005B495D4912
:1000C000324320545241494C494E475F43544C20DF
:1000D0003A2025580A0000005B495D493243204917
:1000E0004E545F454E203A2025580A005B495D4931
:1000F000324320494E545F53544154203A202558EE
:100100000A0000005B495D493243204649464F5F83
:1001100053544154203A2025580A00005B495D4958
:10012000324320434F4E46203A2025580A00000013
:100130005B495D49324320434F4E4632203A2025E9
:10014000580A00005B495D493243205452414E53E6
:1001500020535441545553203A2025580A0000009A
:100160005B495D4932432054494D494E472048532D
:1001700031203A2025580A005B495D49324320541A
:10018000494D494E4720485332203A2025580A000D
:100190005B495D4932432054494D494E47204853FD
:1001A00033203A2025580A005B495D4932432041FB
:1001B000444452203A2025580A0000005B455D491E
:1001C000324320427573206973206E6F7420494456
:1001D0004C45203A205452414E535F53544154559C
:1001E00053203D2025780A005B455D6932634472E7
:1001F000764D6173746572205472616E736D6974AB
:10020000204661696C203A2025640A005B455D69DF
:1002100032634472764D6173746572205265636512
:10022000697665204661696C203A2025640A0000E1
:1002300000001C4000001D400000704000007140A4
:1002400000007240000073400000744000007540E0
:1002500000007640000077400000784000007940C0
:1002600010B50446084611461A46029BA04710BD29
:100270002DE9F84C2DED068B154603B4C1F30A5059
:1002800040F2FF7188420CD101980024000304BFA2
:100290000098002802D1019800281BD4DDE9000154
:1002A00013E101280FDA00A800F092F901280ADB17
:1002B00000F0FEF92221016002B00020BDEC068BA7
:1002C000A249BDE8F48C019A40F2FE3161F31E525E
:1002D0000192441A019800280CD500F0E9F9212177
:1002E000016002B04FF0FF30BDEC068B6FF00041B3
:1002F000BDE8F48CDDE90001954A964BF6F742F92A
:1003000009D2DDE9002300204FF08041F5F768FFB6
:10031000CDE90001641EDDE9002300208E49F6F7D7
:100320005DF8DDE9002341EC180B00208B49F6F75E
:1003300055F802460B4651EC180BFAF7E5FC41EC78
:10034000190B53EC192BF5F74BFF41EC1A0B53EC3F
:100350001A2B83488349F5F743FF834A834BF6F70B
:100360003DF853EC1A2BF5F73BFF814A814BF6F72A
:1003700035F853EC1A2BF5F733FF7F4A7F4BF6F72E
:100380002DF853EC1A2BF5F72BFF7D4A7D4BF6F732
:1003900025F853EC1A2BF5F723FF7B4A7B4BF6F736
:1003A0001DF853EC1A2BF5F71BFF794A794BF6F73A
:1003B00015F853EC1A2BF5F713FF02460B4651ECD8
:1003C000180BF9F7AFFC53EC192BF5F709FF41ECCB
:1003D000190B20B2F8F7C2FD41EC1A0BCDB953EC62
:1003E0001A2B6D486D49F5F7FBFE53EC192BF9F705
:1003F00099FC53EC182BF5F7F1FF04460D4653EC2E
:100400001A2B4FF040406649F5F7EAFE22462B468C
:1004100059E0012D53EC182B34DB00206149F5F72E
:10042000DFFE82468B4653EC182B5F485F49F5F799
:10043000D7FE06460F4653EC1A2B5D485D49F5F78B
:10044000CFFE04460D4653EC192B5B485549F5F792
:10045000C7FE02460B4620462946F9F763FC3246A2
:100460003B46F5F7BBFF52465B46F5F7B7FF044640
:100470000D4653EC1A2B00205049F5F7B1FE2246E9
:100480002B4620E04FF0C0404D49F5F7A9FE044649
:100490000D4653EC182B4B484B49F5F7A1FE064689
:1004A0000F4653EC192B49484549F5F799FE02468A
:1004B0000B4630463946F9F735FC22462B46F5F710
:1004C0008DFF53EC1A2BF5F789FF02B0BDEC068BBC
:1004D000BDE8F48C80B52DED028B41EC180B53EC8C
:1004E000182B1F481F49F5F77BFE1F4A1F4BF5F7D6
:1004F00075FF53EC182BF5F773FE1D4A1D4BF5F7EE
:100500006DFF53EC182BF5F76BFE1B4A1B4BF5F7F1
:1005100065FF53EC182BF5F763FE194A194BF5F7F5
:100520005DFF53EC182BF5F75BFE174A174BF5F7F9
:1005300055FF53EC182BF5F753FE154A154BBDEC40
:10054000028BBDE80050F5F749BF00000000F0FF46
:10055000CD3B7F669EA0E63F0000F0BF0000F03F6D
:10056000F7DE29BFD8F8C23FF4B3FECC1A99C33FD7
:1005700062CB68D96F46C73FC6C912DAC471CC3F97
:100580004AE98A942449D23FF75F97999999D93FCC
:10059000BC5555555555E53F9EBC9AF71C7D7F3E91
:1005A000422EE63F7BCBDB3FABA6320EE526553E27
:1005B0007CC4BC7FDE27743E0EE526151344D33F72
:1005C0004715F73F44DF5DF80BAE543EFE822B65C6
:1005D00030B4436803F0004201211B031B0B43604E
:1005E00004BF0368002B08D10DE00368DD0F45EA66
:1005F000440444605B000360491E4468E302F4D590
:1006000023031B0B436043681A434260084630BC17
:1006100070474268C2F30A5240F2FF739A4209D10E
:100620004168090304BF0068002801D10120704718
:100630000220704743685B0004BF0368002B25D08D
:1006400040F233439A1A521A012A1FDB352A06DB7D
:10065000416801F0004141600021016013E0012187
:1006600002F01F039940491E920607D542681140C7
:100670004A40426002681143002202E002681140D1
:100680004A40026011B14FF0FF30704700207047C0
:1006900090420CD141EA030C50EA4C0C07D099422D
:1006A00005D14FF4001C1CEB410F38BF8942704745
:1006B000014801F0AFB90000000003002DE9704CC3
:1006C00004462DED088B94ED009B43EC182B51EC68
:1006D000190B01F0ABF9064651EC180B01F0A6F925
:1006E00031000E9D06D500284DD4022805D184ED99
:1006F000008B42E1022EF8D121E050B951EC190BE8
:100700000022344BFFF7C4FF0FD084ED008B002094
:1007100033E1012818D151EC190B00222E4BFFF7C1
:10072000B7FF18BF84ED008B51D1FFF7C1FF212126
:1007300001604FF0FF306FF00041C4E90001BDECF3
:10074000088B0220BDE8708C7EB984ED008B2946B1
:10075000204600F04FF9040018BF012C40F00C8136
:10076000FFF7A6FF2221016006E151EC190B0022E0
:10077000184BFFF78DFF0DD151EC180BF5F730FD3D
:10078000C4E9000123E051EC190B0022134BF5F7EB
:10079000F9FE0BD251EC180B0023F5F721FDC4E94B
:1007A0000001BDEC088B0020BDE8708C01220C4BD1
:1007B000F5F7D0FE16D851EC180B0022054BF5F7D3
:1007C0000FFDC4E90001FFF773FF22210160012042
:1007D000D3E000BF0000F07F0000F0FF00C89CC025
:1007E00000C89C40384A394BF5F7FAFC0022002338
:1007F000F5F7C8FE34BF9FED360B9FED370B53EC7A
:10080000102BF5F7EBFDF5F7BDFD0646F8F7A6FB57
:1008100041EC1A0B4FF07842314BF5F7E1FC024600
:100820000B4651EC190BF9F77DFA82468B4653ECD7
:100830001A2B2C482C49F5F7D3FC02460B465046A0
:100840005946F9F76FFA6FF00102284BF5F782FE6F
:1008500041EC190B05D80022254BF5F793FEC0F0AB
:100860007D8053EC192BF5F7BBFC41EC1A0B214AA8
:10087000214BF5F7B5FC214A214BF5F7AFFD53ECC1
:100880001A2BF5F7ADFC1F4A1F4B41EC1B0B51EC2B
:100890001A0BF5F7A5FC1D4A1D4BF5F79FFD53EC10
:1008A0001A2BF5F79DFC1B4B0022F5F797FD53EC37
:1008B000192BF5F795FC41EC190B9FED01AB2BE0E3
:1008C000000000000000F03FFE822B654715F73F57
:1008D000000000000000E0BF000000000000E03F5A
:1008E000422EE63FF2E4D5BCE7E84B3EFFFF8FBC6B
:1008F0000000903C112E5781A03F503F5843128C6E
:100900008F71BC3F4BE8A541B752013F0BBDF3DAF5
:10091000E8708C3F0000E03F51EC1B0B53EC192BAF
:10092000F5F75CFD53EC1A2BF5F758FD82468B4624
:1009300051EC1B0B53EC192BF9F7F4F953EC1A2B70
:10094000F5F74CFD02460B4650465946FAF7DCF9DE
:1009500053EC182BF5F744FC41EC180B84ED008B9D
:10096000A919204600F046F8040018BF012C03D155
:10097000FFF79EFE222101602046BDEC088BBDE8FA
:10098000708C00000278C9B28A421AB11CBF10F8FC
:10099000012FF9E718BF002070470000C9B2830794
:1009A00006D0521E22D310F8013B9942F7D11FE026
:1009B000083A13D302F1040241EA012141EA01415C
:1009C00050F8043B121F21BF4B40A3F1013C2CEA1D
:1009D000030C1CF0803FF3D0C9B2001F083210F89E
:1009E000013B521E28BF91EA030FF8D818BF01201F
:1009F000401E704770B504460D466068C0F30A504B
:100A000040F2FF71884207D16068000304BF20688C
:100A1000002817D0022070BD20B92046FFF7D8FD6E
:100A2000012868DA012D0FDB40F2FF71091A8D42AF
:100A30000AD3606800284CBF9FED300B9FED310B4F
:100A400084ED000B012070BD4142A942616806DAC5
:100A50006FF31E51401941EA0050606042E0401EB1
:100A600063684519012205F1350062F31F533528EB
:100A700001F00041636003D361600020206070BD1D
:100A8000002215F11F0F04DA2268236000202035B0
:100A90006060684214D0521E25689241C0F1200364
:100AA000D2439D4045EAD272256825FA00F6656872
:100AB00005FA03F333432360636823FA00F56560A6
:100AC00060680843B2F1004F606003D80DD1207810
:100AD000C0070AD52068401C2060206828B96068DB
:100AE000401C60604FF0FF3070BD6068884204BFFA
:100AF00020680028F6D1002070BD00BF0000000073
:100B00000000F0FF000000000000F07F91FBF2F316
:100B100003FB1211C0E900317047000007490A7851
:100B2000521C0A7000224A70114681F31188044950
:100B3000087008780028FCD1704700BF705E030081
:100B40007FDA03001FB5FFF7B3FD212101601FBD50
:100B50001AA210EE101ADFF860C0F2EC060A614526
:100B600009DB00EE803A70EE800A83EE200A40F046
:100B7000020010EE101A21F0004CDCF1665C0BD87C
:100B800060EE000A20EE203A03EE010A01EEA02AF0
:100B900042EE202A80EE220A400810F0020F18BF11
:100BA000B1EE400A02EB8002D2ED000A30EE200ADC
:100BB00028BFB1EE400A7047A430893ED7B3DD3F6D
:100BC0006AD5033F2B94A93DB82A593F0000803FC6
:100BD000000080BF00000000920A063FDB0FC93F03
:100BE000920A863FDB0FC93F920A0640DB0F49405D
:100BF000368D274010B5044602E0C068F5F750FE78
:100C0000802080F3118800BF00BF20680028F4D145
:100C10000248407808B980F3118810BD705E030067
:100C200000B50D4A936885B003930290019080232C
:100C300083F3118800BF00BF0368009300AB03601B
:100C4000009800B14360906800AA82600174F5F7D3
:100C5000A3FE05B000BD00BF705E0300012000F0E0
:100C600005BF00000749086808B100207047064822
:100C7000C008C00008600549C908C900091A016018
:100C8000704700BF74DA03000F2003000840030020
:100C900030B482B083680469828AE318C468A342CE
:100CA00028BF1B1B5343446811F8015B1D555B1C97
:100CB000521EF8D18168491C8160012903D102B01C
:100CC00030BCFFF797BF1948407808B980F3118806
:100CD00002B030BC704710B481B0828A03695343BC
:100CE00044681C5D01F8014B5B1C521EF8D1016980
:100CF000491C0161C268914224BF002101618168E1
:100D00004B1E83609142094B5B7807D113B90021D8
:100D100081F3118801B010BCFFF76CBF13B900203C
:100D200080F3118801B010BC70470000705E0300B2
:100D300001E0491C521E72B10B7890F800C09C452E
:100D400005D002D24FF0FF3070470120704710F8F5
:100D5000013B002BEDD1002070470000DFF8C813E5
:100D60000860DFF8C8031021016001680906FCD49F
:100D7000DFF8BC03012101600168C903FCD4012133
:100D800041604168C903FCD4DFF8A8030121016078
:100D90000168C903FCD4002141604168C903FCD447
:100DA0007047DFF894037047DFF880030068C006DF
:100DB00003D5DFF8740300687047DFF87C037047E1
:100DC000F2E7F1E780B5DFF868030068C00702D5F5
:100DD000FFF7F6FF01E0DFF86003DFF8581309685A
:100DE00001F00F01491CB0FBF1F002BD7047DFF8C4
:100DF00044130A68120900F00F0050EA021008605C
:100E00000868C003FCD4704780B5DFF83003006881
:100E1000C00702D5FFF7D4FF01E0DFF81C03DFF8BD
:100E20002013096801F00F01491CB0FBF1F002BD6D
:100E3000DFF80C130A68120900F00F0050EA0210E4
:100E400008600868C003FCD47047DFF8F8027047F8
:100E500080B5DFF8F4020068C00702D5FFF7F5FFA0
:100E600001E0DFF8D402DFF8E412096801F00F01B5
:100E7000491CB0FBF1F002BD80B5DFF8D402006878
:100E8000C00702D5FFF7E1FF01E0DFF8AC02DFF8B1
:100E9000C412096801F00F01491CB0FBF1F002BD5A
:100EA00080B5DFF8B4020068C00702D5FFF7CDFFB8
:100EB00001E0DFF88402DFF8A412096801F00F01F5
:100EC000491CB0FBF1F002BD80B5DFF89402006868
:100ED000C00702D5FFF7B9FF01E0DFF85C02DFF8D9
:100EE0008412096801F00F01491CB0FBF1F002BD4A
:100EF00080B5DFF874020068C00702D5FFF7A5FFD0
:100F000001E0DFF83402DFF86412096801F00F0134
:100F1000491CB0FBF1F002BD80B5DFF85402006857
:100F2000C00702D5FFF791FF01E0DFF80C02DFF800
:100F30004412096801F00F01491CB0FBF1F002BD39
:100F4000DFF808120A68120900F00F0050EA0210D8
:100F500008600868C003FCD47047DFF8F8110A681D
:100F6000120900F00F0050EA021008600868C00380
:100F7000FCD47047DFF8E4110A68120900F00F0092
:100F800050EA021008600868C003FCD47047DFF81C
:100F9000D4110A68120900F00F0050EA021008602C
:100FA0000868C003FCD47047DFF8C0110A68120952
:100FB00000F00F0050EA021008600868C003FCD47B
:100FC0007047DFF8B0110A68120900F00F0050EA0C
:100FD000021008600868C003FCD4704780B50E2872
:100FE00034D8DFE800F01E080B0F1215181B1E2165
:100FF00024272A2D30004FF4004002BDDFF82801DD
:10100000006802BDBDE80140DBE6BDE80140C8E67E
:10101000BDE80140D4E6BDE80140D3E6BDE80140AB
:10102000F2E6DFF8140102BDBDE8014010E7BDE8BB
:10103000014021E7BDE8014032E7BDE8014043E758
:10104000BDE8014054E7BDE8014065E740F26112A8
:101050000FF238110FF22810F7F76EFF0020C0468C
:10106000C046002002BD000080B5401F09282BD8D3
:10107000DFE800F0050A0E2A12161A1E222608467C
:10108000FFF7B4FE012002BD0846FFF7B0FEF9E706
:101090000846FFF7CDFEF5E70846FFF751FFF1E7F9
:1010A0000846FFF75AFFEDE70846FFF763FFE9E759
:1010B0000846FFF76CFFE5E70846FFF775FFE1E735
:1010C0000846FFF77EFFDDE74FF4C9720FF2BC015F
:1010D0000FF2AC00F7F730FF0020C046C0460020FA
:1010E00002BD10B5DFF89040217800290CD040F205
:1010F000A1120FF298010FF28800F7F71DFF0020F0
:10110000C046C046002010BDDFF87010002803D094
:101110004FF040520A6001E000220A6000F0ACFC8F
:101120000120207010BD000008670300000110407E
:10113000001010400018104000007701041010400B
:101140000418104000EA32060410604004186040A1
:1011500008106040081860400C1060400C18604097
:101160001010604010186040141060401418604067
:1011700018106040181860407CDA03000008104026
:101180005B455D25732C2025640A0000443A5C50C1
:101190006572666F7263655C53454E534F525F5381
:1011A0004C4F434154494F4E5F494E4E4F565F316D
:1011B0003731365F38415C434F4E464944454E54C3
:1011C00049414C5C53656E736F724875625C4D416A
:1011D00053535F50524F4A4543545C50524F445C06
:1011E0004135315C545C706C6174666F726D5C6526
:1011F00078796E6F73393631305C6669726D7761FC
:1012000072655C6F735C706C6174666F726D5C6547
:1012100078796E6F735C7372635C636D755C636D1C
:1012200075447276393631302E630000012100F0AA
:101230001F0291402E4A400942F8201070470121B8
:1012400000F01F0291402B4A400942F820107047DD
:1012500080B529484FF0FF31016001631320FFF78B
:10126000EEFF1320BDE80240E0E7244901222028D8
:1012700003D202FA00F008607047203802FA00F04A
:1012800008637047202804D2C2081D4B03EB82027A
:1012900004E02038C2081B4B03EB820201F00F016F
:1012A00000F00700800001FA00F01060704730B4D1
:1012B00000210846144A1368044606E01D46E5402E
:1012C000ED0701D520460121641C202CF6D300290E
:1012D0000BD1136B002406E01946E140C90701D584
:1012E00004F12000641C202CF6D330BC70470000B1
:1012F00000E100E080E200E05C02674058026740E5
:1013000068026740980267407C026740F8B5002495
:101310000FF240061BE0C4EBC405AF197978A85D55
:10132000F7F78CF8B978A85DF7F7AFF8F978A85D0A
:10133000F7F7D2F83979A85DF7F7F4F87979A85D6D
:10134000F7F703F9B979A85DF7F7D9F8641C082C09
:10135000E1D3F1BD0B0201000300000C0201000308
:101360000000000201030303000102010303030064
:1013700002020101030100030201030303001C0F29
:1013800000000200001B0F000002000038B500241E
:1013900009E00E4800EBC4014A79097950F834009D
:1013A00000F08EFB641C022CF3D300240AE00748F3
:1013B00000EBC40569692869FDF702FC2869FDF79F
:1013C000FDFB641C022CF2D331BD00BFDC630300C3
:1013D000F8B5002510E0052E00D10E242046C0B23D
:1013E000FDF75CFB79698900B0FBF1F0411E2046F6
:1013F000C0B2FDF766FB6D1C012D28DA0FF26C0000
:10140000E42101FB05077E6801220221304600F03D
:1014100057FB002803D00FF23800F7F78DFD39464F
:101420002846F7F777FB002E01D10724D6E7012ED7
:1014300001D10A24D2E7022E01D10B24CEE7032EDC
:1014400001D10C24CAE7042EC5D10D24C6E7F1BD95
:101450005B455D0A4552524F5220737069426F617D
:101460007264496E69742121210A000000000000A5
:10147000000000000000000000000101000000006A
:1014800000127A0000127A00000000000000000044
:10149000000000000000000000000000000000004C
:1014A000000000000000000000000000000000003C
:1014B000000000000000000000000000000000002C
:1014C000000000000000000000000100000000001B
:1014D000000000000000000000000000000000000C
:1014E00000000000000000000000000000000000FC
:1014F00000000000000000000000000000000000EC
:1015000000000000000000000000000000000000DB
:1015100000000000000000000000000000000000CB
:1015200000000000000000000000000000000000BB
:1015300000000000000000000000000000000000AB
:10154000000000000000000000000000000000009B
:1015500000B5ADF2D47D00A84FF4FA61F0F7FEFFBC
:1015600006E04FF4FA6300AADFF8640300F04FF9D5
:101570004FF4FA6100A800F0C9FD01281BDB40F21E
:1015800045318842EDD040F2454188420BD047F2C8
:101590000A118842ECD14FF4FA6300AADFF8300355
:1015A00000F0ACF9E4E74FF4FA6300AADFF8200397
:1015B00000F0FAF9DCE70DF2D47D00BD2DE9D0038F
:1015C0000446DFF81083DFF81093A8FB046709FBDB
:1015D0000477DFF80803E0FB0167DFF80403DFF8B6
:1015E000041330187941DFF80033A3FB0223801A7B
:1015F0009941BDE8D00370472DE9F04186B004461B
:101600000D4616461F4600208DF8150001208DF866
:1016100014000020ADF81000002F06D01820ADF8FF
:101620000E0000208DF80C0005E00220ADF80E0041
:1016300001208DF80C004FF47A70684302908DF809
:10164000124070008DF81300102202A940F265408C
:1016500000F0EBFC8046019700962B4622460FF2E5
:1016600064310FF27030F7F767FCB8F1010F01DB5E
:10167000012000E0002006B0BDE8F08194494860F8
:101680007047934988607047914908607047904956
:10169000C860704700208E494860704700208C4920
:1016A0008860704700208A49086070470020884998
:1016B000C860704786494A68002A01D0002801D5D1
:1016C000002070470246521E9241D20F8A750122B5
:1016D0000A750861887D002804D000231A4601217C
:1016E000104689E700231A460969104684E77848BE
:1016F0000021817501750161417D00230A4618466C
:101700007AE701460020724A1368002B07D0517512
:10171000117D002903D1517D03460A466CE77047CD
:1017200038B504466A4DE868002801D1002032BD72
:101730002346224621460120FFF75EFF002800D005
:10174000EC7532BD38B50446614DE87D044202D0E7
:101750000120FFF7E5FF2046401E8041C00F8DF8B5
:101760000000012200A94FF4A26000F05EFC0128F5
:1017700000DB2C76012801DB012032BD002032BDC8
:1017800053480021016041608160C16081754175ED
:10179000012101760021C17500F069BD70B40022FD
:1017A0009FED4A0A134690F9044002E041F82220D6
:1017B000521CA242FADB012C27DB1A461FE051F82B
:1017C000245005EB850600EB8605D5ED030AB4EE43
:1017D000600AF1EE10FA02D5B0EE600A2346641CEE
:1017E00090F90450AC42EADB51F8224051F8235002
:1017F00041F8225041F823409FED340A521C90F9E1
:101800000440A24201DA1446EAE770BC704730B5E2
:101810008FB004461546002C54D0002D52D02879A4
:1018200000F03F003F284DD1E868F7F797FB4FF4F1
:1018300003722E4BF4F7D4FCCDE900012869F7F7C9
:101840008DFB6FF0E7022A4BF4F7CAFCCDE90201E9
:101850006869F7F783FB0022264BF9F755FACDE9C3
:101860000401688BF7F784FB0022234BF9F74CFA4D
:10187000CDE90601A88BF7F77BFB00221D4BF9F79A
:1018800043FACDE90801288B0C906A79A968E888A9
:10189000FFF794FECDE90A01207D002805D061689C
:1018A00008000AD000A8884707E0607D002804D01F
:1018B0002168080001D000A88847A07D002801D039
:1018C000FFF715FF0FB030BD000000000000000062
:1018D0008CD60300000029F90F26020040420F00B9
:1018E000000087C14F88620400CA9A3B0080663EB0
:1018F000FF7F763E000024400000594070B5ADF5F2
:10190000A16D04461546A06800284AD0002D48D095
:101910000026FFA908312846FFF740FF3046009017
:1019200036E0FFA8083050F8260000EB800105EBF8
:10193000810090ED030AB5EE400AF1EE10FA26DDC3
:1019400000A9009A01EB021181ED020A017A00AAB6
:10195000009B02EB03121171417A00AA009B02EB7B
:101960000312517100A9009A01EB021102690A6188
:1019700000A9009A01EB02114269CA60807A00A9AD
:10198000009A01EB021188710098401C0090761CAF
:1019900095F904008642C4DBA168080001D000A8C4
:1019A00088470DF5A16D70BDC168080009D0002AF7
:1019B00007D0080005D01278501E8041C043C00FE8
:1019C0000847704773656E644C6F636174696F6E2E
:1019D000526571005B495D5B202573205D20696461
:1019E0003A257520726174653A256C6920706173BF
:1019F000736976653A257520617661696C3A25755B
:101A00000A00000000F041B800F046B800F04EB8FF
:101A1000000000000349044A096801B91146801A10
:101A20004018704770DA03000000030003B4DDE9DA
:101A30000023C3F30A5140F2FF72914206D001B174
:101A40000CE0190350EA113006D00BE0190350EAFC
:101A5000113014BF0220012002B070474FF0FF3058
:101A600002B070476FF0010002B0704720210903F7
:101A700026311820ABBEF9E70F49002802D07F209D
:101A8000086070470020086070470C490A68C00071
:101A900052EAD0000860704708490A6802F06042C4
:101AA000C043C00052EAD000086070470348006895
:101AB000C000C00870470000040111402804114014
:101AC00038B504460D462B460C2C03D2052B01DA03
:101AD000022A0ADB009222460FF224010FF22800AC
:101AE000F7F72AFA6FF0150032BD00F0DAFD002892
:101AF00002D102482554002032BD0000ECD9030079
:101B00007573694F70656E005B455D25732C2069A8
:101B10006E76616C696420706172616D6574657266
:101B2000202825642C2025642C202564290A000007
:101B3000F0B591B004460D46002600AF17E0DFF87F
:101B4000C405335D1B111B5C3B70335D03F00F0359
:101B5000185C07F8010F761C002007F8010F491CDC
:101B60009142ECDB00A90FF27860F7F7E5F9AE429D
:101B700005DAAA1B212A00DB20220021F0E711B0A0
:101B8000F0BD01684A1C02600878704701688A1C31
:101B900002600878497840EA0120704701680A1D10
:101BA000026008784A7840EA02208A7840EA0240D7
:101BB000C97840EA0160704781B001680A1D02607F
:101BC00008784A7840EA02208A7840EA0240C978D8
:101BD00040EA016000909DED000A01B0704713B526
:101BE0000446012201A92068F0F770FC2068401C1F
:101BF0002060012016BD13B50446022201A9206809
:101C0000F0F764FC2068801C2060022016BD13B52C
